:020000040000FA
:10000000C0070000D1060000D1000000B1060000CA
:1000100000000000000000000000000000000000E0
:100020000000000000000000000000005107000078
:100030000000000000000000DB000000E500000000
:10004000EF000000F9000000030100000D010000B6
:1000500017010000210100002B0100003501000004
:100060003F01000049010000530100005D01000054
:1000700067010000710100007B01000085010000A4
:100080008F01000099010000A3010000AD010000F4
:10009000B7010000C1010000CB010000D501000044
:1000A000DF010000E9010000F3010000FD01000094
:1000B00007020000110200001B02000025020000E0
:1000C0001FB5C046C04600F0EFFA04B00FB41FBD24
:1000D00008205A49096809580847382057490968CB
:1000E000095808473C2055490968095808474020E5
:1000F0005249096809580847442050490968095875
:10010000084748204D490968095808474C204B4981
:10011000096809580847502048490968095808479C
:100120005420464909680958084758204349096836
:10013000095808475C204149096809580847602068
:100140003E4909680958084764203C49096809582C
:100150000847682039490968095808476C20374919
:100160000968095808477020344909680958084740
:100170007420324909680958084778202F490968CE
:10018000095808477C202D490968095808478020EC
:100190002A490968095808478420284909680958E4
:1001A0000847882025490968095808478C202349B1
:1001B00009680958084790202049096809580847E4
:1001C00094201E4909680958084798201B49096866
:1001D000095808479C201949096809580847A02070
:1001E0001649096809580847A4201449096809589C
:1001F0000847A8201149096809580847AC200F4949
:10020000096809580847B0200C4909680958084787
:10021000B4200A49096809580847B82007490968FD
:1002200009580847BC2005490968095808470000D3
:1002300003480449024A034B7047000000000020B5
:10024000C0070000C00700000122D84B5A6000BF61
:10025000D74A1268002AFBD0016000BFD44A126856
:10026000002AFBD00022D14B5A6000BFD04A12684E
:10027000002AFBD07047F0B505460E46174600240D
:1002800006E0A200B158A2005019FFF7DDFF641C80
:10029000BC42F6D30020F0BD0120C043C549086030
:1002A000401048607047014601229204086890425D
:1002B00001D9102070470020FCE7F0B505460C4638
:1002C0001646002706E028462168FFF7BDFF2D1DD2
:1002D000241D7F1CB742F6D3F0BD70B505460C4611
:1002E0002E460BE0304600F075F9FF2C01D80024B3
:1002F00001E0FF3C013C012080023618002CF1D1C6
:1003000070BD0146012212044868904201D90920BB
:100310007047A9484069401C01D10F20F8E7002030
:10032000F6E7FEB504462068030000F037FA05043E
:100330002B4249598B00201DFFF7E3FF0546002D96
:1003400001D02846FEBDFFF7A7FF0120C00200F044
:1003500041F9042221469948FFF78DFF002801D07A
:100360000320EFE708222146944800F06DF90028A9
:1003700006D1002192480068FFF766FF00F00CF9F3
:100380000320DFE7A768E6686068019031463846D9
:10039000FFF7A3FF324638460199FFF78EFFB20000
:1003A0003846019900F050F9002800D1CAE703202F
:1003B000C8E700F0E3F9834800688349086041E03A
:1003C00060680190E668A0680090B200009901980A
:1003D00000F03AF90746002F00D1B3E70E20B1E74D
:1003E000201DFFF760FF0546002D01D02846A9E734
:1003F0006068002807D1FFF74FFF0320800200F05C
:10040000E9F800F0C9F8FFF747FF0120C00200F04B
:10041000E1F8042221466948FFF72DFF002801D0AA
:1004200003208FE708222146644800F00DF90028D8
:1004300006D1002162480068FFF706FF00F0ACF823
:1004400003207FE700BF00207CE770B505460C461F
:10045000182D04D12068FFF764FF206002E001201E
:10046000206000BF00BF70BDF0B589B05248406940
:1004700003905248806881000398081802900398FE
:10048000000B01900121090302984018401E000B47
:1004900000900124002520462946019A00F0C4F866
:1004A0000022401E91410791069001260027304608
:1004B0003946009A00F0B8F80022401E914105919B
:1004C0000490049BDB43059AD2430698184307998E
:1004D00011430791069037490698086007984860CD
:1004E00009B0F0BD70B53448446934488568466841
:1004F000AA003146204600F0A7F8002801D00020CD
:1005000070BD0120FCE72D484068002801D0012083
:1005100000E000200546FFF7E5FF002807D0FFF7C1
:10052000BBFE0320800200F055F800F035F8FFF71D
:100530009BFF002D0ED020484669204884684768FC
:1005400021463046FFF7C9FE224639463046FFF7BE
:10055000B4FE00BF00F020F810B5184844681A48EF
:100560000460204600F0DCF810BD15480068006803
:10057000401C01D100BFFEE710480068002802D0EF
:10058000042806D101E0FFF7BEFFFFF7E5FF00BF3B
:10059000FEE700BF00BFFEE7BFF34F8F0B480C49DB
:1005A000C860BFF34F8F00BFFEE7000000E50140C9
:1005B00000E40140000600400010001000080000A8
:1005C000B8070000BC070000000000200400FA0586
:1005D00000ED00E010B50146104B1A6808460223F2
:1005E0000F4C636000BF0F4B1B68002BFBD0531CEC
:1005F00004D0904202D20A4B186101E0084B986087
:1006000000BF084B1B68002BFBD00023044C636029
:1006100000BF044B1B68002BFBD010BD0010001066
:1006200000E5014000E4014010B5202A04DB01464A
:10063000203A9140002010BD914020239C1A03468F
:10064000E3401943904010BD034610B50B439B0790
:100650000FD1042A0DD308C810C9121FA342F8D025
:1006600018BA21BA884201D9012010BD0020C04328
:1006700010BD002A03D0D30703D0521C07E000208E
:1006800010BD03780C78401C491C1B1B07D1037854
:100690000C78401C491C1B1B01D1921EF1D118463D
:1006A00010BD70477047704710B500F007F810BDD7
:1006B000014B1B68DB6818470000002019481A49E5
:1006C0007047FFF7FBFFFFF7FBFC00BD20BFFDE716
:1006D0001649174C24688C420BD1164B1B68994263
:1006E0000CD1154B154A1360186810498842EDD09B
:1006F0000AE0134880F30888124B18470F4A13602A
:1007000018680A498842E1D080F308880E49884277
:1007100004DD0E48026802210A4302605B68184744
:100720000346DFE7C0070000C0070000FFFFFFFF30
:10073000000C000014100010001000000000002049
:10074000000400206B05000000200020240500406C
:100750000D48704502D1EFF3098101E0EFF3088104
:10076000886902380078182802D1C046074A104725
:10077000074A12682C3212681047000000B5054B7A
:10078000054A9B58984700BDFDFFFFFF4B04000042
:1007900000000020001000000400000030B4744687
:1007A000641E2578641CAB4204D3635D5B00E318D0
:1007B00030BC18471D46F8E7000C00000010000090
:10100000D010002005A401007192000077A3010018
:1010100000000000000000000000000000000000D0
:1010200000000000000000000000000075A40100A6
:1010300000000000000000007192000071920000AA
:10104000E1A40100E7A40100719200007192000088
:101050007192000071920000719200007192000084
:10106000EDA401007192000071920000F3A4010050
:1010700071920000F9A40100FFA4010005A5010080
:101080007192000071920000719200007192000054
:101090007192000071920000719200007192000044
:1010A0000BA5010011A501007192000071920000D2
:1010B0007192000071920000719200007192000024
:1010C00000F002F819F07FF90CA030C80838241895
:1010D0002D18A246671EAB4654465D46AC4201D170
:1010E00019F071F97E460F3E0FCCB6460126334209
:1010F00000D0FB1AA246AB4633431847A495010023
:10110000C49501000023002400250026103A01D3D5
:1011100078C1FBD8520700D330C100D50B607047AF
:101120001FB5C046C04619F0F6F804B00FB41FBD95
:1011300082690249816102481044704745110000EC
:101140000100000001B41EB400B510F044F901B470
:101150000198864601BC01B01EBD0000F0B44046B7
:10116000494652465B460FB402A0013001B506481D
:10117000004700BF01BC86460FBC804689469246A8
:101180009B46F0BC70470000C110000070B50546DA
:101190000C46164602E00FCC0FC5103E102EFAD2B8
:1011A000082E02D303CC03C5083E042E07D301CC7E
:1011B00001C5361F03E021782970641C6D1C761E62
:1011C000F9D270BD70B50546F74C08202070A01C00
:1011D00000F03BFA5920A0802946204606F070FB1B
:1011E00070BD10B506F075FBEF490020891E087030
:1011F00010BD70B5EC4D0C46AD1E297801260029B6
:101200002ED06038030019F0CBF9532F383D4348F6
:101210004E53575D62F1F1F1F1F1F1676C70777B3C
:101220007E848A8F94989CA0A7ACB2BAC1C8F2F809
:10123000FFEDECEBEAE9F1F1F1F1F1E8E7E6E5E4E5
:10124000E3E2E1E0DFF1F1F1F1F1F1DEDDDCDBDA47
:10125000D9D8D7D6D5D4D3D2F1F1F1D1D0CFF100AE
:10126000602801D0D1489AE103CC083C06F085FC07
:101270002060002800D12E7070BD03CC083C06F021
:10128000F5FC8CE12088616880B206F04FFC86E1B5
:1012900003CC083C06F071FD81E12078A26861680A
:1012A00006F07DFD7BE107CC0C3C06F093FD76E17A
:1012B000206806F0A8FD72E12088616880B206F01F
:1012C000C0FD6CE103CC083C06F0CFFD67E103CC28
:1012D000083C06F0E6FD62E12078616801F070F9F3
:1012E0005DE1206801F0BAF959E1237B2179A26818
:1012F000206801F0C3F952E1206801F05EFA4EE186
:1013000000F083FF4BE12088616880B201F07AFB36
:1013100045E12088217980B201F0F0FB3FE120789F
:1013200040B201F0F9FB3AE1208880B201F046FFBB
:1013300035E1206801F054FF31E1206801F0E1FE61
:101340002DE1206801F00AFF29E1208982B203CC57
:10135000083C01F05DFF22E103CC083C01F0A6FF50
:101360001DE12088616880B202F0A3FF17E12088A8
:10137000217980B2E368A26803F08AF80FE120883F
:10138000217980B2A26803F025FA08E12088A268DA
:1013900080B2616803F09AFA01E1211D0EC920882C
:1013A00080B203F000FBFAE0F3E0EDE0E7E0DFE01D
:1013B000DAE0D2E0C8E0C1E0B7E0B0E0A7E09EE04C
:1013C00096E08EE085E07EE070E069E060E056E067
:1013D0004EE072E046E03FE038E02FE028E024E015
:1013E0001EE01AE015E00FE007E000E0D9E02088F9
:1013F000616880B203F017FBD1E02088227A21795E
:1014000080B201F095FBCAE0208880B201F095FB24
:10141000C5E0206801F098FBC1E000F0DAFEBEE014
:1014200007CC0C3C01F007FCB9E000F0BBFEB6E0D5
:101430002088616880B201F0AEFCB0E0A088A268AC
:1014400081B2208880B203F080FFA8E02088616824
:1014500080B203F0B6FFA2E02088616880B203F09A
:10146000BCFF9CE02088616880B203F0C3FF96E077
:101470002088A26880B2616803F0CFFF8FE02089E6
:1014800082B2A08881B2208880B203F0CFFF86E0CC
:101490002089616882B2208880B203F0E6FF7EE096
:1014A0002088616880B203F0F2FF78E0A08881B202
:1014B000208880B204F047F871E02088616880B22B
:1014C00004F04CF86BE02078A268616805F0C7FB77
:1014D00065E0A088A26881B2208880B205F0CEFBCA
:1014E0005DE0211D0EC9208880B205F0CBFB56E0DF
:1014F0002088A26880B2616805F0E0FB4FE0A08818
:10150000A26881B2208880B205F0EDFB47E0A08898
:10151000A26881B2208880B205F028FC3FE02088D4
:10152000616880B205F069FC39E0208982B2A08848
:1015300081B2208880B205F06AFC30E020886168C2
:1015400080B205F087FC2AE02089E36882B2208817
:10155000616880B205F0F8FC21E0211D0EC92088E9
:1015600080B205F0E5FD1AE0206805F07AFE16E08D
:101570002088A26880B2616805F07EFE0FE02088B6
:1015800080B207F09CF90AE0208880B207F0B6F933
:1015900005E02088A26880B2616807F0C0F9206089
:1015A00070BD266070BD00000A0000200130000000
:1015B0008307FF22DB0E9A408907090E9940002815
:1015C0000BDA0007000F0838830827489B0018181B
:1015D000C36993430B43C3617047830823489B004F
:1015E0001B181868904308431860704710B50446EC
:1015F00000210120FFF7DCFF00211820FFF7D8FFB2
:1016000000210B20FFF7D4FF02211920FFF7D0FFA4
:1016100002210D20FFF7CCFF02210E20FFF7C8FFAB
:1016200002210F20FFF7C4FF0221C81FFFF7C0FFF0
:1016300003211620FFF7BCFF03211520FFF7B8FF99
:101640002046FFF7BFFD002010BD782101807047C4
:1016500010B5FFF7C6FD10BD0548704710B5FFF780
:10166000C8FD10BD7047704700ED00E000E400E0E9
:1016700003F9004330B5FA4D044610280BD0112C65
:1016800007D028468178122C08D0132C0BD018F0E4
:101690006CFEAC7030BD18F068FEFAE71129F8D086
:1016A00018F063FEF5E71129F3D018F05EFEF0E7BD
:1016B00010B5EB4994B0C878002816D017206A46B8
:1016C000107000A806220230091D18F0C4FC09A9F8
:1016D000684609F04CFE0446112803D0002C01D0C6
:1016E00018F043FE204614B010BD3220E7E710B5D5
:1016F00002210CF071F910BDFFB595B01D460E46E4
:101700000746FFF7F4FF04000AD02078222804D30C
:10171000A07F8006C00FA84204D1082019B0F0BDF8
:10172000D048FBE73721684601704780002D05D07F
:101730000121017146711799817102E0002069460B
:10174000087109A9684609F012FEA07FDF21084050
:1017500069010843A0770020E0E730B50446084659
:1017600020380D46030018F01BFF0A06090F202839
:101770002E3C42484E5418F0F8FD4CE020782028CA
:1017800049D118F0F2FD46E0B5480178032942D06E
:10179000807813283FD0207824283CD025283AD0C0
:1017A000232838D018F0E1FD35E02078222832D007
:1017B000232830D818F0D9FD2DE0207822282AD00F
:1017C00018F0D3FD27E02078222824D0242822D026
:1017D000262820D027281ED029281CD018F0C5FD87
:1017E00019E02078252816D018F0BFFD13E02078E6
:1017F000252810D018F0B9FD0DE0207825280AD052
:1018000018F0B3FD07E02078282804D018F0ADFDCB
:1018100001E018F0AAFD257030BD30B5924C0B8860
:10182000924A022801D0934204D09D1FA54225D29E
:10183000022802D04D88954203D04D88AD1FA542A5
:101840001CD24C88A34219D88B88FF25F435AB42B3
:1018500014D8022802D0C888904205D0C888824D8A
:101860000A382D1FA84209D2C888904208D0944255
:1018700006D05B1C63438000834201DB072030BD40
:10188000002030BDF0B57A49884242D37A4A794D7A
:101890001368A84201D398423BD30279002A06D0AC
:1018A000082A02D8067B082E05D90720F0BD047B44
:1018B000002CFAD0F6E7002A06D004688C4228D320
:1018C000AC4201D39C4224D3002E06D084688C42C3
:1018D0001FD3AC4201D39C421BD300240BE005680C
:1018E000A700ED598D4214D3624FBD4201D39D42F2
:1018F0000FD3641CE4B2A242F1D800225D4D0CE08B
:1019000084689700E4598C4203D3AC4203D39C42D1
:1019100001D21020F0BD521CD2B29642F0D8002065
:10192000F0BD10B50289554B111F994213D2418960
:10193000042910D3DB1C99420DD891420BD80178B1
:10194000890706D54068002803D0FFF79BFF0028D1
:1019500000D1002010BD072010BDFFB50022099B5B
:10196000002802D0994205D858E0002902D1002071
:1019700004B0F0BD0920FBE7845C002C12D087186E
:101980007D78112D43D010DC2B0018F009FE0A40A1
:101990001726262C2C2E2E363640835C002B30D179
:1019A000521CD2B28A42F8D3E1E71C2D2FDA123D45
:1019B0002B0018F0F5FD042C2C121A2C022CD9D176
:1019C000BB78039C072B237001D25B0701D40A204C
:1019D000CEE7029B01241B7816E0E343DB0708E017
:1019E000012C08D013E00620C2E70F2523072D079E
:1019F0005B19002BF4D03046BAE7029B1B789C079A
:101A000001D50B20B4E702242343029C2370835C9E
:101A1000521C9A18D2B28A4202D9ABE71926760232
:101A20008A42A9D3A3E710B504780B46002C08D04E
:101A30000121134A012C07D0022C0BD0032C25D1F5
:101A400020E00021197023E01970817989090329A8
:101A50001CD11DE0197081798909012916D117E07F
:101A6000A8010020023000007B0C0000FFFF0000F6
:101A700000B00100000000201C000020FD3F00001D
:101A80000232000019708179890901D0104610BD19
:101A9000411C0622581C18F0DEFA002010BD08B5C3
:101AA0001346002806D0FDA00068009048796A46D9
:101AB0008009105C18700622581C18F0CCFA08BD7A
:101AC00030B50C46097895B0222902D2082015B00D
:101AD00030BD282369460B704880132A03D03B2A67
:101AE00001D00720F3E708460A7109A909F03FFC75
:101AF000050003D121212046FFF72FFE2846E6E707
:101B000000B595B0232369460B7048801088888003
:101B10005088C880D08848819088088100208881BA
:101B2000C88109A9684609F022FC15B000BD70B54E
:101B30000E46050003D0002109200FF040FE0120D1
:101B4000D74C022EE0701DD0032E01D018F00DFCF2
:101B50000621201D0FF07EFB607A8006800E6072E9
:101B6000FFF7A6FD608A00280BD0002D09D0830066
:101B70000122002109200FF092FD092801D018F060
:101B8000F4FB70BD0321E01D0FF064FB607A40217F
:101B90008006800E08436072E01C02F027FBDFE73E
:101BA000F0B585B002216846BD4E0171F18AC18051
:101BB000002756E001A80BF076FE050007D0F08A5A
:101BC000002854D00020F0826946C88047E0039C7A
:101BD0002078212843D0A07F01072AD52046223033
:101BE000009068462346628E00892146343301F016
:101BF00014FD050004D011282AD018F0B6FB27E008
:101C0000A07FF7210840A077E17F480889074000BE
:101C1000C90F084341072020005D490FC000014360
:101C2000E1772078282824D129212046FFF795FD47
:101C30001FE0400713D568462246008921460E3230
:101C4000FFF75EFF050005D0112801D018F08DFBCD
:101C500000250EE0A07FFB210840A07709E07F1C53
:101C6000FFB202200BF061FE401CB842A2D8052D45
:101C700007D06846C088F082052D04D0284605B0FC
:101C8000F0BD0020F0820020F9E7FEB5040001D18C
:101C900018F06BFB72202070606808250178804E78
:101CA000091F0B0018F07CFC11FE0A0C53F90C0DF7
:101CB000F9F9380C0C0C0CFE79FE0C0018F055FBF1
:101CC000FEBD80880090FFF712FD070001D118F0DB
:101CD0004CFB6078042128436070307D08433075E8
:101CE00021213846FFF739FD009806F0CAFB00981D
:101CF00003F0B6F9009804F085F9022000990FF07E
:101D00005EFDB87FEF210840B877FFF749FF002854
:101D1000D6D018F02AFBFEBD86883046FFF7E7FCD8
:101D2000002801D118F021FB60688078012801D0DB
:101D300018F01BFB60688179304606F0D5FC00285E
:101D4000E9D06178294361706168C880FEBD8788E9
:101D50003846FFF7CCFC060001D118F006FB60788E
:101D60003946284360706068C088308160680089A7
:101D7000708160684089B08102200FF020FD002052
:101D8000B075B07F8007800F0228DFD1FFF708FF12
:101D90000028DBD018F0E9FAFEBD80783C2803D09B
:101DA000002702280FD000E0012700210091002821
:101DB00005D03C2803D0022801D018F0D6FA0098AC
:101DC000002802D07EE00121F0E7607828436070AF
:101DD000307D28433075002F67D1606802218788E5
:101DE000009738460BF0F0FD0546032138460BF00E
:101DF000EBFD0290052138460BF0E6FD0190042131
:101E000038460BF0E1FD0746002D01D118F0ADFA80
:101E10000298002801D118F0A8FA0198002801D1F1
:101E200018F0A3FA002F01D118F09FFA22212846BA
:101E3000FFF793FC60688079012834D00227A87FDF
:101E40000622800880003843A8776068C08A28810D
:101E50006068008B68816068408BA8816068C07989
:101E6000E875616828461830083118F0F4F86068A1
:101E70000622807B68706168A81C0F3118F0EBF8AF
:101E8000A87F8107890F009806F0DEFA012F0CD099
:101E9000022F17D018F069FAFEBD20E00302FF01FF
:101EA000A80100201FE00127C9E73078032801D0EE
:101EB00018F05BFA002108460FF081FC012000F0C9
:101EC00096FFE9E7B078132801D018F04EFA002108
:101ED00007200FF074FC1120FFF7CCFBDCE7204655
:101EE00001F015FED8E7607828436070D4E7F7B5B5
:101EF00005460078002700090C463E4601287DD0A3
:101F00000022F94902287AD007280BD00A2877D076
:101F100018F02BFA0298002C068001D027806680EA
:101F20000020B9E7686803780D2B38D006DC042B55
:101F300067D0072B3DD00A2B62D106E0122B3FD091
:101F4000132B47D0142BF7D1C2E011270726002C02
:101F50007ED08088A0806968FB238979A171E349DC
:101F600005460A7D1A400A7504210BF040FD052143
:101F700028460BF03CFD002128460BF038FD0121DE
:101F800028460BF034FD032128460BF030FD0221DA
:101F900028460BF02CFD284609F029FBBAE701275B
:101FA0000926002CD4D08088A080686880792072AF
:101FB000B0E712270E268088214600F03EFFA9E7F1
:101FC0001A270726002CC3D04088A08068680079B3
:101FD000A0719FE781783C293FD010271E26002C56
:101FE000B6D08088A0806868C08A20836868C08A6C
:101FF000E0826868008B6083686803E077E0A1E0B6
:10200000C4E034E0408BA0836968607D497F40086C
:10201000C9074000C90F084360756968C007497F58
:10202000C00F49084900084360756968A21DC87956
:102030000831FFF734FD69682246887B0D320F3185
:10204000FFF72DFD68688079002804D0012000E0AA
:1020500077E0207506E00220F9E719270726002C13
:102060006FD0A271A148F722017D11407CE01B27AF
:102070002E26002C65D0A1806968A21D0879491D13
:10208000FFF70DFD68682030C07A60736868C0781B
:102090000428A07B19D040084000A073F921084013
:1020A00069681F22C9788907490F0843A0736968C6
:1020B0004007C97A400FC9000843A07369682046E9
:1020C0000F300C3117F0C7FF24E701210843E4E784
:1020D0001E270E26002C62D0A1806868E21D407A7F
:1020E000A07169688878C91CFFF7D9FC12E7287EBF
:1020F000012804D0022814D018F037F90AE71D2768
:102100000E26002C4BD06888A080A88BE080E88B3E
:102110002081288C6081688CA0817448DF22017D39
:10212000A3E712270E26688800F087FE002C36D021
:1021300068784007400F0328C6D16C48FD22017D16
:1021400093E72CE0287E030018F02AFA060410100A
:102150002020202619270726002C20D0A1806348A4
:10216000A271017D490849000175D3E619270726A8
:10217000002C14D0A180287E012805D00320A07156
:102180005A48EF22017D70E70220F8E721462846F1
:10219000029A01F03AFE7FE618F0E7F8BAE60298F4
:1021A0000680BDE610B5514894B08078132802D05F
:1021B000082014B010BD22206946087009A968469D
:1021C00009F0D5F80446002107200FF0F8FA204660
:1021D000EFE700B5454895B08078122801D0082077
:1021E000A3E41E216846017000218170C17009A915
:1021F00009F0BDF80028F3D1002107200FF0DFFA25
:102200001120FFF737FA00208FE400B5374895B06A
:102210000078022801D0032818D11B2108A80173D7
:102220000021817369460BA809F0A1F8002804D1A8
:10223000684640781B2801D0032076E40021084638
:102240000FF0BDFA68468078002801D008206CE4C1
:10225000012000F0CCFD002067E4F8B5234C03001A
:1022600018F09EF90A066E176E6E6E6E39325F6E4A
:10227000FFF7CBFF002827D105F05FFA002823D015
:10228000222101700021017605F035FA207D01211F
:1022900043E08EB23046FFF72AFA050001D118F06C
:1022A00064F8287821280FD005F047FA00280CD0D0
:1022B000122101700227077646800020A87505F0DC
:1022C0001AFA207D38432075F8BD1322294630467E
:1022D000FFF7F6FBF8BDA578122D09D0132D0AD013
:1022E00018F043F8F8BD0000FFFF0000A80100202F
:1022F000FFF76FFF01E0FFF755FF0028F2D105F06F
:102300001CFA0028EED022210170122D07D00221E4
:10231000017605F0F0F9207D10210843D3E7012173
:10232000F6E7607A8109012908D0800901D018F008
:102330001CF803210020FFF7FAFBD3E70221F9E79D
:1023400018F013F8CEE7F7B514460D0001D118F0D8
:102350000CF828780827012804D0022819D018F092
:1023600004F899E50098FFF7C2F9060001D117F0CB
:10237000FCFF0220B0751030207060783843607028
:1023800007CD183407C4FE482022017D1143017592
:1023900082E50098FFF7ABF9060001D117F0E5FFE1
:1023A000A988F848814208D1EA88824205D11322DF
:1023B00031460098FFF784FB6EE5814202D1E88840
:1023C000002809D01220207060783843607007CD53
:1023D000183407C4002006E0782300220220009968
:1023E0000FF05DF90120B07556E530B50C46E649B1
:1023F00095B08C4238D3E649E44A0968944201D347
:102400008C4231D3203800220125030018F0C8F88F
:1024100006042741454B545C002108200FF0A9F920
:10242000002802D0112015B030BD24206946087064
:1024300000A80522A11C023017F00DFE09A968466C
:1024400008F095FF05002CD10823002211461846FC
:102450000FF025F9082824D017F087FF21E06068E5
:10246000002803D0884201D21020DCE73C216846D6
:102470000170218841806188818009A908F077FF77
:1024800005000ED1606800280BD06946098D0180D7
:1024900007E0206801F0E8FE02E0204600F0E1FCE1
:1024A00005462846BFE73D2007E0857000E08270C2
:1024B00009A908F05CFFF3E734206946087020782A
:1024C000C0076846F3D0F0E70720ACE730B50C460C
:1024D000AF4995B009688C4201D21020A3E720389B
:1024E000030018F05DF80504212123213200208823
:1024F000FFF7FDF8002804D00078222803D2082036
:1025000091E7A4488FE72521684601702188418022
:1025100009A908F02CFF050015D10AA905220231EE
:10252000A01C17F098FD0EE006250CE0206800289E
:1025300005D0884201D2102505E001F08AFE9048BE
:102540000025408AA08028466DE707206BE78C486D
:102550000A30704710B51821894817F0D9FD0120BD
:1025600000F045FC1120FFF785F8854C00206074D1
:10257000E12080006082211DE01C05F0AEF9E11C25
:102580000722C81D17F067FDFFF792F8002801D059
:1025900017F0EBFE00F03CFD01F07DFA10BD10B528
:1025A00004463C2117F0B4FDA07F80088000A0778E
:1025B000202020700020A0752034607010BD70476E
:1025C000FEB5064670480D46814206D36F488542E7
:1025D00005D36F480068854201D210205CE4684C46
:1025E000002E02D0012E31D125E00722E11C6846E1
:1025F00017F031FDE11C2846FFF715FA0028EDD150
:10260000FFF756F8070006D007226946E01C17F0CE
:1026100022FD384640E42878002801D0012805D161
:1026200057480722E11C0A3017F015FD0021092048
:102630000FF0C5F80FE00978002907D0012905D06F
:10264000022905D0032903D0534825E4072023E4B9
:102650000120FFF76CFA667400201DE410B54C49A8
:102660000968884201D2102010BD45490246CB7846
:10267000091D1846FFF713FA002010BDFFB599B0E9
:102680000546002008A908746946087108A908735E
:1026900008753F4814463C4A3C4900681E46002DD8
:1026A00005D095420BD38D4201D3854207D3002C30
:1026B00008D0944203D38C4204D3844202D2102027
:1026C0001DB0F0BD2846204318D01F270BAB0CAA25
:1026D000009728461A99FFF740F90028F0D10DAB72
:1026E00001AA314620460097FFF737F90028E7D1C5
:1026F00068460079C00703D00A20E1E70720DFE73A
:1027000002AF002D0FD01A20694608721A988872FD
:102710002946F81C1A9A17F09EFC0EA902A808F088
:1027200026FE0028CCD1002C0ED020216846017254
:10273000867232462146F81C17F08DFC0EA902A8BD
:1027400008F015FE0028BBD108A80D49007B487091
:102750000020B5E770B506460A200C4608701546FD
:102760001146204608F003FE002807D138212170C9
:102770002046294608F0FBFD002812D008280DE06D
:10278000A8010020FFFF000000B0010000000020B1
:102790001C000020023000000232000000D1F84886
:1027A00070BD2A462146304600F086FB04460828C4
:1027B00001D117F0DAFD204670BDF0B50446F1A155
:1027C00003C997B0F14A002715911490944210D391
:1027D000F048EF4B00689C4201D3844209D3217832
:1027E000012909D16168914203D3994204D38142FE
:1027F00002D2102017B0F0BDE74D2878012801D093
:102800000820F7E707200BF099F8002804D120787A
:10281000002806D0012804D0287D0107890F06D1A1
:1028200001E00420E6E7C10701D1800701D51120AE
:10283000E0E7208AD94A014620399142217807D31E
:1028400001297DD100287BD1618A002978D110E04F
:10285000022901D0032901D1A02871D3012908D070
:10286000CD494978C90704D0618A002968D0B429C4
:1028700066D82178002906D0012908D0022904D081
:1028800003295DD118E0002519E0022517E0002892
:1028900002D1608A00280DD00425606800780028E5
:1028A0000DD001280AD0022808D0032806D0B44849
:1028B000401E9FE70125F0E7032500E00127207A6D
:1028C000002806D0012806D0022806D0032860D1AF
:1028D00005E0002604E0012602E0022600E00326CF
:1028E000002D01D0022D15D1002E13D0E068002854
:1028F00003D0FEF7C7FF002894D1A748407880078F
:1029000002D09F48801E75E7022D03D1022E40D0D1
:10291000032E3ED0182168460170218A4180218A09
:10292000818085719C48C078002801D0012865D13C
:102930006946C8716846077221780930012900E0AC
:1029400027E020D0062117F0E3FB69460E74207DB6
:102950008207C107D20F4007C90F5200C00F1143B1
:102960008000014314A8405C6946C873002810D059
:1029700009A9684608F0FBFC00289AD1002D0AD06E
:10298000022D08D012E061680622491C17F063FB93
:10299000DBE707202EE7002E08D0E068002805D0EE
:1029A00009AA6946FFF7D6FE0028ACD11B2069466C
:1029B00008700120887009A9684608F0D8FC002832
:1029C000A1D108A840791B2818D12B0017F0E8FDE9
:1029D0000504040606040900032000E0022000F0BC
:1029E00006FA012D0CD0608A002809D0002283004D
:1029F000114610460EF053FE002801D00320F9E6E0
:102A00000020F7E6F3B5032683B00D46002909D070
:102A10005E48854270D35E48854203D35D480068B6
:102A2000854269D30398FEF762FE040005D0207842
:102A3000222804D2082005B0F0BD5948FBE7A07F4A
:102A40008707BF0F002D05D029463846FEF7E5FE63
:102A50000600F0D15048012F05D0022F19D017F0F1
:102A600084FC3046E7E7A27D2946012A02D0007D9A
:102A7000800701D51120DEE7002905D1684600F066
:102A80006DFB0028D7D16946039805F09DFD0646E9
:102A9000E7E7A17D022915D1007D800612D4002D23
:102AA00004D0A07F40070BD4002100E0012103984F
:102AB00005F0DDFD0600D4D1A075002DD1D003E0D6
:102AC0001126CEE7002D17D02A4621460398FFF79E
:102AD00017F806461128C4D1A07F4007C1D420466C
:102AE000082229460E3017F0B6FAA07F04210843C9
:102AF000A0770026B5E7FFE710209CE770B50C46ED
:102B00000546FEF7F4FD010004D022462846FEF7F4
:102B1000D7FF70BD224870BD00B595B0312269461F
:102B20000A70887009A9684608F021FC15B000BD3C
:102B300010B50123FEF7E0FD10BD002310B51A46C5
:102B40001946FEF7D9FD10BD70B504460F4894B084
:102B5000844206D30E48844206D30E48006884425D
:102B600002D2102014B070BD2046FEF7DAFE002815
:102B7000F8D109488178112914D00820F2E7000023
:102B800003320000070605040302010000B0010043
:102B9000000000201C000020A8010020E13F0000F0
:102BA00002300000017DC90601D51120DAE71D229F
:102BB00069460A7021780025CA07D20F69468A70D3
:102BC00022898A806289CA80217801268907CA0FF2
:102BD00069464A72C078002803D0012804D0032037
:102BE000C0E708460D7201E008460E7209A908F018
:102BF000BEFB0028B6D12078800708D56068002881
:102C000005D009AA6946FFF7A5FD0028AAD11E2113
:102C1000684601708670C57009A908F0A8FB0028F5
:102C2000A0D1A08900F0FAF804009BD11220FEF791
:102C300021FD204696E7F0B51646BF4A0C46050032
:102C4000BB48BC49126895B005D085420FD38D4270
:102C500001D395420BD3844209D38C4201D39442D1
:102C600005D3864203D38E4204D3964202D210206B
:102C700015B0F0BDB14F387DC106890F01D14007B5
:102C800001D51120F4E72046FEF74BFE0028EFD1D6
:102C900020788107C90F294303D0800703D5002D71
:102CA00001D00720E4E731460220FEF7B6FD0028F8
:102CB000DED1B878112803D0122801D00820D7E738
:102CC00006200AF03BFE002804D09C488078122899
:102CD00002D005E00420CBE7FFF77BFA0028C7D13C
:102CE0002078800708D56068002805D009AA6946C1
:102CF000FFF730FD0028BBD12121684601702189F2
:102D0000418061898180207800278007C10F684653
:102D1000817120788007002815DB2878002807D0EB
:102D2000012808D0022806D0032804D084489FE751
:102D30006846C77102E001206946C8710622691C15
:102D400002A817F088F97D48C078002803D0012830
:102D500004D003208CE76846877302E001206946AF
:102D6000887331886846018271884182B188818286
:102D7000F188C1820783478309A908F0F8FA00287F
:102D800090D1A08900F04AF804008BD11320FEF7FF
:102D900071FC20466CE730B50546674895B0006881
:102DA0000C46814202D2102015B030BD2846FEF7F5
:102DB0009EFC002807D00178222902D3807F80065C
:102DC00003D40820F0E75F48EEE71321684601705E
:102DD000458009A908F0CBFA0028E5D108AA0A2104
:102DE00051567F2901D02170DEE70520DCE730B5A0
:102DF000524D040009D0012C05D0022C08D0032C20
:102E000006D017F0B2FA2C7030BD17F0AEFAFAE720
:102E100028780128F7D017F0A8FAF4E710B50028B1
:102E200009D083000022114607200EF038FC072845
:102E300001D0032010BD002010BD70B50C00064667
:102E40000ED0FEF754FC050001D117F08EFAA680D3
:102E50002889E0802889208168896081A889A081EB
:102E600070BD10B50446006800280BD03049884278
:102E700006D33049884205D32F490968884201D2D8
:102E8000102010BD01F0D8F9A0882C4C6082607C25
:102E900001280DD1002109200EF06BFC002800D084
:102EA0000120617A8909012904D00321FEF73FFE40
:102EB000002010BD0221F9E7F7B500260C460546B3
:102EC0000B271AE02968B00009580978002903D0B7
:102ED000012901D00720FEBDA170296806220958EA
:102EE000E01C491C17F0B7F827702046029908F03B
:102EF0003EFA0028EFD1761CF6B22879B042E1D82C
:102F0000002639270FE0A868B10041581022A01C04
:102F100017F0A1F827702046029908F028FA002837
:102F2000D9D1761CF6B2287BB042ECD80020FEBD89
:102F300000B00100000000201C000020A8010020BB
:102F4000023200000230000001202249C003086064
:102F500021490020087007202049C005886070477B
:102F600030B51D4D04462878A04205D0002C03D072
:102F7000002801D017F0F9F92878A0420CD00021E0
:102F8000174A16482C70002C19D0164B012C04D06F
:102F9000022C0BD017F0E9F930BD1160022111604D
:102FA0005361032109068160416030BD1160032136
:102FB000116053610121C9058160416030BD11601C
:102FC00011600721C905816030BD00B517F0CDF94A
:102FD00000BD000080E100E01600002000F5014087
:102FE00000F50040D002002070B50C46054606F002
:102FF000DDFC2146284607F040FD70BD7047704754
:1030000010FFFFFFDBE5B15100B001007800FFFFCA
:1030100010B50621D84817F07BF810BDFFB591B068
:10302000D6481499814206D3D548814206D3D54863
:103030000068814202D2102015B0F0BD0120FEF7D9
:10304000ECFB0028F8D10124684603218471C902F1
:103050008180002201A9204603F09CFA0028EBD1D0
:103060006846152184714902818000261C2102A82E
:10307000009617F04FF801200146684610310170A4
:1030800000200146684641708178F9273940891C43
:1030900021438170017A02252943017212998186A8
:1030A000C6861F2101870C9011980F9001A80B90E4
:1030B00009AA0BA902A803F041F80028BCD1684670
:1030C000AD4E808C308068468471AF4981808078B5
:1030D00009AA3840801C41084900684681708586ED
:1030E000058713A80F900BA902A803F027F8002862
:1030F000A2D16846808C7080311D149800F0F9F8D8
:103100009AE73EB504460820694608809B488442F9
:1031100006D39B48844205D39A480068844201D272
:1031200010203EBD21460120FEF777FB0028F8D194
:103130002088694688806088C880A0880881E088E7
:1031400048818D4801AB80886A46002103F078FCF5
:10315000694609880829E4D003203EBD1FB504460E
:103160000020029008206946088184480391844227
:1031700006D38348844206D382480068844202D240
:10318000102004B010BD7C4802AA81887F4803F05B
:10319000EDFD0028F5D169460989082901D00320F1
:1031A000EFE7694609882180694649886180694658
:1031B0008988A1806946C988E180E2E701B582B0CB
:1031C0000220694608806C4802AB40886A460021AC
:1031D00003F036FC69460988022900D003200EBDA1
:1031E0001CB50021009102216A46118065490190B9
:1031F0000968884201D210201CBD5F48418863489D
:1032000003F0B4FD694609880229F5D003201CBDEE
:10321000F0B50E46594985B0174605468E4206D38D
:103220005848574A0068964204D3864202D210207A
:1032300005B0F0BD1F2F01D90C20F9E74E4C8D428F
:1032400026D3954201D3854222D3208803A903F0D7
:10325000A8FB0028ECD1287869464873208803A988
:1032600003F080FB0028E3D1694600900878022132
:10327000084369460870497B090703D008210843C1
:10328000694608702088694603F008FB0028CFD102
:1032900069468F802088334601AA002103F0D0FBC5
:1032A00069468988B942C3D00320C1E71CB50C46E2
:1032B000002100910191228869460A8031490190DC
:1032C0000968002801D0884201D38C4201D2102025
:1032D0001CBD002801D0002A09D027486A46018871
:1032E0002A4803F043FD6946098821801CBD0C2053
:1032F0001CBD30B5044693B000200D460790142144
:103300000BA816F007FF1C21684616F003FF6A465B
:103310001120107700205077107802210843107098
:1033200007A80C90012008AA907217486A46C01C92
:1033300010850AA80B902088108460885084A0888B
:103340009084E088D084907FF9210840801C400858
:103350004000907708209086108708A80F9010AA48
:103360000BA9684602F0EAFE002803D110A80088E5
:103370002880002013B030BD1000002000B00100F4
:10338000000000201C000020012A0000FFFF0000B8
:10339000F849884206D3F849884205D3F7490968B5
:1033A000884201D2102070470178C906490F0429CC
:1033B00007D84178072904D38278102A01D88A4295
:1033C00001D207207047C178490702D4007940072D
:1033D00001D5062070470020704710B5C37F1478D0
:1033E0005B08A4075B00E40F2343C3770878EF234F
:1033F000184013789B06DB0F1B0118430870F1235C
:1034000018401378DB065B0F5B0018430870507898
:10341000087310BD30B500240C70C378DB07DB0FD8
:103420000B70C578AD07ED0F6D002B430B70C578A1
:103430006D07ED0FAD002B430B7014700179C907B8
:10344000C90F117003799B07DB0F5B0019431170E3
:1034500000794007C00F80000143117030BD70B586
:1034600014460D46064604F068F9002809D0A2214A
:103470000170142221461830FDF788FE04F03BF954
:1034800070BD132229463046FEF71AFB70BD70B599
:1034900014460E46054604F050F9002809D02221B2
:1034A00001704580217801766178417604F023F936
:1034B00070BD132231462846FEF702FB70BD10B5E1
:1034C000AF4C207C00280BD12046AE4A2146103854
:1034D0000CF03EF8002801D016F047FF01202074C0
:1034E00010BDFFB581B00A9E05461C461746142143
:1034F000304616F00FFE0B9800210160F8070ED041
:103500009E492068096888423BD3123030602068A9
:10351000143070602068B0600B9821680160B807B3
:1035200028D56068002803D094490968884228D3C8
:103530000299002928D0FFF70AF801462846FF30F3
:1035400007225D3016F087FDFFF7B9FF8C48009029
:10355000F0606268002A0DD0FF2029465D30FF31FF
:10356000405D5E311032FEF79AFA102260680099D1
:1035700016F071FD780710D58049A0680968884267
:103580000AD2102005B0F0BD0028FAD0F060FF3557
:1035900001356068A865EDE730610020F2E730B5DD
:1035A000054611200C460870002161702121495DFB
:1035B000002905D003290BD004290DD016F0D5FE23
:1035C00020780009012802D9E87FC008607030BD6A
:1035D0000007000F203002E00007000F303020709D
:1035E000EEE710B5002803D06424245C002C08D03A
:1035F0006348047D0020002C0BD008601060186028
:1036000010BD044664340C6001469031BC3011603A
:10361000F5E75B4C14340C60F0E770B594B01546D8
:103620000C462C226946189E0A704880002B17D041
:103630000822194601A816F00EFD68468581102261
:1036400031460E3016F007FD09A9684607F08FFED7
:10365000002803D1A17F10221143A17714B070BDBF
:10366000002001900290E8E7F0B50646008A97B086
:1036700080B20D460290FEF73AF804464048317891
:1036800048380746883709900B0016F089FF0EFC72
:10369000FB390840647F9BB2FDF9F8F7F6FCA07F88
:1036A0008007800F012806D0002102980AF094F9C3
:1036B000050004D101E00121F7E716F056FE387845
:1036C000C00904D02E482038406EA8610FE02B209E
:1036D000694608730CA903A807F049FE002801D029
:1036E00016F043FE28490D9816F01EFDA96170687A
:1036F000A862B068E8622078252801D016F035FE6F
:10370000324621460298FFF7AAFE17B0F0BDA07F0F
:103710008007800F012806D0002102980AF05CF98A
:10372000060004D101E00121F7E716F01EFE207823
:10373000252804D03078012108433070E5E70220C5
:103740002870B068A860B068002802D000202871F6
:10375000DBE70120FBE72B20694608700849684633
:103760004C3907F004FE002801D016F0FEFD0320BE
:1037700024E0000000B00100000000201C00002038
:103780007C020020FFFF000040420F002A20694613
:10379000087000A810220230716816F05CFC04A8C2
:1037A00010220230B16816F056FCFD49684607F059
:1037B000DEFD002801D016F0D8FD042028700998FD
:1037C0006860A2E7B068002801D116F0CEFDE07F66
:1037D000400701D516F0C9FDB06800903379062284
:1037E0000421029804F09FFE00288ED016F0BDFD43
:1037F0008BE7002C01D116F0B8FD204622301022B4
:103800000546716816F027FC28212046FDF7A5FF24
:10381000A07F8007800F02280CD100231A46214682
:1038200000950298FFF7F9FE11280BD029212046B8
:10383000FDF793FFE07F317A4007400FC90008434E
:10384000E07762E7A07F000701D516F08EFDA07F2C
:1038500008210843A077002060862046343016F007
:1038600057FCE07FFD220146C9071040890F08433D
:10387000E077307A2034207047E705E17AE070E0A5
:1038800055E001E034E003E1A07F8007800F0128CC
:1038900006D0002102980AF09FF8040004D101E04C
:1038A0000121F7E716F061FD2B2069460873BC493A
:1038B00003A807F05CFD002801D016F056FDB848BB
:1038C0008188204621300176090A4176122129702B
:1038D0002146FF315D316960017E2974407E687444
:1038E000AF482C30A860103030346C61E8600CE7D1
:1038F000002C01D116F039FD20782128A1D930798A
:10390000012802D0022808D103E0E07F0421084307
:10391000E077387801210843387032462146029812
:10392000FFF79DFD23212046FDF717FFEDE601225D
:103930000421029804F043FF00289DD01320287032
:1039400017210020297100900246019003AB0298D4
:1039500004F00CFC002801D016F007FD0398A860C5
:10396000D3E60421029804F075FF002884D11420C6
:103970002870CAE6A07F8007800F012806D00021AA
:1039800002980AF029F8050004D101E00121F7E7C7
:1039900016F0EBFC2E462036307E410641D5A17F45
:1039A0008907890FC00713D0EB1DF9335A6D002A20
:1039B0000ED0107CF77DC007C00F7F003843107415
:1039C0005A6DE37F40084000DB07DB0F184310749B
:1039D000307E000713D5EB1DF9331A6D002A0ED087
:1039E000107CF77DC007C00F7F00384310741A6D3C
:1039F000E37F40084000DB07DB0F18431074307E84
:103A0000820701D5022903D0C0060AD5012908D1B1
:103A1000FF20593042592946307C31311032FEF7AF
:103A20003EF8052368460370357E45705C482221C8
:103A30007038029A01704178C908C900C91C4170E8
:103A400042800376457604F001F82078252806D0D8
:103A5000212808D016F089FC2078222803D92221B9
:103A60002046FDF77AFEA07F8007800F012809D04D
:103A70000021029809F0BBFF002800D145E616F0AE
:103A800074FC42E60121F4E77168002008703CE60E
:103A900016F06BFC39E6424810B58C3001780024F2
:103AA0004906490E0170603844660BF0DFFC3C4962
:103AB0003C310846103803F044FF39484C30047458
:103AC00010BD70B50D46FDF712FE040001D116F0D1
:103AD0004CFCFF216531284616F01CFBA07F8007B7
:103AE000800F012809D002212846E8300BF0BFFCE6
:103AF000002801D016F039FC70BD0121F4E70A4618
:103B0000014610B51046E8300BF0CAFC10BDF0B508
:103B100005464068082601789BB008290DD00B297E
:103B200003D00C293AD10121817168688788384611
:103B3000FDF7DDFD04003BD138E047883846FDF74E
:103B4000D6FD040001D116F010FC2078212825D0E4
:103B5000282827D1686802210C3000F077FF002860
:103B600020D068680821001D00F070FF002819D0DF
:103B70002D2168460170478021461022223101A87C
:103B800016F069FA0FA9684607F0F1FB002801D08A
:103B900016F0EBFB29212046FDF7DFFD1BB0F0BD41
:103BA00030020020687830436870F7E716F0DDFBDC
:103BB000A07F8107890F022902D1EF210840A07759
:103BC000207821280DD068688179002902D080787A
:103BD000002812D0A07F8007800F022858D016F04E
:103BE000C4FBA07F8007800F0228D7D1FDF7D8FF44
:103BF0000028D3D016F0B9FBD0E76878304368705E
:103C0000E07FC00701D0042100E0032121200155FD
:103C10002078292817D02428E3D1394606200DF032
:103C2000CEFD22212046FDF798FDA07F8007800F62
:103C300001282BD00021384609F0D9FE0028D0D029
:103C400016F093FBCDE7A07F8007800F012806D0F8
:103C50000021384609F0C0FE050004D101E0012131
:103C6000F7E716F082FB25212046FDF776FD1120AF
:103C700008A90871284609A9E8300BF004FC0228BD
:103C8000AFD00028ADD016F070FBAAE70121D2E733
:103C9000687830436870A4E7F7B58CB016460746DD
:103CA000FDF725FD040051D0207822284ED323288B
:103CB0004CD0E07F400749D4A07F8007800F0128C7
:103CC00006D00021384609F087FE050002D00BE03F
:103CD0000121F7E7A07F8007800F012804D101218F
:103CE000384609F071FE054601AB02AA03A9284631
:103CF000FFF777FC0398002801D116F036FB002D62
:103D000008D00398E83545612078222806D0242879
:103D100004D007E003990020486103E025212046F4
:103D2000FDF71BFD03980D210170476206710D9987
:103D300081600299C1600199016104A90BF0C6FB81
:103D4000022803D0002801D016F00FFB0FB026E7A1
:103D500030B589B00546FDF7CAFC017822292DD976
:103D6000807F8007800F012806D00021284609F0B7
:103D700033FE040004D101E00121F7E716F0F5FA63
:103D80001321684601731721017400200090024638
:103D9000019002AB284604F0E9F9002801D016F0A2
:103DA000E4FA02980590204603A9E8300BF06BFB7B
:103DB000022803D0002801D016F0D7FA09B030BD90
:103DC00010B586B00446FDF792FC017822291AD975
:103DD000807F8007800F012806D00021204609F04F
:103DE000FBFD040004D101E00121F7E716F0BDFA64
:103DF0001420694608702046E8300BF044FB002888
:103E000001D016F0B2FA06B010BDF7B5054600783D
:103E10000027000982B00C463E4602287AD00728C7
:103E200002D00A280AD143E068680178082906D040
:103E30000B292CD00C292AD016F097FA49E1142727
:103E40001A26002C67D04088A080FDF750FC009017
:103E5000002801D116F089FA00980099C07DA21DB2
:103E60001831FDF71CFE686808228089E0816968C6
:103E700020461030091D16F0EEF8207E012108437F
:103E8000F9210840207600984021807F3EE01827E5
:103E90000826002CD6D08088A080FDF728FC0500DD
:103EA00001D116F062FAA11D2846FFF778FB10E158
:103EB000002C01D0288DA080287E01287ED00228E9
:103EC00004D003282BD016F050FA02E11C27072655
:103ED000002CB7D0A088FDF70AFC0090002801D183
:103EE00016F043FA287F8007800F0128A07913D0AD
:103EF00040084000A071FD210840297F4907C90FF3
:103F000049000843A07100988021807F08430099F0
:103F10008877DEE0D0E076E001210843EAE7132766
:103F20000B26002C6FD0A088FDF7E1FB0090807F6E
:103F30008007800F012806D00021A08809F04CFDE1
:103F4000050004D101E00121F7E716F00EFA009810
:103F5000807F8007800F012850D0E96A8878800729
:103F6000800F0128A0794BD040084000A0718A78CA
:103F7000FD255207D20F284052001043A071E322C2
:103F800010400A785207D20E1043A071DF22104071
:103F90004A78D207920E1043A0710020E071C878D1
:103FA00020724B79607ADA0740084000D20F104344
:103FB0009A072840D20F0979520000E024E010430C
:103FC0005B07FB22DB0F10409B0018436072A07A56
:103FD000CB0740084000DB0F18438B07DB0F28405E
:103FE0005B0049071843C90F104089000843A072BD
:103FF0000098007823286CD92621B4E0A96AADE79F
:1040000001221043B2E752E0297FFE4802290ED078
:1040100017270C26002C4AD001290FD003291CD0C9
:1040200004291DD005291BD016F09FF923E019277C
:104030000726002C4DD00121A17105E00121A171BD
:10404000E17989088900E1710178CA094906D2013C
:10405000890E49000A4302700DE00220A07106E0BB
:10406000687F0007000F8030A07105291AD0E07921
:1040700080088000E071A088FDF739FB05460078D4
:10408000212826D0232801D016F06FF9A87F8007B9
:10409000800F01280ED00021A08809F0A8FC222161
:1040A000284661E0E07980088000401CE2E704983F
:1040B000068014E00121EFE7002C01D06888A08081
:1040C000287E03282BD004280CD005284FD016F0CA
:1040D0004CF90498002C068001D0278066800020CF
:1040E00005B05CE515270C26002CE0D0A088FDF774
:1040F000FEFA807F8007800F012806D00021A0886B
:1041000009F06AFC050004D101E00121F7E716F08F
:104110002CF90622A11DA86907F06CF9D9E716272A
:104120000726002CC3D0A088FDF7E1FA0090807F1D
:104130008007800F012806D00021A08809F04CFCE0
:10414000050004D101E00121F7E716F00EF9287807
:10415000C00601D5022000E00120A071009800787F
:104160002328B6D927210098FDF7F7FAB1E71727DA
:104170000C26002C9BD0A088FDF7B9FA00906D7E2C
:10418000002801D116F0F1F80621A01D15F0C0FF9E
:104190000020A071207A032108432072FB210840EF
:1041A0000099C97FC907490F08432072680690D556
:1041B000E07904210843E071A07A29074208E80762
:1041C0005200C00F0243E07AC90F40084000084384
:1041D000FD210A40AB07DB0F5B000840E9061A43EC
:1041E000C90F4900A2720843E07272E710B5044695
:1041F000807992B08009012801D016F0B6F8FFF757
:104200005EF90120694608707F4809907D480BA936
:1042100040380190201D0290601C0C9068460BF005
:1042200055F9002801D016F0A0F80322601C0C9963
:1042300015F011FF12B010BD10B5724C403C0028B3
:1042400005D001461022204615F005FF01202074FC
:1042500010BD10B50446FFF732F96A491022403903
:10426000204615F0F8FE10BD70B50025654C0028FD
:104270001BD06649884206D36549884205D3654903
:104280000968884201D210250DE0062107F09CF84C
:10429000411C07D05B49603948662078802108437B
:1042A000207000E00725284670BD20784006400EAB
:1042B000F6E7F3B500278BB00C46002909D0534828
:1042C00084421BD35248844203D35248006884423C
:1042D00014D30B98FDF70BFA050003D02878222899
:1042E00015D102E04C480DB059E4002C08D1A87F4C
:1042F000C10903D08007800F022801D01020F2E707
:10430000A87FC10601D4010703D5002C01D00820E5
:10431000E9E73C490978C90701D01120E3E7E97FC3
:10432000490701D50D20DEE78007800F022806D15E
:10433000002C04D02046FFF72BF80700D3D1A87F2C
:104340008007800F012806D000210B9809F044FB5C
:10435000060002D00CE00121F7E7A87F8007800F5C
:1043600001280BD000210B9809F02EFB060007D086
:10437000A87F8007800F022804D00AE00121F2E71D
:104380000420B0E7002C04D0224631462846FFF72F
:1043900024F809AB1A4669463046FFF722F900981F
:1043A000002801D115F0E1FF00980E2101700B9952
:1043B00041623146E8318160A97FFB228907890F7C
:1043C000012937D0002C4BD002210171311DC16071
:1043D00031780907490F01743178C906C90F417452
:1043E000817C23788908DB078900DB0F19438174FE
:1043F0001140EA7FD207520F11438174A178C17432
:1044000002AA0BE0BC020020FFFF000000B0010088
:10441000000000201C0000200230000001A92046FE
:10442000FEF7F8FF69460098097A0175694609792F
:10443000417519E001210171017B23788908DB07AF
:104440008900DB0F19430173114022789207D20FC4
:1044500092001143017324212846FDF77EF90BE0F9
:10446000032101710521017325212846FDF775F906
:10447000A87F4006400EA87703A900980BF026F805
:10448000022803D0002801D015F06FFF38462AE734
:10449000FFB5FF4A97B007CA02AB07C300201390CD
:1044A000009001901798FDF722F9050005D02878B3
:1044B000262804D008201BB0F0BDF648FBE7A87FF3
:1044C0008707BF0F012F02D0022F09D00BE01898E9
:1044D000002808D11998FEF75BFF0028EBD102E015
:1044E0001998002814D1189885281BD008DC0028BA
:1044F00010D0812810D0822810D0832808D10FE056
:10450000862811D0882811D0892811D08A2811D066
:104510000720D0E700260EE001260CE002260AE084
:10452000032608E0052606E0062604E0082602E049
:10453000092600E00A26A87F8007800F012806D000
:104540000021179809F048FA040004D101E0012184
:10455000F7E715F00AFF012F0ED1189800280BD1AC
:1045600021462846199AFEF738FF1998807800905E
:104570001998007838400190002020710120694688
:104580000876201D0790002E01D02671FAE0012F39
:104590000CD0A66AE06A0222012112900020A060DD
:1045A0002846173002291AD0012119E0E66AA06ACC
:1045B0001290032030702078FB23C006C00F70706B
:1045C000B07801221840009BF3708008019B8000A6
:1045D00018430221B070002070713071DEE70021B5
:1045E000890009190861681C022A01D0012100E034
:1045F0000021890009190861B0788007800F01281F
:104600005CD1129880788007800F012856D11298CB
:10461000012F007901901298407900901CD03179D7
:1046200008A801747179017508A8027C01980099A5
:10463000024008A8007D0840149010433ED09649DF
:104640001A98884206D39549884215D39449096837
:10465000884211D210202EE70CAA0DA91998FEF756
:10466000D9FE08A8007C01990840307108A8007D97
:10467000009908407071D7E72146FF31204651313B
:104680003C3001910090022F34D000211A9B20462B
:104690000C33FEF726FF0028DDD12146FF312046EE
:1046A0005531503001910090012F25D00021204636
:1046B0001A9B149AFEF715FF0028CCD11298807827
:1046C000400702D4E87FC0072ED002A8012F15D0E2
:1046D000129909784900405A21780907490F490081
:1046E000C8408007800F13902CD0012815D00228D5
:1046F00010D114E00121C9E70121D8E72178090789
:10470000490F4900405A129909784900C84080076A
:10471000800F1390032805D006E0022000E001205E
:1047200013900FE002201390012F0BD1B078FB21E2
:104730000840E97FC907490F0843B0702078000797
:10474000400F3070207810224008400020701299ED
:10475000D2434978C907C90E114308402070C006EA
:1047600021D4139802281ED001281ED00020A06159
:10477000E0612062606220461830A060E87F400857
:104780004000E877204606A9E8300AF07CFE0028C1
:1047900003D0022801D015F0E8FD25212846FCF7BA
:1047A000DCFF002087E6032008E020460D211B30B7
:1047B00015F0AEFC20461830A0600420694608754C
:1047C000E87F01210843E87705AA29461798FEF7F4
:1047D0005EFED7E7F0B587B015460F0004460CD053
:1047E0002D48854206D32D48854206D32C480068C3
:1047F000854202D2102007B0F0BD2046FCF777FFBB
:10480000060004D03078272803D00820F3E7214899
:10481000F1E7B07F8007800F012806D000212046F5
:1048200009F0DAF8040004D101E00121F7E715F0FE
:104830009CFD0020002F05D0022F08D0012F11D0A1
:104840000720D8E701216A461171A06018E02346CD
:1048500018336946A360087110222946184615F0DE
:10486000FAFB0DE021461831A16069460871A0618C
:10487000E061206260620621284606F0A5FDA06185
:104880002078C1071CD0400840002070022009E0B9
:10489000BCA501000230000000B0010000000020B3
:1048A0001C00002069460870204618300290D03065
:1048B0000AF0E9FD022803D0002801D015F055FDCB
:1048C00025213046FCF749FF002094E7F8B515464E
:1048D0000E460746FCF70BFF040004D02078222880
:1048E00003D00820F8BD6048F8BDA07F8007800F86
:1048F000022802D05C48C01CF8BD5C4886420DD33B
:104900005B495C4A8E4202D313689E4206D38542BD
:1049100004D38D4204D31068854201D21020F8BD23
:1049200000953288B31C21463846FEF776FE1128E2
:1049300016D00028F3D1E17F2A7C4908D20749002C
:10494000D20F1143E1772A7C49079206490FD20E14
:10495000D2001143E177A17F4906490EA177F8BD46
:10496000A17F0907FBD420460822B11C343015F082
:1049700072FB30886086204610222946223015F0CE
:104980006AFBE07FFD210840297CC907890F0843A5
:10499000E077287C410820200155A07F08210843AA
:1049A000A0770020D7E770B594B00D460646002BDF
:1049B00002D0072014B070BDFCF799FE040007D0A8
:1049C0002078222802D3A07F400603D40820F1E7F4
:1049D0002548EFE7002D19D02D216846017046804B
:1049E0001022294601A815F036FBE07F297C4008FB
:1049F000C9074000C90F0843E077297C40078906B2
:104A0000400FC90EC9000843E07703E02E21684635
:104A10000170468009A9684606F0A9FCA17FBF2263
:104A20001140A177C6E710B50C46FCF760FE0028E0
:104A300005D0104909688C4203D2102010BD0A48E5
:104A400010BD2146FEF7ABFD002010BD05E0027849
:104A5000401C002A01D0002070470A46491E89B236
:104A6000002AF4D1012070470230000000B001009C
:104A7000000000201C00002070B50D46007804994D
:104A80001446042804D005282ED015F06EFC70BD05
:104A9000A88B062250430E30188033200880002C4B
:104AA000F5D0A88BA081002611E0A87F012812D0A4
:104AB00012207043411906227243088C1219D081CA
:104AC0001020223110320AF0F2FD761CB6B2A08915
:104AD000B042EAD870BDB000411906227243088C7A
:104AE0001219D0810220ECE7A88B1222504310301B
:104AF000188034200880A87F012809D0022807D018
:104B000015F033FC002CE5D0A88BA081002612E024
:104B1000A073F7E7A87F012811D03046122148433F
:104B200041190A8C0019028210221230223115F02C
:104B300092FA761CB6B2A089B042EBD870BDB00034
:104B400041191222088C724312191082022022315C
:104B500012320AF0ACFDECE7F8B500780C461646C8
:104B600020340E36069F022806D0032833D00628AC
:104B70007ED015F0FAFBF8BDCD8B0A2068430E30CD
:104B8000188031203880002AF5D0087F9581801F59
:104B9000C7B21AE020886168308048780A7800023D
:104BA0001043F080C8788A78000210433081B21C2C
:104BB0003846091D0AF07BFD002F01D0002802D0E5
:104BC00000203071708008340A3628466D1EADB260
:104BD0000028DFD1F8BDCD8B0A2068430E30188045
:104BE00032203880002AF5D0087F9581401FC7B257
:104BF00043E0616822880878F2803279C30752085E
:104C00005200DB0F1A43FD231A408307DB0F5B00C2
:104C10001A43FB231A404307DB0F9B001A43F72379
:104C20001A400307DB0FDB001A43EF231A40C306C9
:104C3000DB0F1B011A43DF231A408306DB0F5B01E6
:104C40001A43BF231A404306DB0F9B011A433271FC
:104C5000C00970718A784B7810021843308132464F
:104C60003846C91C0AF023FD002804D0002000E0CB
:104C700009E0B070308008340A3628466D1EADB2A7
:104C80000028B6D1F8BD087FCD8B801E86B2304695
:104C9000083068431030188035203880002AF1D061
:104CA000174695811037E800D681C01900900DE0B5
:104CB000208838800098786032466168009815F046
:104CC000CAF90098083480190837009028466D1EEC
:104CD000ADB20028ECD1F8BDFFB5099E1D460C46CB
:104CE000002A05D0607EFF300130D080E08B10813B
:104CF00000980078030015F053FC0C9C0716232D38
:104D0000374150667070709C087F1746082803D0A2
:104D1000032801D015F029FB0E20288030200BE05D
:104D20000020B881FFBD087F1746042801D015F088
:104D30001CFB0E20288031203080002FF0D1FFBDD9
:104D4000087F1746042801D015F00FFB0E2028809D
:104D50003220F1E7087F1746022801D015F005FB45
:104D60000E2028803320E7E7087F1746022801D06D
:104D700015F0FBFA102028803420DDE7087F174665
:104D8000042801D015F0F1FA102028803520308059
:104D9000002FD4D00020B88113E0207F17460528CB
:104DA00003D0062801D015F0E0FA12202880362022
:104DB0003080002FC3D0E08BB8810020388200986B
:104DC0004088F881FFBD087F1746072801D015F0FD
:104DD000CCFA0E2028803720AEE714202880382017
:104DE00017463080002AEDD0E08BB8810020788211
:104DF00000980078092806D00A280BD00B2810D07C
:104E000015F0B3FAFFBD087F0C2801D015F0ADFAFC
:104E100001200CE0087F0D2801D015F0A6FA04202F
:104E200005E0087F0E2801D015F09FFA0520B87321
:104E3000FFBD15F09AFAFFBD70B50C460546FCF7AC
:104E400056FC002804D00078222803D2082070BD28
:104E5000FE4870BD0521284608F0BEFD20600028F0
:104E600001D0002070BD032070BDFFB585B00D4698
:104E7000074617206946088108980326144600282B
:104E800005D108A93846FFF7D7FF00283FD1002DEC
:104E90000BD000220321384603F091FC00283FD0BC
:104EA0000898007800283BD106E02078092824D013
:104EB0000F282ED015F059FA0020009002460190DC
:104EC0006846018903AB384603F050F9002801D049
:104ED00015F04BFA0898A760801D606002A9204673
:104EE000039A04F0FAF9002827D0030015F058FBC4
:104EF000071A182323211C1E2300072600223146EF
:104F0000384603F05CFC0028D6D1D048801C09B09C
:104F1000F0BD00220321384603F051FC0028CBD11C
:104F20001120F4E70020F2E70820F0E7C748401C12
:104F3000EDE70720EBE70320E9E7039800906846D8
:104F4000038904223146384603F0EDFA0028DED109
:104F5000002DDCD008990D70D9E730B587B01D461B
:104F60000C46002A11D0042369460B7013888B81EC
:104F70005288CA81A2788A7422880A8200236A46EB
:104F80002946FFF772FF07B030BD1020FBE7F3B5ED
:104F900081B001980C4600780826030015F000FB4C
:104FA00012413B3B17123E0A0A0A0A0A0A0A0A0A77
:104FB0000A0A0A41002C01D115F0D7F96078304374
:104FC000607030E0002CF9D115F0CFF9F6E70198C8
:104FD0000521808887B2384608F0FEFC0546002C83
:104FE00001D015F0C2F9002D01D115F0BEF93946F6
:104FF000A81D04F069F902F0A0FB040006D0607857
:1050000030436070678002F076FB0EE01321384673
:10501000FDF774FD14E015F0A8F904E015F0A5F90A
:1050200001E015F0A2F9002C0AD06078000707D53E
:10503000932020702046582218300199FCF7A6F8DA
:105040000020FEBD10B500210170801D04F039F96B
:1050500010BD0A4610B50146901D04F03DF910BD83
:1050600070B50546052108F0B7FC040001D115F024
:105070007CF92946A01D04F027F970BDF7B586B06C
:105080000C46054600206946088188806F88052106
:10509000384608F0A1FC060001D115F066F9002C95
:1050A00003D0A7800020E0802081297E2046123096
:1050B000C91E142700900B0015F072FA0FFCFDFAC0
:1050C0006009AD696F812CB6CCE89595FA0030780F
:1050D000012801D015F049F9A88B6A46C1000E31AC
:1050E000918030211181002C13D0A08100200DE08F
:1050F000C100327909190A747288CA818200531971
:10510000DA8B4A821A8C401C8A8280B2A189814241
:10511000EED8ECE03078012801D015F026F9E88BC4
:105120006A46C1000E31918030211181297F091F0B
:10513000C9B20491002CECD0A08100271AE0F8003D
:105140000219401900920390416A0E3204980AF045
:10515000AEFA002804D00099002008740099C88194
:1051600003987F1C018C0098BFB241820398418C48
:1051700000988182A089B842E1D8B8E002A80090E6
:1051800001AB224629463046FFF776FCAFE0307887
:10519000072807D015F0E9F804E03078072801D097
:1051A00015F0E3F8E88B69461230888036200881D4
:1051B000002C38D0A98BA1817188E18123E030785F
:1051C000082801D015F0D1F8A88B6A4601460E30A8
:1051D000908037201081002C25D0A1812046AA8BF9
:1051E0000E30296A4FE0E88B6946123080B23922CE
:1051F00088800A81002C75D0A98BA181287E102877
:1052000007D00221A173E98B2182EA8B296A0098D9
:1052100039E00121F6E702A8009001AB22462946B9
:105220003046FFF799FC62E03078092801D015F08C
:105230009CF8694638208F800881002C57D0A98BB4
:10524000A181002060822082012001E00230000064
:10525000A0734CE030780A2801D015F086F8288C2D
:1052600069461430888038200881002C3FD0042102
:10527000A173A98BA181E98B2182298C61822046AF
:105280002A8C1430696A14F0E6FE30E030780B287E
:1052900001D015F06AF8694638208F800881002C0B
:1052A00025D00521A1730020A081208260821EE00C
:1052B0001BE000E008E002A8009001AB224629466E
:1052C0003046FFF709FD12E00D2069463A2288803A
:1052D0000A81002C06D00120E0800020208120736C
:1052E00005E0FFE70899088016E015F03EF86846EB
:1052F000089980880880002C0ED06846008920809C
:10530000684680886080287E032805D0102803D056
:10531000112801D0002030700020F8E5F7B556883C
:105320000F4682B015460521304608F055FB0400B3
:1053300001D115F01AF8A41D33462A4639460094C7
:10534000029804F050F905B0F0BDF7B58CB00D46E9
:10535000144607A90C98FFF76FFD002812D1884E5C
:105360000127002C10D00321684601701021818292
:1053700008A802460690204605A90AF0BEF90028B2
:105380000CD007200FB0F0BD082168460170858160
:10539000C68105218774C90201820BE00798A178B4
:1053A000017121884180684605218774C902018204
:1053B0008581C68102460121079B0C98FFF755FDA8
:1053C000E0E708B501236A4693706E4B13800A46E6
:1053D00002236946FFF7C1FD08BD08B501236A46EF
:1053E0009370684B5B1C13800A4603236946FFF7E2
:1053F000B4FD08BD00B587B000290CD002236A4671
:1054000013700B8893814988D18100230421FFF711
:105410002CFD07B000BD1020FBE710B5002903D01C
:105420000623FFF79AFD10BD072010BD70B588B0A8
:105430000D461446064607A9FFF7FEFC00280DD1CD
:10544000002C0DD00621684601708581C481079B20
:1054500002465C8007213046FFF707FD08B070BDAB
:105460000521684601708581F1E710B588B00029F3
:105470000BD007246B461C709A81049100236A4666
:105480000821FFF7F2FC08B010BD1020FBE770B553
:105490000024172288B0002914D00D782B0015F0B5
:1054A0007FF80623050519041B231522D21E93B28B
:1054B000CA88002A02D08E68002E03D09A4203D9EF
:1054C0000C20CBE71020C9E7042D05D08A88002ADC
:1054D0000AD101E00620C1E7012D11D0022D05D02F
:1054E000042D18D0052D23D00720B7E709236A46DD
:1054F00013704B889381CB88D381896804911DE018
:105500000C236A4613704B889381CB88D3818968BA
:105510000924049112E00D236A4613704B8893818D
:105520008B88D381CB88138289680A24059105E092
:105530000E236A461370497811730B240023214609
:10554000FFF793FC8AE700B587B00F236A46137014
:10555000918100231946FFF788FC5AE700B587B010
:1055600000290BD002236A4613700B889381498867
:10557000D18100230521FFF778FC4AE7102048E796
:10558000FFFF000002280000002803D081780129D5
:1055900039D101E0102070470188FE4A881A9142F3
:1055A00033D01BDCFC4A881A91422ED00BDC002938
:1055B0002BD00320C002081A27D0012825D00121B2
:1055C0000903401A07E001281FD002281DD0FF2838
:1055D0001BD0FF380138002815D116E0FF22013218
:1055E000811A904211D008DC01280ED002280CD07C
:1055F000FE280AD0FF2806D107E0012905D002299C
:1056000003D0032901D0002070470F20704700B558
:105610000B2826D009DC030014F0C2FF0B1D212546
:10562000251B25292325271F1B0011281BD008DC3B
:105630000C2816D00D281CD00F2814D0102808D103
:105640000FE0822809D084280FD085280FD0872822
:1056500011D0032000BD002000BD052000BDCF48B3
:1056600000BD072000BD0F2000BD042000BD0620A6
:1056700000BD0C2000BD0D20800200BD00B5030060
:1056800014F08EFF070507050D0D090B0D00002016
:1056900000BD112000BD072000BD082000BD032073
:1056A00000BD00780207120F04D0012A05D0022A9B
:1056B0000AD10EE0000907D108E00009012805D051
:1056C000022803D0032801D007207047087000206B
:1056D000704706207047002807D0012807D002280D
:1056E00007D0032807D007207047002004E01120CE
:1056F00002E0212000E0312008700020704738B51A
:105700000C4605004FD06946FFF7CBFF002822D199
:105710002088032189028843694609788907090D91
:10572000084320806946681CFFF7BBFF002812D1A0
:105730002188032000038143684600788007800C9D
:1057400001432180A8784007820F2020012A03D03E
:10575000022A03D0072038BD814300E001432180A5
:1057600088B20105890F08D0012189038843A978EF
:105770000907C90F89030843208080B28104890F7B
:105780000AD0A9784004C906C90F400CC9030843D0
:1057900020808004800F02D12088400403D5208817
:1057A000402108432080002038BD70B50446002009
:1057B000088015466068FFF7A2FF002815D12189EF
:1057C000A089814210D861688978C90708D0012171
:1057D0004902884208D8491C14F0A6FC298009E037
:1057E000FF21FF31884201D90C2070BDFF30FF300E
:1057F00003302880002070BD10B5137804785B0852
:10580000E4075B00E40F23431370FD242340047876
:10581000A407E40F640023431370FB24234004789F
:105820006407E40FA40023431370F7242340047893
:105830002407E40FE40023431370EF24234004788B
:10584000E406E40F240123431370DF24234004788B
:10585000A406E40F6401234313700078BF244006BC
:10586000C00F2340800103431370002906D008783D
:10587000C10701D1800701D5012000E00020C0014F
:105880005906490E0843107010BD30B50A8803232D
:105890009B0204889A4323059D0F02D1A3049C0F09
:1058A00001D09B0F00E001239B021A4303230A80CF
:1058B0001B039A4303889804840F02D11805830FB1
:1058C00001D0800F00E00120000302430A8030BDB8
:1058D000F3B593B00D000FD0139800280FD012210C
:1058E000284614F015FC03AAFF21012005F075FBE2
:1058F0000024264637467BE0102015B0F0BD072077
:10590000FBE76846807D01280BD16846818A052027
:10591000C002081A0AD001280AD002280CD0032895
:105920000CD0042C0ED0052C0FD10DE0012400E08A
:1059300002246846468A08E0032406E068460424F8
:10594000478A02E0052400E006246846418A13984D
:1059500081424DD12C74002E48D00DAA0EA90520ED
:1059600002920191009010230022FF21304605F0A1
:10597000D5FB00282AD16846808E2A46C0B20EA9DF
:1059800009F095FE002821D1AE81002F2ED00DA95F
:1059900008AE05E0022900000128000003300000E5
:1059A000052002910090132300220196FF21384622
:1059B00005F0B4FB002809D16846808EF11CC01E9A
:1059C000C0B22A1D09F073FE002801D0032094E71D
:1059D00008A88178427808021043E881062C05D196
:1059E0006846807DA8726846808A2881002084E706
:1059F00003A805F0FBFA002883D0FFF708FE7CE738
:105A0000002805D0FE4A012903D0022903D0032033
:105A10007047518800E09188814201D10020704791
:105A200007207047F0B58BB00E4605461C4617465A
:105A3000142103A814F06EFB012069460873087452
:105A4000119A4A748F82002C0AD0A178C90707D016
:105A500069468875E0884883A0880883A068079015
:105A600001F06BFE040022D0658017216846018496
:105A7000002000900246019009AB284602F076FB18
:105A8000002812D16846083670C008AA099B1099F0
:105A900004F0A5FD06466078000701D501F02BFE55
:105AA000002E0AD03046FFF7E9FD0BB0F0BD132100
:105AB0002846FDF723F80320F7E709980090684689
:105AC000038C04220121284602F02DFDEDE770B57C
:105AD00006468AB000200D4607900590069003A95F
:105AE0000490052402460291019010230094294657
:105AF000304605F013FB00280DD108A804A9009139
:105B0000029001946846838900222946304605F0B8
:105B100021F9002801D0FFF77AFD0AB070BD10B559
:105B200004F0B9FF10BDFEB50026054602960078C8
:105B30000C460827030014F033FD0CD0071036E2A2
:105B40006B6B8CA8CBAEBBD0002C01D014F00DFC3D
:105B5000288980B201F084FFC1E0A888042180B2C6
:105B6000009007F039FF0190002C01D014F0FDFBEC
:105B70000198002801D114F0F8FB01980099083031
:105B800004F04BF901F0D9FD040007D060783843E8
:105B900060700098608001F0AEFDA2E013210098D3
:105BA000FCF7ACFFABE0002C01D114F0DEFB608809
:105BB000042107F011FF0090002801D114F0D5FB5B
:105BC0000099002008802A7994461EE0C3005B19E2
:105BD0009B6800936B461B881A0708D5DA0606D522
:105BE0006046C20050194038C08F088006E05B0450
:105BF00009D50871C2005019C088488060783843C0
:105C0000607002266BE0401CC0B28445DED866E0BE
:105C1000E888694608800090002C01D114F0A5FBAB
:105C20000098C00B04D02878062805D0052830D06D
:105C300060783843607052E06088042107F0CCFE41
:105C4000060001D114F091FB00203071A88870800B
:105C50001FE0002C01D114F088FB6088042107F0BC
:105C6000BBFE0090002801D114F07FFB00980830A3
:105C700004F063FF0121484002D1E888C00B2ED018
:105C8000009861880226C180D2E7002C01D114F06F
:105C90006CFB0226CCE7002C01D114F066FB022637
:105CA00061880122204601F011FF01200290BFE728
:105CB000A889002C87B201D014F057FB68680090C7
:105CC0002889694688800122384601F015FF06E0E0
:105CD000002CADD114F049FBAAE714F046FB002CD0
:105CE0000DD0607800070AD50298002807D18420DB
:105CF00020702046582229461830FBF747FA3046D4
:105D0000FEBDF7B50C460546007E224688B00A3235
:105D10000392921C02920027811E16323E46019287
:105D20000B0014F03DFC08FD05FC34347FBEFBFC89
:105D30006888042107F050FE0190002801D114F07A
:105D400014FB01980088002802D052270726F2E0B1
:105D500051271E26002C7DD06888A0800120A071CC
:105D6000019803990079C0004019C08BFFF7B0FD7E
:105D7000002870D101980079C0004019C08B2081A3
:105D800001980079C0004019408CA083F0E0698C34
:105D90000091062820D1E88BC00B1DD00846223088
:105DA000512786B2002CD6D0A88B0299FFF790FD20
:105DB000002850D16888A0800220A071A88B208183
:105DC0000120A072288CE08300982084696A009AE0
:105DD000019814F040F9CBE008462030502786B2F5
:105DE000002CB8D0A88B0399FFF772FD002832D1A0
:105DF0006888A080A88BE080287E062810D001E06B
:105E0000C402002002202072288CA083E88BC00BE3
:105E100060720098E0832046696A2030009AD8E7D3
:105E20000120F0E76888042107F0D6FD0490688C13
:105E300000900498002801D114F097FA04980830D3
:105E400004F07BFE0121484002D1E88BC00B26D034
:105E5000009801E07DE023E02230512786B2002C3B
:105E600078D06888A080A88B0299FFF731FD0028C0
:105E700016D10220A071A88B20810420A072288C4A
:105E8000E08300982084696A009A019814F0E3F88E
:105E90000499002008710498A98B418068E00320D0
:105EA00003E66888FBF723FC00906888042107F06C
:105EB00093FD03900098002801D114F056FA03983E
:105EC000002801D114F051FA0398FF49C088884294
:105ED00002D05127222601E050272026002C39D05D
:105EE0006888A080502F07D00220A0712146287F0B
:105EF000083101F068FA3BE0287FA11D01F063FA48
:105F000000980021203040780090019103980B46C2
:105F1000428868880399FFF785FD02E004E025E0E8
:105F20001BE00028BCD123E0E849A88BC988814246
:105F300006D154270626002C0CD06888A08017E0D4
:105F400053270826002C05D06888A080A88BE08005
:105F50000EE0FFE70A98068010E055270726002C80
:105F6000F8D0A88BA0800020A07101E014F0FDF90A
:105F70000A98002C068001D027806680002094E5D6
:105F8000D24900200870704730B585B00C4601F04A
:105F90002FFA0546FF2801D114F0E7F900202080F0
:105FA00020716080401EE08020462946083003F0C2
:105FB00027FF6A462946012005F00FF8102412E059
:105FC0006846808800070ED56846C0882946FFF7D6
:105FD0007EFD68468188FF2321438180C088294651
:105FE000019A05F025F9684605F000F80028E7D089
:105FF00005B030BD0A46014610B51046083003F022
:1060000014FF10BD70B50546042107F0E5FC04003F
:1060100001D114F0AAF920462946083003F0FDFE0C
:1060200070BDF3B58BB00D460B98FBF760FB060017
:1060300005D03078222804D208200DB0F0BDA44845
:10604000FBE704210B9807F0C7FC0746002D02D0A0
:10605000A88800280ED0012168460173022100247F
:1060600001744474002D07D0A88869460883286805
:10607000059003E00920E0E70483059401F05DFB4F
:10608000050026D00B98688017216846018401948A
:10609000009409AB00220B9802F068F80028CCD1DC
:1060A000384608300B99029020360095019171789E
:1060B00008AA03A8099B04F092FA0446687800072E
:1060C00001D501F018FB002C09D02046FFF7D6FAC5
:1060D000B3E713210B98FCF711FD0320ADE70998F6
:1060E00000906846038C042201210B9802F01BFAF1
:1060F0000021C943F980A0E7FFB585B00E9E7788DF
:106100003846FBF7F4FA05460421384607F064FCEC
:106110000446002D01D114F028F9002C01D114F00F
:1061200024F90834089869460394C1C105A80DC82C
:106130002035697803F0A8FE09B0F0BDF0B504463B
:10614000002099B00D4601460D9010A88181164699
:10615000018181805D4A68469180018510A8018097
:1061600068460187818581841078012808D002283B
:1061700006D0032804D0042802D0082019B0F0BDAE
:10618000544A94426AD3554F534938688C4201D3DC
:10619000844263D34F4A954260D34F498D4201D325
:1061A00085425BD36168002912D04A4A914255D397
:1061B000494A914201D3814250D360892189884262
:1061C00003D801225202914201D90C20D6E70D904A
:1061D00016AA0EA92846FFF7E8FA0028CED168686B
:1061E00080784007800F02280AD16846008F80041B
:1061F000800F05D02869002802D0396888422DD345
:106200000AA92069FFF77BFA0028B7D12069002886
:106210000BD0607880076846008D03D58004800F1E
:1062200073D002E08004800F6FD16846008D810634
:1062300016D58004800F606805D0002810D039681A
:1062400088420BD301E000280AD02249884205D3B6
:106250002149884204D33968884201D210208DE751
:1062600009A96069FFF74BFA002887D16069002807
:1062700008D06846808C0105890F012945D180042A
:10628000800F42D00BA9A069FFF739FA00289DD1F1
:106290006846808C800638D46846808D810634D468
:1062A000A169002906D00105890F01292DD180049B
:1062B000800F2AD0E068002804D00078002824D07D
:1062C0001C2822D204AA0BE0FFFF0000C402002019
:1062D0000230000000B00100000000201C0000207F
:1062E000611C2046FFF788FA0121890210A801806D
:1062F000012768468773F849818104AA033217A9E8
:10630000286809F0FAF9002801D0072036E710A81C
:10631000007F15A9C01CC2B200200C920190FF3270
:10632000009003460291FF3203A80332109904F053
:10633000ACFD002826D110A9888A0F902A892969E6
:10634000E64801910092029010A90A8B6B89286897
:106350000E9904F09AFD01007ED1E0480025001F4F
:10636000818868464174090A8174052104A86A4637
:1063700023C210A82A46FF21808A0C9B04F0EAFC65
:10638000002802D0FFF743F9F8E66846007C0322B4
:10639000C1090020920290430122920280181490B9
:1063A000002928D0014610A801806846292187735A
:1063B00009028181058608A8007C002341086078D5
:1063C0004900C007C00F014308A80174FD20014027
:1063D0006078C34A8007C00F4000014308A80174D9
:1063E0000CA9022001910090029503A8109904F0D5
:1063F0004CFD010030D16068002828D020690028B9
:106400000DD10AA90EA8FFF740FA6078800706D4DC
:106410006946088D03210903884369460885AE490A
:1064200068468773FE318181AD492089891E13F04A
:106430007BFE62680D9811AB0192009002930A46B0
:10644000002303A80A9904F020FD010004D120785C
:10645000C10603D4800600E085E02AD5684605869B
:10646000606900280DD109A90EA8FFF70EFA684649
:10647000818C032080028143012080020918684634
:1064800081846946888CC82108436946888492487B
:106490008F73FF30888112AA0CA902200292019109
:1064A000009000238E4A03A8099904F0EEFC010035
:1064B00059D12078C00729D068460586A0690028F0
:1064C0000DD10BA90EA8FFF7E0F96846818D0320D6
:1064D0008002814301208002091868468185684650
:1064E000818D402001436846818587737D49818184
:1064F00013AA0CA902200292019100900023784A6D
:1065000003A80B9904F0C1FC01002CD1E06800281D
:106510002DD010A814990180724968468773491CD0
:106520008181E16808A80A78027449784174E068BA
:106530004122418868464186E0680023017908A825
:106540000175E068D200C18808A84175090A817503
:106550000CA8072101900091029503A8109904F05E
:1065600094FC010003D00F9800F046FF06E65B485C
:106570000321001F0170002E0AD08088308010A8EF
:106580008088708010A80089B08010A88089F08071
:106590000020F3E530B501248BB015460B460128E9
:1065A00002D002281CD104E0684605218473C90288
:1065B00003E0494968468473891E8181002B12D00B
:1065C000032100208902884301218902401869467D
:1065D000888405AA04A9184609F08FF8002804D079
:1065E00007200BB030BD1020FBE76A46127C3B4809
:1065F0000092801E05A9FF3201910290FF32002314
:1066000003A80332099904F040FC002802D0FEF7E9
:10661000FEFFE6E73148001F002D01D041882980A8
:1066200004700020DDE770B592B00446012608A88A
:1066300086702D496846018410AA08A93046FFF7E4
:10664000A9FF002840D12078244DC00700242D1F29
:1066500000283BD01C21684613F05CFD6846017899
:10666000202001436846017008A886701F496846CB
:10667000018411940794817FF92001406846891CA8
:106680008177002001466846017700200146684670
:10669000417704218185C485018607A80A9011A845
:1066A0000D9008A809900EAA09A96846FFF746FDB3
:1066B000002809D16846008FE8806846808F2881CD
:1066C000401C68812C70002012B070BDEC802C81C1
:1066D00010A80088F4E7000003280000C80200208A
:1066E000030200000329000001180000052A000031
:1066F000F7B5FD4900260A789EB0012A04D0022A87
:1067000002D0082021B0F0BD4A88824201D0062084
:10671000F8E71F98824201D10720F3E7012210A970
:106720008A75F2488882002003239B020146994320
:106730009302CB1810A90B8669468A81EC4ACA815C
:1067400018A9887110A9888419A904916946CA8278
:106750000690FF20087503A804F06BFC0024254672
:10676000274608AA052103A804F066FC002810D0DB
:1067700082286FD1002C6FD0002D6DD010A884809E
:10678000C5800021017418A8807B11AC012865D058
:106790006DE008A88079002F21D0012857D16846E4
:1067A000818CD24881421CD113AA0DA905206B46C9
:1067B00007C36846408C10230022FF2104F0AEFC82
:1067C000002868D110A88089042801D006284CD15F
:1067D0006846818E1F98814239D10F2092E70128A7
:1067E00035D16846808C0521C902884202D0491CF7
:1067F00088422CD1BC4841886846408C814201D1F6
:10680000012700E00027002C01D0002D10D01F9997
:1068100088421CD113AB0DAA05216E460EC6044654
:1068200010230022FF2104F079FC002833D101E07D
:1068300035460CE010A88089022801D0102814D118
:10684000C0B21BAA0DA908F032FF00280DD168467E
:10685000468C86E71FE0FFE7052053E714A91BA835
:10686000221D08F04AFF002801D003204AE710A8A3
:10687000007C0023001DC2B210A802742098029070
:106880000194009215A81C9904F0FFFA002802D187
:10689000954902220A70FEF7BAFE33E710B50B469F
:1068A000401E86B084B203AA00211846FEF7A4FF5A
:1068B00004AA052103A8029201910090012300225D
:1068C000FF21204604F046FA04466846008A012863
:1068D00001D013F04AFD2046FEF799FE06B010BD28
:1068E000F0B5814F0446387887B00E46032804D0AF
:1068F000042802D0082007B0F0BD04AA03A920464E
:10690000FEF753FF0500F6D1606880784007800FDE
:1069100002280DD1684680898004800F08D0206944
:10692000002805D073490968884201D21020E2E7A7
:10693000208905AA6B46216907C369460A8A6389CB
:106940002068039904F0A1FA002802D0FEF75FFE48
:10695000D1E7002E02D06846808A3080042038704B
:106960002846C8E738B50C00054609D000236A461A
:10697000FF2104F035FC002804D0FEF748FE38BDA6
:10698000102038BD69462046FEF7B9FE0028F8D130
:10699000A078FF21C307DB0F2846009A04F048FCCB
:1069A000EBE73EB50C0009D002AB6A46002104F0CB
:1069B00017FC002804D0FEF72AFE3EBD10203EBD85
:1069C0000321204613F0A4FB6846008801A90005B6
:1069D000800FFEF780FE00280BD1684600792070FA
:1069E0006846008801A98004800FFEF774FE002825
:1069F00001D003203EBD684600796070A278EF2088
:106A0000024068460088C10B09010A43F7210A4089
:106A10004104C90FC9000A43A270F9210A40800647
:106A200001D5022000E00120400069460243097AB6
:106A300050084000C907C90F0843A07000203EBDA0
:106A40007FB514460522019203AD029500930A46D4
:106A50002388FF2104F07EF9694689892180FEF7A9
:106A6000D6FD04B070BDF3B5002691B068460C4663
:106A70008686354600291CD0E068002806D0A0682C
:106A8000002816D001886A46918606801198FAF788
:106A90002EFE002810D0007822286FD3119800F025
:106AA000A7FC00900421119806F096FF070007D17B
:106AB00004E0102013B0F0BD0F48FBE713F055FCC5
:106AC000A078012803D0022801D00720F2E720880F
:106AD000002813D0401E80B203AA009904F07DFA6A
:106AE000002862D127E00000C40200200228000034
:106AF000FFFF00001C00002002300000FE48D9E724
:106B000069464A8A21888A420BD26846807D0025E0
:106B1000012810D16846808AF84988420BD10125A6
:106B200009E08A4203D1002D2BD06D1C01E0022D1B
:106B30000BD0032D04D203A804F058FA0028DFD0AC
:106B400082281CD0002830D11EE06946897D0129A9
:106B5000F1D16946E94B898A5B1ECA1A994210D065
:106B600005DCE748081A0CD00128E4D109E0012A25
:106B700007D0FF3A012ADED10325E1E732E0022DFA
:106B800013D10D20800295E7E068002814D00DA9EC
:106B9000052202910192009069468B8EA28820887E
:106BA000FF2104F0D7F8002802D0FEF730FD81E77E
:106BB0006846A168808E08806846008AC00601D5B4
:106BC000D04877E70798002803D06846008B022852
:106BD00001D003206EE70798A1780078012903D03F
:106BE000800710D4082065E7C007FBD000220721EA
:106BF000119801F0E4FD002802D00725022004E0EE
:106C0000BD48401C56E70225032008A908702188CA
:106C1000684681841721018700960FAB00220196F8
:106C2000119801F0A3FA0028ADD111980837009609
:106C3000019002970EAA052108A80F9B03F0CFFC34
:106C4000002802D0FEF71AFD34E70F98009068463E
:106C5000038F04222946119801F065FC2AE770B5DC
:106C6000064615460C460846FEF78EFC002804D161
:106C70002A4621463046FFF78DFC70BD10B5FFF760
:106C800037FD10BD70B51E4614460D0014D0002C03
:106C900012D0616800290FD00121FEF7B1FE002853
:106CA00009D12068FEF770FC002804D13246214645
:106CB0002846FFF743FA70BD102070BD70B5154629
:106CC0000C000ED00221FEF79BFE002808D12068A0
:106CD000FEF75AFC002803D129462046FFF700FEA4
:106CE00070BD102070BDF8B5064687480D46016896
:106CF00014468A4231D36068002807D0834A904204
:106D00002BD3834A904201D3884226D381488642BE
:106D100004D03046FAF7EBFC00280CD0304600F0E7
:106D200067FB0646284600F001FB002805D1606895
:106D3000002803D013E07048401EF8BD00236A46C7
:106D40003146284604F04CFA002802D0FEF75FFCDA
:106D5000F8BD68460088800601D41020F8BD61881F
:106D6000224628466368FFF76BFEF8BDF7B5664E0E
:106D70000746306886B01446824202D2102009B01D
:106D8000F0BD384600F034FB05466248874201D02A
:106D9000FF2D08D0002304AA2946079804F020FA02
:106DA000002827D102E05448401EE8E76846008AE0
:106DB000C00601D55348E2E703A900200291052748
:106DC000019000976288534B2946079804F0A6F972
:106DD00000280FD161683268914208D30191029076
:106DE0000097238862882946079804F097F9694636
:106DF00089892180FEF70BFCC1E7002906D0464BAC
:106E00000A881B899A4201D83B4870472BE610B587
:106E100086B004236C46A3823F4BDC88002C06D04E
:106E20001B898B4201D2914203D9334856E5062093
:106E300054E56B4619825A820021009101911C8011
:106E40000221997005A9029104A903916946FFF7EF
:106E50000AFE43E5F3B50C4683B081202B4F69460B
:106E60000872BC425BD32A48844203D32648006898
:106E7000844254D30398FAF73AFC060010D03078D5
:106E8000222826D300220121039801F098FC002833
:106E90000AD00421039806F09FFD050008D105E003
:106EA0001548401E05B0F0BD1120FBE713F05DFA58
:106EB0002846083002F0D0FF2178012903D00229AA
:106EC00004D00720EEE7820703D504E03422104205
:106ED00001D10820E6E7241DA278D20721D0E2885C
:106EE000002A1ED0A268BA4219D3094B9A4218D37D
:106EF000054B1B689A4211E0033000000328000094
:106F000000280000013400001C00002000B0010037
:106F100000000020FFFF0000C402002001D210206A
:106F2000C0E7228802AB00F0CBF90028BAD168464E
:106F3000017A20367078019100906A8823462946AC
:106F40000398FEF76FFDADE7FFB58FB0002004900A
:106F50001E4615460C460F460F98FAF7C8FB002848
:106F600004D00078222803D20820A3E5F948A1E53F
:106F7000B00801D007209DE5032E00D100260F9810
:106F800000F036FA0390002C28D0022D7ED3F2496F
:106F90008C4212D3F14AF24B944202D318688442D5
:106FA0000BD360190090012809D0401E884204D3F9
:106FB000904204D31968884201D210207AE5AD1EB0
:106FC000AAB22146E74804F025FA00991E394A7F03
:106FD0000B7F11021943884269D1ADB2E248B10773
:106FE00002D50189491C00E0012189B20091F10715
:106FF00001D0068900E0DB4E05AA0399009803F052
:10700000ECFF0DE0F878B9780002084310284ED85C
:107010000499091D401880B20490A84247D8271847
:10702000002F62D0787839780002084300998842AE
:10703000E8D35AE06946098B0A0756D5002C41D09F
:10704000049AA718121D92B20492FA78BB78120221
:107050001A439446102A2AD8049A6244AA4226D88F
:107060007A783B7812021A43904220D1C80620D584
:1070700004990DAA05206118029200910190787878
:107080003978000208436346002200E00FE00399CC
:1070900003F060FE002802D0FEF7B9FA0AE5F8789E
:1070A000B978000208436946898E884201D00B20D6
:1070B00000E5F878B978000208430499401880B2D6
:1070C000049006E0C90604D50399FEF700FD0028E8
:1070D000E4D16846018B1020814368460183408BD0
:1070E000FF23069A039904F0A3F805A803F07EFF96
:1070F000002803D16846408BB0429BD904210F98E9
:1071000006F06AFC040001D113F02FF92288002A4E
:107110000CD00025052000902B46214601950F98A4
:10712000FEF780FC0028B9D12580C3E40020C1E42B
:10713000F0B500248DB01F4616460D46002A1AD021
:10714000B90802D007200DB0F0BD032F00D10027F1
:1071500000F04EF90390FF280FD0002D0FD080488B
:107160000068854207D331884A19012A07D06A1E70
:107170008918814203D21020E5E77648E3E77A498F
:10718000B80701D5488900E00120FA0702D04989F3
:10719000491E00E0734905AA8FB2039903F01DFF51
:1071A00038E06946098B090734D504AB0521002274
:1071B0000293009101926B4B039903F0AFFF0028FB
:1071C00021D1002D21D06A46128A3188A2182819AF
:1071D000121D914234D369464A8B0270120A4270E2
:1071E0000A8A8270120AC27004A90522001D009248
:1071F000029101906946488B0B8A0022039903F0A3
:107200008DFF002801D003209DE76846008A2018E2
:10721000001D84B205A803F0E9FE002804D08228EE
:1072200006D0FEF7F4F98EE76846408BB842B8D92D
:10723000002C07D0002D10D03188A01C814203D231
:107240000C2080E705207EE722462946454804F0C9
:10725000E1F829190870000A4870A41C3480002045
:1072600071E73F490968884201D2102070473E49C2
:10727000498901800020704770B5064614460846CB
:1072800020430DD0364D00290CD0286881420ED302
:10729000304603F0FEFF002804D0FEF7B8F970BDB9
:1072A000072070BD002C09D02868844201D210202C
:1072B00070BD21463046FFF774FB70BD002070BDE5
:1072C000F0B51C46002A13D0D31FFA3B81251F4678
:1072D000D6B2112B1BD23B0013F062F911250D1011
:1072E00025222515221325252222222225222500AA
:1072F0000020187015E0022915D011E0012912D0E4
:107300000EE0C00600E0800600280CDA08E0104617
:10731000FF3881381F2803D9FF3AFE3A022A02D8E3
:1073200026700020F0BD25700720F0BD00B585B0A7
:107330006946FEF7CDFA00280AD16846007C0300B2
:1073400013F02EF908053B3B3B3B1414053D03208D
:1073500005B000BD0230000000B0010000000020B8
:107360001C000020FFFF0000C40200206846807857
:10737000012807D1684600880321C902401A1CD0A1
:1073800001281AD068468079012806D1684680888D
:1073900015214902401A05280FD96846807A01282C
:1073A0000FD16846018929200002081A05D0022859
:1073B00003D0032801D0042803D10F20C8E712F01E
:1073C000D4FF0020C4E770B50C4605461A212046BC
:1073D00012F09EFE00202080002D06D0012D02D04C
:1073E00012F0C3FF70BD062000E00520A07070BD44
:1073F00010B506F0BBFA10BD10B50C4603F0C0FD89
:10740000002801D012F0B1FF2046FEF700F910BDB0
:107410007CB50A460546694605F0FDFE04460BE0CC
:10742000002201A9284605F0F6FE044668460079C8
:10743000002801D012F099FF002C04D06A46107881
:10744000411E1170ECD220467CBDFFB597B0FE49BD
:1074500006460B9003C90A910990507A117A154695
:107460004018C7B2002E0FD00024F01C8008800006
:10747000B04201D012F079FF28880B99401C80B2ED
:107480000090002C02D008E00124EEE7C0B208F022
:10749000AFF8002801D012F068FF00980B990001A6
:1074A00008182969C01C0C91810889003A460B9183
:1074B000002C09D1002008700C9880B203F017FC52
:1074C000002801D012F051FF0B990C9823460818A0
:1074D0000B90A87A297A3A464018C1B20BA800F05E
:1074E00027FD0B98C01C800880000B90697A0091E2
:1074F0002B7AAA7A002C00D000200CA906F058F9AB
:10750000002801D012F031FF6946098E0B98BC4665
:107510004018C01C800880001A9F209B219A229945
:107520000192009302910B90002C00D000203B466A
:10753000624604A906F006FB002801D012F015FFF0
:107540006946098A0B984018C01DC008C000821BFC
:1075500018990B900A60002C54D101210907C96ABF
:10756000C9430906090E03D1B8490968491C03D06B
:10757000B749401AB749C86201222C21B64806F023
:10758000ABF803F0B9FEB54C6178A06804F0CBF815
:10759000E068401E07280BD8302269460A708870C0
:1075A000684605F076FB002802D00CA804F083F9A9
:1075B00000211E22084601F07BFEFAF7CBFF00F007
:1075C0002DFFFEF7DDFC09AB00220521A4A0FBF78F
:1075D00025FD002801D012F0C8FE28460C30FFF728
:1075E00022F8002801D012F0C0FEFF2189009E4839
:1075F00012F090FD984801211C38417602218176D5
:107600000621C1761BB0F0BD10B5974CA0780928B3
:1076100001D312F0AAFE20787021484300190021FE
:1076200001714179F722C908C900C91C1140EF2234
:10763000114041710121E170001D10BDF8B50D46EA
:10764000014600201E46188014460B0012F0A8FFC9
:10765000074F050B17114F1D4F0032462146284694
:1076600000F034FFF8BD324621462846FAF73FFCC9
:10767000F8BD324621462846FEF743FBF8BD3246A8
:1076800021462846FDF7FAFCF8BD0020374606469D
:10769000009028780009062801D012F066FE287EA6
:1076A00000280BD0012812D012F05FFE3E80002C83
:1076B00002D00098208066800020F8BD02200926B4
:1076C0000090002C11D0A88BA080A87F0BE0032095
:1076D00014260090002C08D06888A080286AE060FA
:1076E000A88C2082287F2072E0E73E80E4E712F039
:1076F0003CFE0320F8BD70B55B4CE07800281BD041
:107700002078702148430019407900254007400F38
:1077100001191F2040010918087E401E08762078B4
:10772000401CC0B22070092800D12570A078401CF0
:10773000A07009F06EFCE57070BD47481C38C07E33
:10774000002800D060E77047F0B5434D002687B0B1
:107750007C3D686F00280BD0FFF7EFFF002872D048
:107760007022696FF9F712FDFFF7C5FF6E67F0E74A
:1077700039481C38407E002865D0FFF745FF044695
:10778000354805F0BCFF6060002801D112F0EDFD26
:10779000606803F012FE002811D02046FAF775FA4F
:1077A0006078010706D5C008C000401C6070FFF774
:1077B000A2FFCEE72848616805F0AAFFC9E726487E
:1077C000616805F0A5FF01A800F0EDFB002875D168
:1077D00068460321808806F0FFF80290684680889A
:1077E00006F0BDFA07460298002801D112F0BDFD4F
:1077F00002984068002802D00078FF285ED0FFF78A
:1078000003FF0446211D3846039105F0B8FE002809
:1078100003D003980068067001E012F0A6FDA08A6C
:10782000002801D012F0A1FD606803900670684640
:1078300080886080204600F08CFE384605F0D2FE3D
:10784000002815D112E039E0C8A501000010001091
:107850000000002000050040200700201800002044
:107860006E524635780000002403002012F07DFDA2
:107870006078010702D4C00606D409E0C008C00041
:10788000801C6070FFF737FF02980399416060E742
:1078900002984168002908D00878401C0006000EB4
:1078A000087086D112F061FD53E700213846FFF7DA
:1078B000AFFD0028EBD112F058FD4AE707B0F0BD4C
:1078C00010B5FE4CE160A060FD4801F05BFC60700B
:1078D00010BDFA4900200870704770B5F94E054692
:1078E000706A94B00C46401C04D1B06AC0430004D6
:1078F000000C0BD0306AC007C00F2870706A12F0FD
:107900000BFCB06A2071000A607111E02B206946FF
:10791000087009A9684603F02AFD002801D012F07A
:1079200024FD0120287006220AA9204612F093FBAC
:107930002878002803D06079C0210843607114B012
:1079400070BDF0B5DF4C0646206895B00D46374651
:107950000837401C08D16068401C05D1A068401C55
:1079600002D1E068401C11D02068314612F0D4FBEF
:107970006068311D12F0D0FBA068394612F0CCFBD4
:10798000E06831460C3112F0C7FB1FE02B2069463E
:10799000087009A9684603F0EAFC002801D012F03B
:1079A000E4FC08220AA9304612F055FB2B20694658
:1079B000087009A9684603F0DAFC002801D012F02B
:1079C000D4FC08220AA9384612F045FB20692E464D
:1079D0000836401C08D16069401C05D1A069401CD4
:1079E00002D1E069401C12D02069294612F094FBB4
:1079F0006069291D12F090FBA069314612F08CFBE2
:107A0000E06929460C3112F087FB15B0F0BD2B243C
:107A10006846047009A903F0AAFC002801D012F0FE
:107A2000A4FC082209AF28460AA912F014FB6846F4
:107A3000047009A903F09BFC002801D012F095FC0A
:107A40000822391D304612F006FBDEE730B59E4CA9
:107A50000546606F002801D012F087FC656730BDD5
:107A600038B50546032105F0B7FF0446284606F061
:107A700076F90546002C01D112F077FC60680028E9
:107A800004D00078FF2801D112F06FFC6946284627
:107A9000FFF7BEFC002801D112F067FC6068009976
:107AA000884201D100206060874C6034A07E0228AB
:107AB00001D312F05AFCA07E401CC0B2A07601286F
:107AC00003D17E48407801F07FFB38BD70B5044695
:107AD0007E4816460D46814201D112F046FC012E29
:107AE00002D012F042FC70BD66202070002020768B
:107AF000A5830120A07770BD70B515460C460646DB
:107B0000FFF71BFE00280CD0662101704680012182
:107B1000017621680162A18881840577FFF7EBFD7A
:107B200070BD13213046FAF7E9FF70BD70B5054608
:107B300062480C464068814201D2102070BD284640
:107B4000F9F7D5FD002805D0284606F01DF90500F7
:107B500004D101E05E4870BD12F007FC284605F034
:107B600096FD222112F0E0FAC0B2062801D9801F4A
:107B700000E000202070002070BDF0B504464F48A2
:107B80000F4601788BB0002902D008200BB0F0BD61
:107B9000504941608C4201D38F4201D21020F5E759
:107BA000617A227A8B18FF2B27D82088FE2824D8C8
:107BB000082B01D90420E9E7002800D10A20208001
:107BC0002069002801D10B20C0010A230D254B4359
:107BD0005543ED184B000626CB185643F6181B23C9
:107BE0007343206107931B236B430693D82801D26C
:107BF0000920CBE7A07A884201D90720C6E7606850
:107C000000F06AF909900028C0D10698029580B268
:107C1000069001900798009683B2224604A900209E
:107C2000FFF713FC2548049940683A680918914207
:107C300002D90C203960A9E70699029501910799AC
:107C400022468BB2009605A91C4CFFF7FEFB059956
:107C50000498884201D012F088FB059861684018AA
:107C6000606038600120207009988FE7F8B50546FC
:107C700012480F464068814208D3002D01D085424A
:107C800004D3E81C80088000A84201D01020F8BD71
:107C900011488178002921D03988009141787022DB
:107CA00051430C182079241D0007000F3B46002289
:107CB0002146FFF7C3FC060014D025E01800002081
:107CC0004977000080000010A4060020FFFF00009C
:107CD00002300000F0100020240300200020388033
:107CE0000520F8BD002D13D039880098814201D9B4
:107CF0000C260DE020783B460007000F2A4621465F
:107D0000FFF79CFC060005D00C2E01D00020388027
:107D10003046F8BDDD484178491CC9B24170092997
:107D200001D1002141708178D94D491E8170607860
:107D30004107490F01290CD0022904D0032918D08A
:107D400012F013FBE4E7C006E2D46088FFF788FE78
:107D5000DEE7CF4861681C3005F0DAFC687E401C25
:107D6000C0B268760128D3D1CA48407801F02CFA15
:107D7000CEE7E87E401CE876CAE7C74A10B59042D5
:107D800008D3C44AC54C5268A04201D3904201D3E3
:107D9000914201D2102010BD07F063FC10BDBE4B14
:107DA00010B5994208D3BB4BBC4C5B68A14201D3D0
:107DB000994201D39A4201D2102010BD022803D06B
:107DC000102801D0092010BD07F071FC0028FAD05E
:107DD000052010BDB04B10B598420CD3AD4BAF4C45
:107DE0005B68A04201D3984205D3994203D3002A8D
:107DF00003D09A4201D2102010BD07F07EFC00286B
:107E0000FAD0072010BD10B50446A24894B04068CF
:107E1000844202D2102014B010BD0F2008A90873AC
:107E200069460BA803F0A3FA0028F4D16846007A4B
:107E3000207068464089608068468089A080002064
:107E4000E9E710B500290BD0924A5268914202D35B
:107E50000B68934201D2102010BD8A88002A02D0FC
:107E6000FEF7DFF810BD092010BD8B4A10B5914216
:107E700006D38A4A914205D3864A5268914201D27A
:107E8000102010BD421E1E2A02D800F0C7F810BDF7
:107E90000246203A1F2A02D8FAF7A7FA10BD072097
:107EA00010BD10B57B4A5268914208D3421E1E2A6B
:107EB0000BD8794A914202D3012804D101E0102065
:107EC00010BD062010BD072010BD0246203A1F2A13
:107ED000F9D8FAF7FBFA10BDF0B500280AD06E4BBE
:107EE000984206D36D4B984205D36A4B5B68984223
:107EF00001D21020F0BD8378467805789B195B1974
:107F00008C189C4206D147790379C078FF183F1836
:107F1000BC4201D00720F0BD954205D1904203D16B
:107F20008E4201D18B4201D00620F0BD0020F0BD71
:107F3000F8B506460220002A02D050004018401D25
:107F4000C7B23068C01C820892003260002B25D175
:107F50004E483B460A21283809F070FB002408E00F
:107F6000230012F01DFB0A0608060A0A0C0C06067E
:107F700006114B4804E04B4802E04B4800E04B48F8
:107F800009F07CFB054601E012F0EFF9A54201D0B3
:107F900012F0EBF9641CE4B20A2CE1D33068390129
:107FA00040183060F8BDF1B594B03A2008A90873C4
:107FB00069460BA803F0DBF9002801D012F0D5F9CF
:107FC0003B4E00246D4623E02F19B87DC10706D033
:107FD000400704D460004019C08800F0D8FB2C484A
:107FE000807E002812D0B87D80070FD56000401930
:107FF000C0880022062100F0E2FB002806D06000C5
:108000004019C18814980026018005E0641CE4B280
:1080100068460079A042D7D83046F6E41E4A91421D
:1080200006D31E4A914205D31A4A5268914201D2A0
:1080300010207047012802D0022812D121E00A78CE
:10804000022A04D0012A02D01948401C70474878FF
:10805000002806D0032804D88978002901D00329F4
:1080600001D907207047022A02D0012A09D104E071
:10807000022806D1022904D105E0032801D10329F1
:1080800001D0062070470020704700002403002024
:10809000040700201800002000B0010000000020AC
:1080A0005B2200008F840000E92F000021F5000012
:1080B00004300000FFB581B00A9F164638460B30E9
:1080C000C5B20C46019800F063FCA84206D2072E08
:1080D00002D0112005B0F0BDF948FBE7607B1E28F7
:1080E00001D312F042F9A078C0091FD10B980022E9
:1080F000011FC01F02700F70380A48700498887002
:10810000000AC870019805F03FFE0090002801D1D8
:1081100012F02BF93F1DB9B2009805F0C8FA0028FB
:1081200001D112F022F9019803F079FA207B617BEA
:108130004018491CC0B261731E2801D31E38C0B25A
:108140004100401800198673C17BF122490849009B
:108150001140C1730574072E04D06089401B6081F3
:108160000020B7E72089401B2081F9E7FFB585B0E3
:108170001D4616460F9F05F007FE040001D112F0C0
:10818000F4F806986946001D82B2204605F08BFA85
:10819000002821D068460089042801D212F0E5F8B1
:1081A000002E03D068460089001F3080002D02D0C9
:1081B0000198C01D28606846008A002801D012F08E
:1081C000D4F80E990020002900D00880002F00D09C
:1081D0003860002009B0F0BDB948FBE7F0B50F46A4
:1081E000054687B016465088032105F0F5FB0400CC
:1081F00001D112F0BAF8002069460872A078400652
:1082000001D112F0B2F8042F5ED32978C807C01745
:10821000401C06D162786B789A4255D122781207B9
:1082200052D0142947DA012943D0122902D0132948
:1082300041D129E00C2F3ED1A1784906490E0129F0
:1082400039D02078012100090001401C2070687895
:1082500060706846017268792A79010211436846A4
:108260008181E879AA79010211436846C181687A5F
:108270002A7A0102114368460182E87AAA7A010249
:108280001143684641821AE0062F14D12078000974
:10829000000120707188012009F091FA02216846DE
:1082A0000172C91E818168792A79010211436846E9
:1082B0001FE0062F0AD06946097A00291BD0708872
:1082C000324602A9FAF73FF807B0F0BD207800095E
:1082D000000120707188012009F071FA02216846BE
:1082E000017268792A79010211436846818100216F
:1082F000C943C181E3E70028E6D0274676880024F9
:10830000009405AB2246062130460194FFF72EFF6C
:10831000002801D012F029F8059801210170697830
:108320004170022181700021C1700471210A4171E4
:1083300006210523009101901A4639463046FFF781
:10834000B9FE0028C0D012F010F8BDE7F7B584B030
:10835000154604990598FCF7E1FFC0B20828B3D18F
:108360000020694608816888032105F035FB040078
:1083700001D111F0FAFF01230021207B627B0CE088
:10838000460086193619B67B9E4201D1491CC9B2F6
:10839000401CC0B21E2800D100201646521ED2B288
:1083A000002EEDD1002902D1172069460881002056
:1083B000009001906946688803AB00220989FFF7A5
:1083C000D5FE002801D011F0D0FF009502AA039B32
:1083D00004990598FDF790FEC0B2030012F0E0F892
:1083E00005041B1516151B006846008900280CD0D3
:1083F0000399019100906888042301222146FFF728
:1084000059FE002801D011F0B0FF5DE76878102117
:108410000843687058E711F0A8FF55E70020294984
:1084200002464300401CCA520828FAD37047002174
:108430008170017809090901017001214170002151
:10844000416001734173704770B50D46032105F01B
:10845000C3FA040001D111F088FFA0786906C009B1
:10846000C001490E0843A070012D02D0022D02D098
:1084700003E0EE2000E066202081CC20608170BD0A
:10848000704710B50146012009F099F910BD3EB5BD
:108490008DB20321284605F09FFA040001D111F0A6
:1084A00064FF2078694600090001207002200870EE
:1084B00005488880C88000222846F9F744FF3EBD61
:1084C0000430000050070020FFFF0000F7B505460C
:1084D0000078002700090C463E46012801D011F023
:1084E00044FF287E032809D011F03FFF0298002C9A
:1084F000068001D0278066800020FEBDEA8B7027B1
:1085000010460A3086B2002C0AD06888A080A88B5A
:108510002081E28020460A30296A11F09CFDE5E7BF
:1085200002980680E8E7FFB583B00F461C46164662
:1085300003210C9D039805F04FFA010007D0334644
:108540003A46019500940398FFF7B4FDBCE6FA485B
:10855000BAE6F8B5024680680179C3780902194382
:10856000837944791D0293892543C01C1B1F9942BE
:108570001AD1042D19D0052D22D0062D19D0402D49
:1085800012D3061D0F461446284600F007FA0828A5
:108590000AD01120207003202076A583E78326626D
:1085A0006078082108436070F8BD001DFFF7CEFE1B
:1085B000F8BD031D50880A461946FBF76DFBF8BD50
:1085C000001DFFF70BFEF8BDFEB50D460646032164
:1085D00005F002FA040011D020780007000F0128EE
:1085E0000AD0002000900246019002AB0C213046D8
:1085F000FFF7BCFD002803D01120FEBDCE48FEBD14
:1086000002981221017061780523891C41700821AC
:1086100081700021C17029880171090A417169883E
:108620008171090AC171A9880172090A4172E98838
:108630008172090AC1720C21009101901A462146EB
:108640003046FFF737FD002801D011F08EFEF023F1
:1086500000223146012009F022F8207800090001AB
:10866000401C20706078801C60700020FEBDFEB54C
:108670000D460646032105F0AFF9040006D0207828
:108680000007000F012803D00820FEBDAA48FEBD48
:10869000002000900246019002AB06213046FFF711
:1086A00065FD002801D01120FEBD02981321017044
:1086B00061784170022181700021C1700571290A21
:1086C000417106210523009101901A46214630464A
:1086D000FFF7F0FC002801D011F047FE20780009D8
:1086E000000120700020FEBDF3B583B00D460321CC
:1086F000039805F071F9044600200090002C01D188
:1087000011F033FE607BA8422BD211F02EFE28E040
:10871000207B410041180E19401CB77B317CC0B250
:10872000019120731E2801D100202073607B401E20
:108730006073F07BC00704D00398042F18D011F0A9
:1087400014FEF07B0107480F05D0490F0398042958
:1087500011D011F00AFE072F10D061890198081876
:10876000608128466D1EEDB20028D1D10098B1E499
:10877000FBF726FBE5E7FBF7EBFAECE70098401C7C
:10878000C0B200902189019808182081E9E710B54E
:10879000032105F021F9040001D111F0E6FD207B51
:1087A000617B4018C0B220731E2801D31E3820738D
:1087B00000206073A07880210843A07010BDF8B538
:1087C0000D4617460646032105F006F9040005D0BC
:1087D000002D08D0002F03D0062002E00120F8BDB4
:1087E0000820A84201D811F0C0FD2A462146304693
:1087F00000F0CEF8222111F097FCC6B2002F27D04E
:10880000002E25D1207B617B1EE0420082181219C8
:10881000937B072B03D0D37B1B075B0F04D0401C3B
:10882000C0B21E280DD00DE04300C0180019C07B57
:10883000F12318406B071B0F1843D073002907D191
:1088400004E00020491EC9B20029DED111F08DFDDF
:108850003046F8BDF8B50D46032105F0BDF804001B
:1088600001D111F082FD681E052801D311F07DFDB4
:108870001E21227B607B002311E0560096193619D9
:10888000B77BAF4206D1F17B49084900F1735B1C0D
:10889000DBB21146521CD2B21E2A00D1002206467B
:1088A000401EC0B2002EE8D11E2906D2480008188A
:1088B0000019C17B01221143C1731846F8BD10B5E0
:1088C0000446402801D2072010BD00F067F80828B0
:1088D00002D03120000210BD0021184802E0491CDE
:1088E000082903D24A00825A002AF8D1082903D065
:1088F00049004452002010BD042010BD10B540288E
:1089000001D2072010BD00F049F8082805D0002149
:108910000A4A40001152084610BD052010BDFEB5A0
:1089200015460C0006460BD0002D09D06088402863
:1089300008D20720FEBD00000230000050070020D2
:108940001020F7E72188002901D0172901D90C2030
:10895000F0E700F023F8082818D0002000900190DC
:108960000246218802AB3046FFF700FC0028E1D127
:1089700022882946029811F06EFB02980090238805
:10898000628807213046FFF7CEFDD3E70520D1E707
:10899000072A01D04889704708897047014600209E
:1089A000044A02E0401C082803D24300D35A8B42F9
:1089B000F8D170475007002030B40121BA48C902ED
:1089C0000160CD1005604A030260B84803681C02CC
:1089D000240A002304600468240A24020460B448C2
:1089E0000468240A24020460B248012444608460BC
:1089F000B14C23606360A360B04B19601D601A60C6
:108A0000AF4B19601A600121016030BC704710B48F
:108A10000121A548CA0202600B0203600C06046033
:108A2000A44841608160A74841680029FCD1A2495F
:108A30000020086048608860A0480260036004600D
:108A400010BC704701219D48C9020160C910016036
:108A50007047002805D0012805D0022805D19A4882
:108A600070479A4870479A48704700B511F07DFCEE
:108A7000002000BD30B50021964C974D974A8E4B93
:108A8000002806D001281BD0022820D011F06DFC50
:108A900030BD01200004A060A86011601960904BF7
:108AA000C2039A608F4A90607F4A001210608E481D
:108AB0000160864801608D4801608D48017030BDBD
:108AC00001204004A060A8605160596030BD0120C1
:108AD0008004A060A8609160996030BDF0B59446B4
:108AE0007C4A844F7C4E00240125002806D00128B2
:108AF00030D002283ED011F038FCF0BD891E0902AA
:108B0000090A0120000490603C6470606D4A1164A1
:108B1000012B1DD00021764B6246597076494D607D
:108B2000CD6076494C6002248C6004240C616E494F
:108B30003D320A606D490D60604A89151160694ACD
:108B400050605F4801606649C00548601D70F0BD17
:108B50000121E0E701206A4D40046A4F012B04D156
:108B60002C64506070603964F0BD90602C6470605B
:108B70003964F0BD0120644D8004644F012BF4D1B1
:108B8000EEE750484068704770B54B4D28680026A6
:108B9000504C012806D1A068C00303D50120000471
:108BA000A0602E606868012809D1A068800306D5FE
:108BB00001204004A0606E60012007F03CFDA86821
:108BC000012809D1A068400306D501208004A060D7
:108BD000AE60022007F02FFD70BD10B54449087843
:108BE000002818D001203E4AC00790603D4AC00BC3
:108BF00090602D4A001210603B4A00201060334AFA
:108C000010603A4A106008704A78002A02D0487012
:108C100007F011FD10BD0320FAE701203C490006D2
:108C20000860704701202549000608607047012050
:108C30003749400508607047012020494005086019
:108C400070472D4801214160C1601C4980150860B2
:108C50007047410A2F4AC005C00D5043FF30013014
:108C60005143400A0818704710B42B4C430B634320
:108C70001B0C5C020C60274C6343C31A27485C0240
:108C80005843244B400D4343E31A0124DB03E4051E
:108C90001B191B1613700A681018086010BC704767
:108CA00010B507F092FD10BD80E100E008E400E09F
:108CB00018E400E000B0004040B1004080E200E075
:108CC00000E100E000B5004048B1004040810040B4
:108CD00044B1004000B3004040B3004040B5004004
:108CE00000F50140008300404085004000820040C4
:108CF0002800002000B100400080004000850040B6
:108D000004B1004004B5004008B1004008B500407F
:108D100000E200E0093D0000378600006F0C010012
:108D200010B507F040FD10BD03490020C86303499A
:108D30000220086070470000C01F004080E200E091
:108D400010B5EFF31080C407E40F72B6C548417840
:108D5000491C41704078012801D108F077F9002CB6
:108D600000D162B610BD70B5BE4CE07800280AD1C3
:108D70000125E570FFF7E4FF08F070F9002804D042
:108D8000002008F04BF9002070BDB748A571456080
:108D9000F9E770B5EFF31080C507ED0F72B6B14C6F
:108DA0006078002801D111F0E0FA6078401E607010
:108DB0006078002801D108F04DF9002D00D162B68D
:108DC00070BD10B5A748C178002904D00021817179
:108DD000C170FFF7DEFF002010BD10B5044608F09B
:108DE0003DF9A049C978084000D00120206000204A
:108DF00010BDF8B5024600269A4C3746E6710820A9
:108E000004210125130011F0CBFB0D080A0C0E10F4
:108E10001214161E26212325280065711FE002204A
:108E200001E061711BE0607119E01020FBE7202078
:108E3000F9E7012613E0FFF783FF08F00FF9002898
:108E4000FBD002260BE06171E57108E0102002E022
:108E5000202000E040206071F6E711F086FA08F06B
:108E600009F9002809D008F00BF9B04205D13046C5
:108E700008F009F90028FAD02EE001239B07DD60F5
:108E80007A4847607A498E61774A022151609D6035
:108E9000076178490A69D243D206D217521C009260
:108EA0000A6910231A430A6100E020BF6F48406836
:108EB0000028FAD0304608F0E6F80028FAD00098EA
:108EC000002804D16B480169102291430161664971
:108ED0000220886065484760E07900280DD008F0DE
:108EE000BDF8009008F08CFA0099634A002902D07E
:108EF000A260E06001E0E260A060002E01D0277176
:108F0000F8BD257100F08EF8F8BD10B5044608F0E4
:108F1000ABF8002805D053490120C8704A78521C8C
:108F20004A702046FFF765FF10BDF8B54F4DA868A1
:108F30000026012802D1AE6008F070F868680128A8
:108F400000D16E6028680127464C012812D12E609E
:108F5000A079002803D0002008F060F8A6712078DE
:108F6000002807D008F07AF8002803D001208007F5
:108F70000761A770207900282AD02869012827D105
:108F80002E6180074761E079002815D008F066F867
:108F9000009008F035FA0099002901D0E16800E05E
:108FA000A168411A022901DA8A1C11DC0099002902
:108FB00001D0E06000E0A060FFF7C2FE08F04EF8CC
:108FC000002804D0012080070761A77000E0277007
:108FD000E868012809D1A078002801D111F0C5F96D
:108FE000EE60A6702670FFF7D4FEF8BD10B51D4CDC
:108FF000E078002801D108F02DF801208107886170
:10900000A078002809D0194CE068002803D108F0A6
:109010003AF80028F8D10020E06000201249C0434F
:10902000886010BDF8B51048192787600F490020E7
:109030000860C86008F012F8BD070124094E002836
:1090400002D02C61B47000E03470FFF779FE06485E
:109050004760074970798863AC6104490020086162
:109060006C61F8BD2C0000200003004000010040AE
:109070000005004000ED00E0FFFFFF7F8107C90E03
:10908000002808DA0007000F083880082C4A800002
:109090008018C06904E080082A4A800080180068AF
:1090A000C8400006800F704710B50D20FFF7E6FF9F
:1090B000C4B20420C043FFF7E1FFC0B2844201D034
:1090C00011F053F920490120486010BD01211F4AC9
:1090D000480310601E4B00221A601E4A51601E4A4F
:1090E00010601E4A116019498039086070470121DB
:1090F000164A48031060194A5160154A0021116050
:1091000015490860704710B511490868012802D058
:1091100011F02BF910BD0C4880680022C0B20A6023
:1091200008F0B8F810BD10B5094801680029FCD056
:10913000FFF7E9FF012008494003086010BD000067
:1091400000ED00E000E400E000D5004080E100E038
:1091500000D1004000D3004080E200E000D0004099
:1091600001203B49400608603A4908603A490A68CC
:10917000FF231B029A4383121A430A603449803941
:109180000860704700B502460420344904E0C3007B
:109190005B181B79002B08D00346401EC0B2002B81
:1091A000F5D111F0E2F8FF2000BDC300CA50002243
:1091B00059184A718A7101220A7100BD274A00219B
:1091C000C00080180171704710B50446042801D30F
:1091D00011F0CBF82148E1000C182079012801D0CA
:1091E00011F0C3F86079A179401CC0B2814200D06F
:1091F00060710120164940068031086010BD70B5CD
:10920000154804250068154E0004800F144C0228F0
:1092100018D011F0AAF815E02078C1008819027959
:10922000012A07D1427983799A4203D04279827127
:10923000705880472078401CC0B22070042801D3A9
:109240000020207028466D1EEDB20028E4D170BDCC
:1092500080E100E080E200E018E400E06007002028
:109260003C0000200E4A12680C498A420AD1184775
:109270000B4A1268094B9A4204D101B508F0A2F8D2
:1092800003BC8E460749096809580847064807493C
:10929000054A064B7047000000000000BEBAFECA37
:1092A0008C00002004000020D0100020D0100020EE
:1092B00010B5FE4B586019721A80C90010F02AFFD1
:1092C00010BD00210180704710B50022D2430280FA
:1092D000032008F074FA10BD7047F0B50E4604463E
:1092E000017801208840F24999B0084000906168F7
:1092F00015460888EF4A904206D0009A002A06D008
:10930000EB4A521E104202D0012019B0F0BD009A63
:1093100010430880002D12D0002028702178EA1C0C
:109320000027681C01920B0011F03AF910F30E1699
:10933000233A59616F3CB4B08AB8F2F1F0F3207867
:109340000B28EBD00420E0E702212970A1890170ED
:10935000090A4170032097E004212970A189017056
:10936000090A41700198E1890170090A41700520DC
:109370008AE006212970A1890170090A41700199CA
:10938000E2890A70120A4A70218A0171090A417140
:10939000A28AE81DA16910F05EFEA08AC01D73E0DC
:1093A000082129702178082901D110212970A1896B
:1093B0000170090A41700198E1890170090A417040
:1093C0000520308020466A1D02A9103006F095F96C
:1093D00000287DD169463088097A401854E00A2176
:1093E0002970A1890170090A417003200BE00C214A
:1093F0002970A1890170090A41700198E189017001
:10940000090A4170052030809CE0A0898446400014
:10941000401C81B2308888425AD3052958D30E2087
:109420002870002008E0236942009B5A52195370AB
:109430001B0A401C937080B26045F4D33180B9E0C0
:109440009A48417A002973D0491E4172217B4068B5
:10945000C9004518A98828680822401808382169D9
:1094600010F0F9FD02216846017100214171286860
:109470000390A98868460181002101A8FBF787FDB8
:109480000020A880002E00D0308093E02978802230
:1094900011432970297840221143297029788909BC
:1094A000890112312970A1890170090A4170E2898C
:1094B000E81C216910F0CFFDE089C01C30802878BD
:1094C00041063FD5C00975D001216846017200E010
:1094D0002CE0002141723188091D81810495E189C8
:1094E000019808180590001D06907048017A68469A
:1094F0000177002102A8FBF74AFD074630880C30AF
:109500003080022F06D0002F54D065E03DE033E0DC
:109510001CE05EE065486946097F4268CB00D218CE
:10952000037A994202D29188002902D0042753E09D
:109530002FE0417A491C41721560308890800020EC
:10954000308049E06168A089888033E02978890902
:10955000890116312970A1890170090A41700198A9
:10956000E1890170090A4170228A681D616910F061
:1095700072FD208A401D46E7287880098001183056
:109580002870207B687002207EE7606801880904EB
:1095900001D4052720E0C088A189884201D0062790
:1095A0001AE01E202870012030806068018849047C
:1095B000490C0180009800280ED03C480022008809
:1095C000A1688300032008F06AF861682078887039
:1095D00007E00020308003276068009902888A43F2
:1095E0000280384691E6FFB59BB0249D0E460028C8
:1095F00005D0172803D82A882E4B9A4202D107207B
:109600001FB0F0BD3278530601D4D20901D0082032
:10961000F6E700226B461A705A701446327802AB95
:109620001793431E19939BB216939706CB1CBF0E3C
:109630001893821E711C3B0010F0B2FF209011F0B5
:1096400066F074F0B4F0D6F0EFF0EEF0EDF0ECF080
:10965000EBF0F0F0EAF0E9F0E8F0E7F090F0052840
:109660007CD1042168460170A9780171F078B27844
:10967000010211436846C1803179417070788006DB
:10968000800E0C282ED009DC801E030010F088FF0D
:109690000919661C662166246627660012282AD0EE
:1096A0000ADC0E2821D01028DAD121E08007002022
:1096B000FF710000FFFF000016281FD01828CFD12F
:1096C0001FE02878800701E028784007002845DA65
:1096D0004FE128780007F9E72878C006F6E72878F0
:1096E0008006F3E728784006F0E728780006EDE7E3
:1096F0002888C005EAE72888C004E7E728888004AE
:10970000E4E728884004E1E72A78920726D5032871
:10971000A6D105206A4610704878097800020843EF
:10972000908026E129784907F0D5062816D370786D
:1097300091B2012802D0022892D101E0022700E074
:109740001027062268460270727882710022828099
:10975000179AB01C1692BA1C18921EE0BDE042780F
:109760000378801C17901202891E16981A431991CB
:10977000028016983A46801C179910F06CFC169AD5
:109780001798D219921C19996B4616929A88C0198B
:10979000C91B521C9A80189A89B28A42DFD90029C3
:1097A0008DD1E6E028780007B0D519986A4681B2D5
:1097B0000720107000209080701C921D11E04378EB
:1097C00007781B023B431380C37887781B023B4317
:1097D00053806F46BB88091F5B1C001D89B2BB808C
:1097E000121D0429EBD2DAE72978C90675D50228BB
:1097F00073D30821684601700021C180717801711E
:109800008C4692B2B01C179919E091E098E086E07E
:109810006FE063E038E02DE021E015E0C4E043783C
:1098200007781B023B430B80831C4B606346D21AB4
:109830006F46FB8860445B1C92B2FB800831944504
:10984000EDD9002A49D194E02878800645D509222F
:1098500068460270AA888280169AC28012E0287830
:1098600040063AD50A206A461070A888908016985B
:10987000D08007E0287800062FD50B206A461070AC
:1098800016989080029174E02988C90525D5022890
:1098900023D30C20694608700020C88070780871B6
:1098A000844692B2B01C179914E0437807781B02E3
:1098B0003B430B80C37887781B023B434B80031DDF
:1098C0004B606346D21A6F46FB8860445B1C92B2C1
:1098D000FB8008319445E8D9B3E763E02988C904DF
:1098E00060D501285ED10D2168460170A98881806C
:1098F0003FE02988890455D5052853D30E226946AF
:109900000A70AA888A801899401F4A78097812023A
:109910000A436946CA800881701D039029E029889E
:1099200049043FD501283DD10F206946087020E049
:109930002A88120436D44A780B7812021A43EA8035
:1099400003282FD332789206920E1B2A26D011229A
:109950006B461A702A880123DB031A432A804A784F
:109960000B78110219436A469180C01ED080189866
:10997000029030788006800E1B2809D01D2807D061
:1099800003201E9907F01BFF2888C00BC003288006
:1099900068461D99FBF7FBFA204631E610226B461C
:1099A0001A70DCE70724F7E70824F5E700B597B05D
:1099B000032806D16A461070019100216846FBF722
:1099C000E6FA17B000BD0000FFB593B004460020D2
:1099D0001D9E049015981C9D1027082806D0E0694C
:1099E00001F0B0F8002809D03770CCE028880921B0
:1099F000384328801F980227017016E0E169012092
:109A000088710521E269C9029180E1698872E16982
:109A1000F8480881E16900208873288820210843DC
:109A2000288011211F98042701701F980225801C8F
:109A30000390307810900A20307020461830119032
:109A400001F0F7FA00206FE01598102809D1022DD7
:109A500007D06846828A04990398401A8270110AD6
:109A6000C1706846C08A1699884203D9E249097ACA
:109A7000149106E0884204D11099002901D0317078
:109A800021E003990870000A48701E980088401B66
:109A9000C01B83B2FF20C01B984200D2034603982C
:109AA000149AC0190CA90092019002912020015D26
:109AB0006846C08A002201F031FB3070002806D0D1
:109AC000C0B2832862D06846C08A208345E00F98E0
:109AD000002805D0C848006800790A2830D33CE047
:109AE0006846008EC119C9B20491022D0FD01F998A
:109AF000049A4978914203D16A46128C824209D075
:109B0000BD48049100680178032909D027E0084680
:109B10001F994870B84800680178042906D008E009
:109B200000790A281BD201200F9009E06946C98AF2
:109B3000818003990498081803900498281885B226
:109B400005AA1499119801F077FA002805D11E98FA
:109B50000088401BB84200DB76E7022D0ED0159836
:109B6000102807D1049A03996846808A891A887058
:109B7000000AC8701E980580002030709E4800685A
:109B80000078032802D0002017B0F0BD0220FBE7C8
:109B9000F8B50546406B00271346002836D0491F0C
:109BA0008EB2698F954A914208D042185479127941
:109BB000240214430919891D8CB200E00024A11964
:109BC0002A8F083191421FD899785A7809020019D2
:109BD00011430170090A41701979DA7809021143B9
:109BE0008170090AC1700671310A41713246591DEE
:109BF000801D10F030FA6C87696B00200919B61DC2
:109C000089190870487002E0092700E08327384668
:109C1000F8BD30B50B88048F9C4212D9446BE01814
:109C20004478057824022C430BD04479057924022A
:109C30002C436404640CA41D1B190B8010600020CD
:109C400030BD822030BDF7B588B00025684605825A
:109C500005275DE00398417802780E0216434179AA
:109C6000027908021043000452D40A9801230680A6
:109C700005A802905B0200220097019530460999E1
:109C800001F04CFA04004AD16846018A0183039826
:109C90004179027909021143437802781C02144386
:109CA000B4421ED10A041CD44B0401215B0C89036D
:109CB00000950B4301970295C17880780A02024310
:109CC0002046099901F046F8040011D1039948791A
:109CD0000A79000210430122D20310430871000ADE
:109CE000487103AA06A90898FFF793FF0400CED095
:109CF0000399009501970295487809780002084376
:109D000069468B8A0022099901F024F8822C06D139
:109D100003AA04A90898FFF77CFF04009AD06846BC
:109D2000058209E003984179027909021143490447
:109D3000490C0171090A417103AA04A90898FFF7A7
:109D400068FF0028EED0822C02D020460BB0F0BD78
:109D50000020FBE730B50446406B002597B0002893
:109D60000DD00B2268460270228F0281606B039136
:109D7000019000216846FBF7D6FE6846057000207A
:109D8000C04365636087258717B030BDF8B50F46BF
:109D90000546696B0020069E144600290FD0012B52
:109DA0000DD1324639462846FFF74DFF002806D12F
:109DB000002C04D032463946284600F0D2FEF8BDC9
:109DC000F8B5069E4D1D3788ADB2079CAF4201D253
:109DD0000620F8BD3580172525706070000AA07038
:109DE000E270100A20710A461946601D10F033F91E
:109DF0000020F8BD012800008C070020FFFF0000B4
:109E000000220280C262831D0263C3614263531E4B
:109E10004387028720300170704710B50022D2437B
:109E20000280042007F0CBFC10BD30B597B00D4682
:109E30000446FFF78FFF208E002809D001206946D5
:109E40000870E06A0190002102956846FBF76BFEFE
:109E50000020E062206397E70146098800200A0796
:109E600000D501200A06120F01D002221043CA05B4
:109E700001D5042210438A0501D51022104349055B
:109E800001D5202108437047FFB5A7B00700309DDA
:109E9000339C29981E46229016D0007841060FD494
:109EA0008106890E1E2909D021884A05520E0BD140
:109EB0003288172A08D3FB4A914205D0C10906D03F
:109EC0008006800E122802D004202BB0F0BDF64987
:109ED00028980872002018AA039010726A4610741D
:109EE00004AA0A60319A4A6020AA90809081229840
:109EF00000781C908106681C0190781F1D9029989D
:109F0000890EC21C2492224620321B92083A401C21
:109F100002920B0010F044FB1FFEFE11FE1FFE8E8E
:109F2000FEFDFEFCFEFBFEFAFEFDFEF9FEFEFEF867
:109F3000FEF7FEFEFEFEFEF6FE00032F76D102E0E7
:109F400018A9087236E303202870019917220A70B5
:109F500000224A70ECE2052FF0D141780278080225
:109F60001043208320A98880249A5178127809020E
:109F70001143618300287DD088427BD80020207265
:109F8000E080401E6084029801F053F8052028709C
:109F9000A81C0190022000901BAA2899029801F0A9
:109FA0004BF8002867D118A8807C012803D0022034
:109FB0006870102002E001206870022024900022C6
:109FC00025A91CA805F099FB00282BD120A8007D0D
:109FD0002499814226D132880099801C511A8142ED
:109FE00020DB10A8C18D01980170090A4170019908
:109FF0001CA8891C01910099019A891C009125A92E
:10A0000005F07BFB20A8007D01991BAA091801918E
:10A010000099081880B200902899029801F00CF875
:10A020000028CCD00098022825D081E273E018A93E
:10A0300008727EE2072F6ED341780278090211433D
:10A04000218320AA9180249B5A781B7812021A43FC
:10A05000628300290ED091420CD8012121724179EE
:10A06000027908021043E08000202073E06900F0CC
:10A0700069FD01E098E0A9E000280ED1E169012026
:10A0800088710521E269C9029180E1698872E169FC
:10A0900086480881E16900208873F81F608422984F
:10A0A000C01D6062029800F0C4FF07202870681C81
:10A0B000009001200190002010A9C8852FE0019890
:10A0C000012814D0E0698079012830D000981E382A
:10A0D000417F007F0902014300980170090A417025
:10A0E0000098801C00900198801C80B2019010A8FC
:10A0F000C18D00980170090A41700098801C009081
:10A10000019809E025E2A9E135E1D9E01FE297E0F5
:10A1100075E034E02FE2ABE0801C80B201901BAA16
:10A120002899029800F088FF002803D007E010A8C3
:10A13000818DD1E731880198081A0428BFDA019887
:10A14000012843D0E0698079012804D010A8818DCE
:10A150005448814206D110A8818D00980170090AE7
:10A16000417009E000981E38417F027F0802009983
:10A1700010430870000A48700198801CD8E1072F2E
:10A1800001D0152F74D14178027808021043208342
:10A1900020A98880249A517812780902114361839A
:10A1A000002801D0884201D9012040E70120207217
:10A1B0000020E0802073052F0AD01D982299E269C3
:10A1C000C0B2491D05F073FA002801D00A202EE71D
:10A1D0000020C04360841AA8019023A92298029607
:10A1E00003950091007800238206920E204628995C
:10A1F000FFF7EAFB0390208B20A9888099E1032FC9
:10A20000C0D1402220A98A814178027808021043F7
:10A21000208320A988801EAB289A0293009231885F
:10A220000022491E8BB21B99097800F077FF18A90C
:10A230000872002831D10B20287010A8008F3DE053
:10A24000052F9FD1802220A98A81417802780802B7
:10A2500010432083249984464A78097812020A43DD
:10A26000628420A988801248824202D30720DEE659
:10A27000ADE03F208002024362841FAB2899029325
:10A2800000913088401E83B21B980178604600F030
:10A2900045FF18A9087200280CD08328AED10220EF
:10A2A000DAE00000FFFF00008C070020012800001A
:10A2B000010200000D20287010A8808F401C37E19B
:10A2C0001C990C22C9095143C91CB94204D91C98D4
:10A2D00040067CD500202BE1427803781002184319
:10A2E00020AA9080844622980078400609D505204F
:10A2F0006A46107422980078C00905D000201074B6
:10A300003CE106206A4610742498289A1F90009019
:10A310000023781A029383B21E9001921B980022A8
:10A320000178604600F016FD18A9087200226946FF
:10A330000A742299097849060DD52088C00506D5EA
:10A3400020A9208B8988884201D1002060620020EA
:10A3500018A90872ECE0832801D102200390FF21A4
:10A36000013120A88181808820831E9860841F98F5
:10A3700060621320DAE0052F29D3417802780802C1
:10A38000104320A98880218F002902D0F94A9142E8
:10A3900006D10A216A4611740121C943218702E0CE
:10A3A00007216A46117422990022491D289B0292B6
:10A3B000009101221D99D203019311438BB224997C
:10A3C0004A78097812020A431B99097800E0EBE009
:10A3D00000F0C0FC18A90872002269460A74012224
:10A3E000520220A98A81832808D0002815D0218F05
:10A3F000E04881427BD1002020879AE03946204600
:10A40000229AFFF7C5FB18A90872002801D08328FB
:10A4100023D120A88088208341E739462046229A0C
:10A42000FFF7B6FB18A90872002816D1618F606B80
:10A43000009643180195D87899780002084384461D
:10A4400058791A790102114358781A78000210439A
:10A4500062469B1DFFF7B4FC03906AE02298022F2E
:10A460004078019072D1002801D001286ED10820D7
:10A47000694608740198087521A800901B9800226D
:10A4800001782046019BFFF781FC69460022487550
:10A490008A75002809D10198012811D0002804D11B
:10A4A000B448218F401C81420AD0208F002807D059
:10A4B0000020694608740120800220A988810EE0EE
:10A4C00004A83199FBF72FFB03900020694608741C
:10A4D0000120800220A988810398022808D0A6487C
:10A4E00000688079002806D018A908722AE061E087
:10A4F000019820831DE00398002803D0812018A92B
:10A5000008723DE021A800901B98012201782046A6
:10A51000019BFFF73BFC18A9087220463299FFF710
:10A5200019FC18A9087A002803D1192028700120E5
:10A5300030806846007C002804D004A83199FBF7DD
:10A54000F2FA03900398002830D019E016E00620B4
:10A55000F6E42078000711D5012F0FD109216846B4
:10A560000174A18881820420329907F028F908211A
:10A5700020A88181AEE61C98400615D504200390E2
:10A5800020A9208889890843208020A988898005FE
:10A5900008D5218F7748814204D12998E062278627
:10A5A00003200390039890E40420C9E418A8007ADB
:10A5B00000280ED00120287022980078687020A80A
:10A5C0008088A870000AE87018A8007A2871052011
:10A5D000308020A92088898988432080E2E7FFB560
:10A5E000A1B000201C9021982C9C0178012088406B
:10A5F0006249604A084010A988862188521C91420D
:10A6000003D0002804D0080702D5012025B0F0BDF2
:10A61000249E00203070239910AA0988118518AA59
:10A6200010735549229A0A726A460546107404A8A6
:10A6300008602A9848602198249E0178701C1E901A
:10A64000204620300390012930D0022909D0032967
:10A6500075D13078800980011D3030702198808854
:10A66000A08021980078022804D1307880098001E8
:10A670001B3030701FAAF11C05206B4607C310A8C1
:10A68000008D0022C01E83B2039801782198808833
:10A6900000F044FD0028DBD1219881881E980170CC
:10A6A000090A417010A9888FC01CCDE0219841791A
:10A6B00018A8017321980079012802D00228C7D177
:10A6C00044E120887F2212011040219F10AA908629
:10A6D00002060837120F1BD00006800F05D03888FD
:10A6E000228B904201D0052597E1002910D1B8783E
:10A6F000C0070DD0B868002205216B4607C3039838
:10A70000FB880178BA88388800F024FB002875D1CE
:10A7100010A8808E80284DD006DC102810D020286C
:10A720000ED0402894D12BE0FF38013868D0FF3894
:10A7300001387DD0FF38FF38022889D1D8E00FE1F9
:10A74000C00601D5082000E010201C9004206946B6
:10A750000874002088821AA81BA91DAA03960092DB
:10A76000019102903B88052120461C9AFFF72CF9A5
:10A77000A2E00000FEFF00008C07002009F80000A6
:10A780000A201C9018A8007B002836D11FAA05209B
:10A790006B461E9907C310A8008D0022401E83B28D
:10A7A00003980178208B00F0B9FC014618A80173CA
:10A7B0000B2018E00C201C9018A8007B0028E4D186
:10A7C0001FAA05206B461E9907C310A8008D628C36
:10A7D000401E83B203980178208B00F09FFC014655
:10A7E00018A801730D20307010A8818F491C0185B5
:10A7F000042168460174218B8182D2E061E0FFE789
:10A800003988208B81425CD112211C9118A9097BC7
:10A8100000291AD1616A002912D0B978C90750D02D
:10A820000023B9680522029301920091FB8800E0A1
:10A830000CE00399BA88097800F08CFA18A908731B
:10A8400013203070012010A90885AAE03888218BD8
:10A85000884236D116211C9118A9097B002907D0FE
:10A86000606B002843D000206A461080D54F30E04E
:10A87000616B002915D0B878C00722D1608F01968E
:10A880000B181AA80090D8789978020258790A43D0
:10A890001D790102294358781D78000228439B1D29
:10A8A00008E0B978C9070CD01AA901960091BA88B6
:10A8B000F988BB68FFF784FA050072D0062D50D0E6
:10A8C0003FE005253DE00F4601AA69462046FFF717
:10A8D000A0F96946628F09888A4201D00028F2D027
:10A8E000618F626B0020511808704870678758E0CC
:10A8F00018201C9018A8007B002809D0208B002865
:10A900001AD03888208320462B99FFF723FA48E095
:10A910002046183000900398237E017801222046BB
:10A92000FFF734FA18A908730028ECD11920307009
:10A93000012010A90885E6E7052520462B99FFF799
:10A9400009FA6846007C032861D066E0208801216E
:10A950004902084010A98886FF38FF38022806D02F
:10A96000062510A92088898E8843208055E09549C6
:10A97000208F491E884200D0B5E616201C902198F1
:10A98000806800280AD06063219989892187002185
:10A99000C943618700210170417002E00020C0437B
:10A9A000208710A8808E7F21090102468A430ED09D
:10A9B0007823002204202B9906F071FE219810A91B
:10A9C0000078A0702088898E0843208002E02188CA
:10A9D000814321806846007C002805D07A48416880
:10A9E00004A8FBF7A0F8054618A8007B002814D09F
:10A9F0001C98707001203070208BB070000AF070CD
:10AA000018A8007B3071052110A8018505E06E486B
:10AA1000416804A8FBF787F8054620884005400EEA
:10AA200025D1208E002822D0239910AA09881185CB
:10AA300024992A9B2B9A01930091039402921AABBA
:10AA4000E26A2299FFF720FA054603280FD0012079
:10AA500069460874E06A05902B980690002104A8C6
:10AA6000FBF761F8002800D005460020208610A8DA
:10AA7000018D239801802846C8E500B597B00428C9
:10AA800007D102206A461070019100216846FBF749
:10AA90004AF817B000BD10B54B4C0378002221686E
:10AAA000012B02D0022B42D126E00B78002B01D0E3
:10AAB000042B03D10A712268032111702168838855
:10AAC0000A79D200921D8B5221680A79D20008328D
:10AAD0008918C2880A80216803890A79D2000A325B
:10AAE0008B52428920680179C9000C314252216899
:10AAF0000879401C08711EE00A7482888A802168E7
:10AB0000C288CA80226801891181226841895181E5
:10AB1000C1682068C1606168FBF705F8014602283A
:10AB200007D02068007C002802D1002903D08120B2
:10AB300010BD832010BD002010BD406B002800D048
:10AB4000012070478178012909D100880521C902B7
:10AB5000884202D0491C884201D10020704706205B
:10AB60007047F7B586B00024684615460F468481C5
:10AB700005261AE0049841780278090211432980D9
:10AB8000811D019602940091417902790B021343D1
:10AB9000C178827809020A434178007809020843A3
:10ABA000394600F0D7F8002806D104AA03A9069870
:10ABB000FFF72FF80028DDD0822800D1002009B04F
:10ABC000F0BD0000FFFF00008C07002010B58B785F
:10ABD000002B11D082789A4207D10B88002B0BD022
:10ABE00003E08B79091D002B08D08B789A42F8D1AD
:10ABF00003880C88A342F4D1002010BD812010BD31
:10AC0000052826D0002A02D0012A0DD102E00988A9
:10AC1000090501E009888904890F07D0012918D0A6
:10AC2000022909D003290ED081207047002A01D0C3
:10AC3000032070470220704703280AD0042808D058
:10AC4000002804D007E0042803D0022803D0052000
:10AC50007047002070470F20704770B51388054675
:10AC600014460B8018061DD5FE481022807AA84293
:10AC700003D813430B80002070BDA0689343007875
:10AC8000E840C007C00E03430B802078A1788007FE
:10AC9000800D0843F4490FF047FAA068694308188B
:10ACA000401C70BD906870BD37B569468B881380B5
:10ACB00019061BD5EB4C0125A47A9168844209D86A
:10ACC000FE280FD1D80602D5A5406D1E00E0002554
:10ACD0000D7007E085400C78DB06DB0FAC4383404A
:10ACE0001C430C7010881021884310803EBDF8B5BD
:10ACF0000746C81C80080E468000B04201D086205E
:10AD0000F8BD082A01D90E20F8BDD64D00202E60CE
:10AD1000AF802881AA723446E88016E0E988491C91
:10AD2000E980810610D48007A178800D0843CE49C0
:10AD30000FF0FAF9206800F0C8FA2989401880B2AB
:10AD40002881381A8019A0600C3420884107E5D486
:10AD50000020F8BDFFB589B09F041646139DBF0CB7
:10AD60000193099800F0A3FA04000AD020780006A5
:10AD700009D5BC48817A0A98814204D887200DB051
:10AD8000F0BD0120FBE7224669460A98FFF765FF00
:10AD90000690002069460872052D14D00122214634
:10ADA0002846FFF72DFF0028E9D1207840060AD574
:10ADB000022168460172099981810188C181068258
:10ADC0004782129805900198000404D500273E465A
:10ADD0000125079709E02078A1788007800D0843B6
:10ADE000A14907900FF0A0F90D46019840040AD53B
:10ADF0000798A84207D12088E1788005800F0002DB
:10AE00000843B04201D3AE4201D90720B7E7B819D1
:10AE100080B20190A84201D90D20B0E76846007ABF
:10AE2000002804D002A8FAF77AFE0028A7D10798D4
:10AE3000A8420BD120880321090288430199890582
:10AE4000890F0902084320800198E07014980028B7
:10AE500000D007801298002815D006983A4680192D
:10AE600012990FF0F8F8224669460A98FFF7F5FEA6
:10AE7000694608881021884369460880224600995F
:10AE80000A98FFF711FF002079E7FFB5754D0C22F6
:10AE9000E8882968504383B00C180D9F72490598C3
:10AEA0000FF042F90091049800F00FFA29682A89FE
:10AEB0008E46611A0C310918944651188AB2A98835
:10AEC000914202D8842007B0F0BD6A46168A320645
:10AED00003D5B20601D58520F5E7EA88521C92B267
:10AEE000EA800E9B002B00D01A80B20601D5A76025
:10AEF00006E0604480B22881091A70460818A060F4
:10AF00002246FE200499FFF7CFFE0598A070009816
:10AF1000E07020880599800889058000890F084322
:10AF200003210902884300998905890F0902084312
:10AF300004210843208003988078A071039800883A
:10AF4000A08000202073310601D5AC7A00E00124F6
:10AF5000B10600D5002700260EE005210020019152
:10AF600002900097E88831460C9B069AFFF7F2FEA4
:10AF70000028A8D1761CF6B2A642EED30020A2E7A4
:10AF8000F1B5009800F093F9060002D00025009C6E
:10AF900014E00120F8BD204600F089F9074600784A
:10AFA00031498007820DB87810430FF0BDF838683A
:10AFB00000F08BF94019641C85B2A4B22948C188FD
:10AFC000601E8142E7DC00992648491EC180018944
:10AFD000491B018100203070F8BD002804D0401EBC
:10AFE00010809170002070470120704710B5044612
:10AFF00001881C48C288914201D3822010BD00689C
:10B000000C22514342189079A072908820811088B8
:10B01000D1788005800F00020843A081A078211D0F
:10B02000FFF71BFE20612088401C2080E08000206C
:10B0300010BD012101827047F7B50546002084B09C
:10B04000C0431080686817468178684681706868D8
:10B0500001886846018000218171288A2C88A042DD
:10B0600005D303E0980700200102000004462C826B
:10B0700035E0288A401C2882301D6968FFF7A6FD4C
:10B0800000282AD139889948814201D1601E388030
:10B090006888A04228D33088F1788005800F0002AC
:10B0A000084302906946301DFFF790FD002814D137
:10B0B00069898E4881421BD0002231460598FFF7EE
:10B0C0009FFD002809D16A890298824205D1E9686A
:10B0D000B0680EF093FF00280AD0641CA4B220468A
:10B0E00000F0E5F80600C4D1641E2C828220EAE656
:10B0F0007C80B079B871B088B8803078B17880073A
:10B10000800D084378810298B8813946287A324602
:10B110000831FFF7A2FD38610020D4E6FFB585B005
:10B120001C460F46059800F0C2F8050009D02878A3
:10B13000000608D56E48807AB84204D8872009B046
:10B14000F0BD0120FBE707982A468605B60D694643
:10B150003846FFF782FD07460E98052816D00022D4
:10B160002946FFF74DFD0028E9D1287840060DD586
:10B17000012168460171059901810188418186811B
:10B18000C48101A8FAF7CBFC0028D8D12888AA7876
:10B190008107890D11438005800FEA780002104372
:10B1A000079A964207D0534A914204D3611E8142C6
:10B1B00001DD0B20C3E7864201D90720BFE7801BD2
:10B1C00082B2A24200D922461098002800D0028004
:10B1D0000F98002802D0B9190EF03DFF0020AEE70D
:10B1E000F8B51D4617460E4600F061F8040008D079
:10B1F0002078000607D53E48807AB04203D88720E1
:10B20000F8BD0120F8BD224639463046FFF725FD3E
:10B21000002D0BD02078A1788007800D0843354998
:10B22000884201D2012000E0002028700020F8BDF3
:10B23000F8B51E4617460D4600F039F8040008D050
:10B240002078000607D52A48807AA84203D88720AC
:10B25000F8BD0120F8BD224639462846FFF724FDF7
:10B26000FF2E14D02588A178A807800D0843214916
:10B270000EF05AFF002E03D1FF31FF31033189B2A6
:10B28000A170A80880008905890F0843208000204C
:10B29000F8BD10B50C4600F00AF8002805D08188EA
:10B2A00021808079A070002010BD012010BD1049C0
:10B2B000CA88824207D3002805D00C22096850436F
:10B2C0000C38081870470020704703B508466946D7
:10B2D00009888A0607D4090604D50549897A4143B5
:10B2E000491C88B20CBD00200CBD0000FFFF00000F
:10B2F000980700200102000010B506F095FB05F04C
:10B300000DFFF7F721FE0DF099FC06F0A3FA06F009
:10B3100023FB10BD00B51E2827D00FDC0C2820D041
:10B3200008DC03000FF03CF90913211521211B1B38
:10B3300017192100122818D1072000BD302814DD6C
:10B340003A3803000FF02CF9030F11091100002007
:10B3500000BD1C4800BD042000BD0D2000BD0F2015
:10B3600000BD082000BD112000BD032000BD10B5A8
:10B370000C4601F08EFC00281BD0204600F09BFA02
:10B38000002813D022780E2A0AD00F2A08D0022AC9
:10B3900006D0032A04D0102A06D00EF0E6FF0AE0F9
:10B3A000A078FFF7B7FF10BD112010BD0EF0DDFF34
:10B3B00001E00EF0DAFF002010BD10B500F07BFABE
:10B3C00010BD00000230000030B5034600200246E8
:10B3D0000DE09C5C2546303D0A2D02D30020C04381
:10B3E00030BD0A25684330382018521CD2B28A4238
:10B3F000EFD330BD70B50D46144608E00A210EF0BB
:10B4000093FE2A193031203A641ED177E4B2002C21
:10B41000F4D170BD10B5002310E0040A000204430B
:10B42000A0B2CC5C44402006000F60400407240C0E
:10B4300044402006C00C60405B1C9BB29342ECD39E
:10B4400010BD000010B509F0C7F8042803D009F0BA
:10B45000C3F8052803D108F03EF800280BD109F005
:10B46000F1F9032803D009F0F3F9032805D107F017
:10B470008DF9002801D0012010BD002010BD70B54D
:10B480000C460546062102F0A7FA6060002801D0AC
:10B49000002007E00721284602F09EFA606000289D
:10B4A00003D001202070002070BD022070BDF0B5D7
:10B4B00085B00C46064600276946FFF7E0FF0028E6
:10B4C0006CD16846007800280BD007F0D8F8B0425D
:10B4D00064D00022214630460BF0F5F9002875D1E2
:10B4E0002DE007F0F8FDB04258D00022214630464A
:10B4F0000AF02CFE002869D1019D9020405D28357E
:10B50000002804D1687E002801D0012000E000203E
:10B51000029028462030417B002914D0817B890786
:10B5200011D50021617001222270A170A680C27B1A
:10B53000A2712A8E22816A8E6281417346E0019D4A
:10B540002835687EE4E7304602F01EFC03900028B0
:10B5500004D10EF00AFF01E07F1CFFB20021039826
:10B5600002F0A9F80028F7D1002F07D060700D2055
:10B570002070A680E7800120A07027E0304602F00E
:10B58000EEFB070001D10EF0F0FE0298002805D076
:10B590000021384601F042FC002802D0002005B00E
:10B5A000F0BD68460078002807D101988030406AD5
:10B5B0004188B14201D100210170002060700A2150
:10B5C0002170A070A680A97EA17168760120E6E7AF
:10B5D00010B5017840680029008806D0072102F0E4
:10B5E00006FA002800D00C2010BD0621F7E71CB594
:10B5F00004466946FFF743FF002801D00EF0B5FE70
:10B60000204606F072FF002801D10EF0AEFE68461B
:10B61000FFF7DEFF002801D00EF0A7FE1CBD1CB511
:10B620006946FFF72CFF002801D00EF09EFE684609
:10B6300001F038FCF84800218068803041821CBD50
:10B64000FEB504460E46062002F06FF905460720B7
:10B6500002F06BF92818C7B20025BE1915E0208842
:10B66000401C80B22080B04201D30020208080B2F4
:10B67000B84203D3B04201D20020FEBD6946FFF7B5
:10B68000FEFE0028F9D06D1CEDB2AE42E7D80020D6
:10B69000C04320801220FEBD0EB50020C043694685
:10B6A00008800FE0684601A90088FFF7E8FE00283F
:10B6B00001D00EF05AFE01A8FFF78AFF002801D042
:10B6C0000EF053FE00216846FFF7BAFF0028E9D0CC
:10B6D0000EBD7CB5D1A103C9D24D002401910090CB
:10B6E000AC7001F0D8FB2946EC7004204039088783
:10B6F00010204887C81DCC4AF93042800471C280AE
:10B70000E03844740C7084730475C03004771D30C5
:10B710000522694604460EF09EFC28462146BC30B0
:10B720000AF0BAFD7CBDF8B5BB4C0D4660602170D7
:10B7300006F0B2FEFFF7B0FFFFF7CBFF207808F06E
:10B740004DFDB8498431084681380F46064607F05A
:10B75000A0FD60680AF069FD0CF090F8284609F039
:10B76000F7FB3946304606F0BAFF60680BF031F956
:10B7700001F091FBAB480021C170F8BDFEB504009B
:10B7800001D10EF0F2FDA74D203D687C002809D0C4
:10B790000020607010212170A97CA170E97CE1700B
:10B7A00068747AE09F4E403E3078002809D02C2201
:10B7B000B11C20460EF04FFC0E202070002030708F
:10B7C0006BE0A87B00280AD00120E070E87BA07025
:10B7D000287C60700F2020700020A8735DE09148E5
:10B7E0000221C6300290FFF72BFF002801D00EF097
:10B7F000BCFD8C4FC037F8880190062002F095F808
:10B800000646072002F091F83018C6B2701CC0B28C
:10B810000090F888B04214D10021204607F010FCB7
:10B8200000283AD1287D002839D0002666701320E0
:10B8300020701C21A01C0EF06BFC0220A0702E7545
:10B840002BE00099884223D10021204606F0F0FE2B
:10B85000002824D0207813281FD1A0783C281CD1A0
:10B86000A088072102F0B8F8050001D10EF07DFD97
:10B87000288806F03AFE002801D10EF076FDA08857
:10B88000072102F0B4F8002807D00EF06EFD04E0A6
:10B890002146FFF70CFE002801D00120FEBD022149
:10B8A0000298FFF7CDFE002803D1F9880198814264
:10B8B000AFD10020FEBD61E710B508F008FC0028FC
:10B8C00001D00EF052FD0AF0AEFC002801D00EF0BF
:10B8D0004CFD07F0A2FC09F025FB002801D00EF07A
:10B8E00044FD0BF074F8002801D00EF03EFD06F088
:10B8F000CFFE002801D00EF038FD0BF0B9FF002874
:10B9000001D00EF032FDFFF7C7FEFFF7E2FE06F0B2
:10B91000A7FD01F0C0FA43480021C1704038017111
:10B92000012141710222C270017010BD10B53D4C61
:10B93000403C2078002804D00A210E2001F078FA3B
:10B9400010BDFFF77FFD002801D00C2002E001F0C0
:10B95000A2FA00202071012060710A21E17020709C
:10B9600010BD70B52F4C0646403C2078002804D00E
:10B9700039210E2001F05CFA70BDFFF763FD00284D
:10B9800001D00C2010E0274DE87808280BD20001E8
:10B99000001910223146443001F054FAE878401C76
:10B9A000E870002000E0072020710120607139213B
:10B9B000E170207070BD70B51A4C0646403C20788E
:10B9C000002804D00B210E2001F032FA70BD30782F
:10B9D000002803D0012801D0122015E0114D803538
:10B9E0002879082822D2FFF72DFD002801D00C204D
:10B9F0000AE00C4833782979721C883006F0BCF8CC
:10BA00002879401C287100202071012060710B21D1
:10BA1000E170207070BD000040000020FFFFFFFFBC
:10BA20001F000000E4070020FFFF00000720EBE7F5
:10BA300010B5FC4C2078002804D038210E2001F0ED
:10BA4000F7F910BDFFF7FEFC002801D00C2003E041
:10BA5000F44900204031C870207101206071382104
:10BA6000E170207010BD10B5EE480178002904D0B7
:10BA70000F210E2001F0DCF910BD002101710E2113
:10BA800081700F21C170FF2181710021C9430181A3
:10BA9000E54949680A7882728A8882814988C18129
:10BAA00001214171017010BD10B5DE490A78002AEC
:10BAB00004D03B210E2001F0BBF910BDDB4A008809
:10BAC00050800120107100220A7148713B22CA7017
:10BAD000087010BD10B5D34C2078002804D02B215D
:10BAE0000E2001F0A5F910BD0821A01D05F0B2FB44
:10BAF00000202071012060712B21E170207010BDA9
:10BB000070B5C84C2178002904D031210E2001F0F5
:10BB10008FF97FE700214156042910D000290ED06B
:10BB2000081D0CD0001D0AD0001D08D0001D06D035
:10BB3000001D04D00A3002D01220207104E000253C
:10BB4000084606F064F825713120E070012060712C
:10BB500020705FE730B5B34D044628788DB00028DB
:10BB600005D02A210E2001F063F90DB030BD10225E
:10BB70002146684601F066F91022A11804A801F0D8
:10BB800061F968460DF0E5F810222C46A81D08A9B9
:10BB900001F058F9002020710E20A0702A20E070DA
:10BBA000012060712070E0E7F0B59E4C85B02078F0
:10BBB000002804D03A210E2001F03AF9EFE40020E9
:10BBC000A0719A4869464088888002A9FFF757FC0F
:10BBD000002805D0002101A8FFF732FD002853D12D
:10BBE000684681880180684602A90088FFF747FC03
:10BBF000002801D00EF0B9FB6846008802F0C4F8B6
:10BC0000050001D10EF0B1FB039E2846283601F055
:10BC100046FD0121484005466846767E008802F0D0
:10BC20009EF8070001D10EF0A0FB0021384601F07C
:10BC3000F5F8024630431CD0A179684649000088D7
:10BC4000091908817748A3791830195C520049080E
:10BC5000490031431954FD26A37931401143195449
:10BC6000FB231940A279AB0019431154A079401C61
:10BC7000A07100216846FFF7E3FC002804D1684664
:10BC8000018880888142AED100202071012060713E
:10BC90003A21E170207082E470B5624C054620784C
:10BCA000002804D034210E2001F0C2F8B2E608F0DA
:10BCB00093FC052804D0284608F07DFA002000E017
:10BCC0000C202071012060713421E1702070A1E608
:10BCD00010B5544C2078002804D00E21084601F0FD
:10BCE000A7F810BD504906220C31A01D0EF0B3F983
:10BCF00000202071012060710E21E170207010BDC4
:10BD000070B5484C06462078251D002804D0322105
:10BD10000E2001F08DF87DE63146002006F0B2FDE0
:10BD2000287000280DD100213246084607F09EFBFE
:10BD30002870002805D13C48062231460C300EF010
:10BD40008AF9012060713221E170207062E670B5DD
:10BD5000344C05462078002804D030210E2001F014
:10BD600067F857E608F0A3FA002803D109F07BFB37
:10BD700000280DD0287809F031F9287807F0D3FB96
:10BD800000202071012060713021E170207041E6B7
:10BD90000C20F6E7F8B5234C06462078251D002830
:10BDA00004D017210E2001F043F8F8BD31460120E0
:10BDB00006F068FD0127287000280FD132460121C6
:10BDC00007F054FB2870002808D116480622314697
:10BDD0003C300EF040F913484030877067711720EF
:10BDE000E0702770F8BD10B50E480178002904D026
:10BDF00030210E2001F01CF810BD1221017101212B
:10BE000041713E22C270017010BDFEB5054C054661
:10BE10002034A07B00280BD028210F2001F008F847
:10BE2000FEBD0000A407002040000020A408002060
:10BE3000282020740121A173A8781A2824D00EDCB0
:10BE400003000EF0ADFB162F2F2F2F2F212F2F2F9A
:10BE50002F2F2F2F2F2F2F2F2F2F2121212F2A2828
:10BE600020D00ADC1E3803000EF09AFB0C1C1C1CB0
:10BE70001C1C1C1C1C1C1C1C0E1C3A3803000EF045
:10BE80008FFB0411031103112888F74A904209D847
:10BE90001F20E07328886946FFF7F1FA002803D0D5
:10BEA000022014E0122012E068460078019F00286A
:10BEB0000FD0C637019E00280DD0C736684600F067
:10BEC000DDFF002802D03878002806D00C20E0736F
:10BED000A6E79C37EEE79D36F0E701203870A8789A
:10BEE00030700020E073684600F0DCFF98E7F0B5A2
:10BEF000DE4C0746207885B0002804D025210E208E
:10BF000000F096FF5AE6388802A9FFF7B8FAD74E34
:10BF10000021083600280CD00220207131603171D8
:10BF2000E1800E20A0702520E0700120607120705B
:10BF300044E6039D28460830483501900020A87546
:10BF40000522304601990EF086F8A87D0028F5D12B
:10BF50003888E080E5E7FEB5C44C06462034A07B77
:10BF6000002804D010210F2000F062FF58E71F20A6
:10BF7000E073102020740127A77330886946FFF70B
:10BF80007EFA002810D1684600F078FF00280BD018
:10BF90006846019D007828350028019806D0CA30EF
:10BFA0000178002909D104E0022007E08030406ACE
:10BFB000F6E72035697B002902D03A20E0732FE7AD
:10BFC000A97B89070DD106210170684600780028F9
:10BFD00004D1019831888030406A4180684600F081
:10BFE00061FF0020E0736F731AE7F8B59F4D0646B6
:10BFF0002878002804D01D210E2000F019FFF8BD7C
:10C000001F202871012068711D21E970287008F037
:10C01000E3FA0C27042855D0052853D0B079122410
:10C02000012801D000281DD13078002801D0012836
:10C0300018D1F079002801D0012813D170888C49DB
:10C04000021F30248A420DD2B288121F8A4209D2BE
:10C050002887B0886887B0790024012804D0002898
:10C060000CD014E02C71F8BD804840308078002856
:10C0700028D07E4A3C320121084602E07D4A002158
:10C08000012007F0F3F9040001D00EF06EF9F07909
:10C09000012801D0002802D107F004FA0446002C40
:10C0A00001D01F2011E03078012802D0002803D0F1
:10C0B0000AE00021022001E00021012007F002FA3D
:10C0C000002801D02F71F8BD00202871F8BD70B58F
:10C0D000664C2178002904D01E210E2000F0A8FE15
:10C0E00098E41F212171012161711E22E2702170EB
:10C0F00002781221012A01D0002A04D140780028B8
:10C1000003D0012801D0217184E400260C25012AE6
:10C1100009D008F061FA052803D007F085FF002850
:10C1200006D0257176E4618F208F08F0CDF8F6E710
:10C1300026716FE4F0B55049054603C989B04B4EEE
:10C14000059120360490B07B002805D021210F20D6
:10C1500000F06EFE09B0F0BD1F20F0732120307496
:10C160000120B0732A88424B111F3020994243D2DC
:10C1700069880C1F9C42FAD291423DD8EB893F4915
:10C180009A1F8A42F3D22A8A941F8C42EFD293429A
:10C19000F3D8698AFF23F4339942EED8A98A374C41
:10C1A0000B460A3B241FA342E1D2D208914223D975
:10C1B000E98A2A8B9142E0D829791220002902D0FD
:10C1C000012919D102E069790029F9D1297B0029D7
:10C1D00001D00129F5D108F0FFF905280BD008F0AE
:10C1E000FBF9042807D0307D002804D106F073FF46
:10C1F0002349884201D00C20BCE0062106A801F0AA
:10C20000BFFB040040D003210BF091FF20460D300E
:10C2100002902788042105F01DF8394602980CF099
:10C220001CF818A00068274607901137032107A8BB
:10C2300004F099FF002007A90A5C3A54401CC0B2E0
:10C240000328F9D3288A6080688AA080A88AE080C1
:10C250002046002720308773C7736879002815D0DF
:10C26000012817D114E00000FF0E0000A4070020F1
:10C27000FD3F00004C0000201CBA00007B0C0000B9
:10C28000FFFF000011223300092073E0677601E010
:10C290000120607620460622A91D1A300DF0DBFE33
:10C2A0002046052204A90830F4F770FF012120463A
:10C2B000A0300390017369460F72012102A804F0B7
:10C2C00052FF6946087A4107C206490F920F80065D
:10C2D0008918C00F081869460872401D2076092881
:10C2E00001D208302076002120460BF020FF208864
:10C2F0000322092106F0ECF8002801D10EF035F8F0
:10C30000287B002804D0012806D00EF02EF833E058
:10C310000021FA4A012007E0F948807800280DD072
:10C32000F74A0121121F084607F0A0F8002823D081
:10C33000208806F0DAF8002811D012E0208806F0F4
:10C34000D4F8002801D10EF010F82088062101F061
:10C350004EFB002800D14EE70EF007F84BE70EF039
:10C3600004F82088062101F042FB002801D00DF0DE
:10C37000FCFF1F20F073EDE62879012801D000288A
:10C3800003D107F08FF800280CD12146032007F0D5
:10C3900099F8002806D16A882988204607F04AFFC4
:10C3A000002805D0208806F0A0F8002804D005E079
:10C3B00003980770F773CDE60DF0D7FF20880621AC
:10C3C00001F015FB0028C6D00DF0CFFF13E738B5FC
:10C3D000CB4C403C2078002804D022210E2000F0D5
:10C3E00027FD38BD1F202071012565712220E070D6
:10C3F000257008F0F1F8052802D00C20207138BD16
:10C4000000202071684607F093FF0028F7D10098BC
:10C41000008806F06AF8002801D10DF0A6FF009808
:10C420000621008801F0E3FA002801D00DF09DFFFD
:10C43000B34820380575B1480C380078FCF7C4FEC5
:10C4400038BDF8B5AE4E0546203EB07B002804D07E
:10C4500023210F2000F0ECFCF8BD1F20F0732320F7
:10C4600030740120B0736A88A64B911F3020994226
:10C470004BD2A9888C1F9C4247D28A4245D8EA8871
:10C48000FF23F4339A4240D82A899E4C13460A3B34
:10C49000241FA34239D2C9088A4236D96989AA8998
:10C4A000914232D82888062101F096FA02270446E4
:10C4B000002809D000F0D3FC002805D08034606A41
:10C4C0000178002906D101E0F773F8BDA16B097866
:10C4D000002901D03A2018E005218171606A00210D
:10C4E0000181626AA8885081626AE8889081626AE4
:10C4F0002889D081606A028943899A4204D8827966
:10C50000082A01D89A4202D31220F073F8BD2A8873
:10C510004280606A0770F173F8BDFEB5784C05463D
:10C52000403C2078002804D024210E2000F080FC1C
:10C5300076E4012666712420E070267028460BF010
:10C54000ABFE002801D0002000E01220207100285E
:10C55000EED16B4F0522A03738463E7729461D3075
:10C560000DF079FD002038776946062001F0BEF90C
:10C57000002801D00DF0F9FE684601F094F900287A
:10C5800015D16846878868468088062101F024FA1C
:10C59000050001D10DF0E9FEA0352E73684601F0CB
:10C5A00082F9002803D168468088B842EBD1002088
:10C5B000207135E470B5524C0646203CA07B002823
:10C5C00004D026210F2000F033FC89E51F20E07302
:10C5D000262020740120A0733088062101F0FCF988
:10C5E000050009D000F03BFC002805D08035686AC2
:10C5F0000178002906D101E002200BE0A96B09783F
:10C60000002901D03A2005E007210170696A3088CD
:10C6100048800020E07363E510B5394C403C207839
:10C62000002804D006210E2000F002FC10BD0020DE
:10C6300020710E20A0700620E0700821A01D0DF0D2
:10C6400067FDA17901200143A1716071207010BDC7
:10C65000F8B52B4C0746203CA07B002804D02C21A9
:10C660000F2000F0E5FBF8BD1F20E0732C202074A4
:10C670000120A0733888062101F0AEF906000AD027
:10C6800000F0EDFB002806D035468035686A017859
:10C69000002906D101E002201FE0A96B09780029DA
:10C6A00001D03A2019E04036317F002917D0082206
:10C6B000B91C001D0DF0CFFC686A79898181686A18
:10C6C000394610220C310E300DF0C5FC696A03208A
:10C6D0000870696A388848800020E073F8BD0C2033
:10C6E000FBE770B5064E0446403E30780C25002826
:10C6F0000AD018210E2000F09BFBF1E44C00002032
:10C70000E40700207B0C000008F09CF803285AD0B6
:10C7100008F09EF8032856D06079002801D001283F
:10C720002DD1A079002801D0012828D1A07B002894
:10C7300005D0012803D0022801D003281FD1607B37
:10C7400000281CD0C0081AD16288012080038242D0
:10C7500002D82188814203D9207901280FD119E01C
:10C760002079002806D0012814D0022805D00328FB
:10C7700005D102E0202A0BD30CE0A0290AD22079AF
:10C78000042805D12088202802D36188884201D955
:10C79000122518E0FE48217981756079002802D0C1
:10C7A000012804D00FE0FB4A0021204608E0F848A9
:10C7B00020308078002806D0F54A01211C3220461E
:10C7C00005F0EAFF05460120357170711821F170FE
:10C7D000307085E410B5EE4C203C2178002904D05F
:10C7E0001A210E2000F024FB10BD01781F2902D968
:10C7F0001220207106E0002121710278411C1046B0
:10C8000006F066F8012060711A21E170207010BDF9
:10C8100010B5DF4C203C2178002904D020210E20C7
:10C8200000F006FB10BD01781F2902D912202071EB
:10C8300006E0002121710278411C104606F03AF80A
:10C84000012060712021E170207010BDF8B5D04C3E
:10C85000203C2178002904D01B210E2000F0E8FAAA
:10C86000F8BD012767710C2121710078002601288D
:10C8700004D0002852D01220207171E005F059FF39
:10C8800000286DD0C248807D002818D0012816D01D
:10C89000042814D007F0DCFF002861D107F0D2FF94
:10C8A000002803D007F0CEFF022859D1002008F05D
:10C8B00098FB002801D00DF058FD267150E007F0DC
:10C8C000C1FF00284CD107F0C3FF002848D105F074
:10C8D000D6FEB149884243D10721684601F050F89D
:10C8E0000500AE48856001D10DF03FFD03212846CB
:10C8F0000BF0C5FB284606F085F8288806220D2196
:10C9000005F0E6FD002801D10DF02FFD284608F0C6
:10C9100068FB0028D1D00DF028FDCEE707F092FF8C
:10C92000032803D007F094FF032819D107F08DFFE7
:10C930000546002008F081FA002811D12671002D4B
:10C940000ED0288805F0D1FD002801D10DF00DFD95
:10C950002888072101F04BF8002801D00DF005FDD3
:10C960001B20E0702770F8BD70B5894C0546203C4F
:10C970002078002804D02D210E2000F059FA24E65A
:10C980002888072101F028F8002824D00146C0316A
:10C990000E46897A002909D13421095C0F2901D07A
:10C9A000102903D1FC21095C00290BD00C20207137
:10C9B0000E20A0702D20E0702888E080012060719A
:10C9C000207002E61022A91CD8300DF044FB042090
:10C9D000B0720020EBE70220E9E770B56C4C054629
:10C9E000203C2078002804D02E210E2000F020FAD0
:10C9F000EBE52888072100F0EFFF00281AD0014658
:10CA0000C0318A7A002A05D12030007D0F280DD050
:10CA100010280BD00C2020710E20A0702E20E0706A
:10CA20002888E080012060712070CEE505208872A2
:10CA30000020F0E70220EEE77CB5554C0546203C8F
:10CA40002078002804D037210E2000F0F1F97CBDB9
:10CA500028886946FEF713FD002807D002202071C0
:10CA6000012060713721E17020707CBD01987F2228
:10CA7000014628300272427200228272A878203168
:10CA80008870E878C870287908712271E8E71CB5C9
:10CA90003F4C203C2178002904D013210E2000F0C7
:10CAA000C7F91CBD00886946FEF7E9FC002801D0E3
:10CAB000022005E001992220405C012802D00C20D0
:10CAC000207106E0302000222271405C207208882C
:10CAD000E080012060711321E1700E21A1702070AF
:10CAE0001CBDF8B52A4C0546203C2078002804D00F
:10CAF00035210E2000F09CF9F8BDA878002801D05F
:10CB0000012804D1A888FF21F531884201D91220DB
:10CB100020712888072100F05FFF0126002813D02C
:10CB200001460027C0310F70AA884A8080300677FE
:10CB3000AA78012A00D000220A70407F002801D084
:10CB400008F073FB277101E0022020716671352027
:10CB5000E0702670F8BDF8B50D4F0446203F3878D8
:10CB6000002804D03C210E2000F062F9F8BD208896
:10CB7000072100F031FF060038D0B58864886800CE
:10CB8000F2887188401C844222D30548414309E061
:10CB9000C40700204C000020FFFF000040000020E0
:10CBA000C4090000800050430DF0BEFA401EFF2172
:10CBB00080B2F531884200D90846844200D220462E
:10CBC000691C401C0DF0B0FA6D1C6843401E85B214
:10CBD000E820805D002800D13584FD800020387178
:10CBE000012078713C21F9703870F8BD0220F6E719
:10CBF00070B5B34C05462078002804D033210E20B0
:10CC000000F016F9E1E407F01DFE002801D00C2029
:10CC100018E02978002911D00A290FD014290DD045
:10CC20001E290BD0282909D0322907D04B2905D03D
:10CC3000642903D0FF2901D0122003E0284608F020
:10CC400062FA00202071012060713321E1702070B0
:10CC5000BBE470B59A4C05462078002804D03D21ED
:10CC60000E2000F0E5F8B0E407F0ECFD002803D159
:10CC700007F0EEFD002801D00C2003E0287805F035
:10CC800033FE00202071012060713D21E170207091
:10CC90009BE410B5017801240B000DF081FC3FBC32
:10CCA000BC21BCBCBC91BCBCBC2427BCBC424C5EFF
:10CCB000BCBC56BCBCBC2B94BC989CBC767ABCA0BB
:10CCC0007E828589628DBC5ABC524F72A4A8BC3743
:10CCD0002F33B86AACBC6E3F3B4566B0B448BD006C
:10CCE000FEF7EAFD98E0FEF721FE95E0801CFEF7D6
:10CCF00062FE91E0801CFFF74DF88DE0801CFEF78E
:10CD0000FFFE89E0801CFEF7FBFF85E0801CFFF73B
:10CD10001EF881E0801CFEF724FE7DE0FEF788FE11
:10CD20007AE0FEF7D5FF77E0FEF73EFF74E0801C67
:10CD3000FFF759F870E0FEF796FE6DE0FEF7CAFEC9
:10CD40006AE0801CFEF706FF66E0801CFFF79FFE8E
:10CD500062E0801CFFF759F85EE0801CFFF7FBF8EB
:10CD60005AE0801CFFF7C3F856E0801CFEF79CFEDB
:10CD700052E0801CFEF790FF4EE0801CFFF75CFE47
:10CD80004AE0801CFFF764FC46E0801CFFF72DF9A9
:10CD900042E0801CFFF79BF93EE0801CFFF7CAF9D8
:10CDA0003AE0FFF714FB37E0801CFFF74AFB33E063
:10CDB000801CFFF7B2FB2FE0801CFFF7FBFB2BE092
:10CDC000FFF72AFC28E0801CFFF78BFC24E0801C86
:10CDD000FFF700FD20E0801CFFF738FD1CE0801C01
:10CDE000FFF716FD18E0801CFFF7BEFD14E0801C65
:10CDF000FFF7F3FD10E0801CFFF773FE0CE0801CD2
:10CE0000FFF7A9FE08E0801CFFF723FF04E0801C69
:10CE1000FFF7EEFE00E00024204610BD10B50C46E2
:10CE200000F0ADFB002802D022680021117010BD77
:10CE3000234A2032537C002B03D19074D1740120FB
:10CE40005074704730B5134606E0CC18203CD51A14
:10CE5000E47F5B1E4455DBB2002BF6D130BD41218F
:10CE6000095C002908D18030017C002904D0007CB5
:10CE7000042801D0012070470020704701784068E5
:10CE8000002905D040304078002802D000207047AB
:10CE9000E5E7012070470A4900208031886740316A
:10CEA0000871704710B50178012908D140688030B9
:10CEB000417F002903D00021417708F0B6F910BD69
:10CEC000A407002070B40588E40B69184904E40342
:10CED000490C0C4301212D04C903EE0F8C43F603CA
:10CEE00034436604760C96420FD2921B92B21B33E7
:10CEF0009A4207D2E20BD203EB17DB035B189CB21A
:10CF00008A431443046070BC70470F23DC41520411
:10CF1000A21A1123DA41EB17DB035B189BB28A4399
:10CF20001343036070BC70470818C01D504345315F
:10CF30004018704770B51D460446A818049BC01DD4
:10CF40002A4658434532801886B2B14201D20DF0CC
:10CF50000CFA6068C10B0120C903C0038143616002
:10CF6000A168C90BC9038143A160E168C90BC9036A
:10CF700081430020E16020762082A0826082E082EE
:10CF80006076243EA5762680012070BD008870471B
:10CF9000F0B5044684B02430039001900E46E0685A
:10CFA000A168154642044F04520C7F0CBA4206D1C8
:10CFB00048400004C00F02D0002004B0F0BDBA42C7
:10CFC0001BD9A17ED01B401AC01F00B285422FDCA6
:10CFD0000198C91D38180918C91E716035810021D2
:10CFE000F1603182021D326005702A0A4270817040
:10CFF000C1700120207604B0F0BD2088A17EC01B46
:10D00000401AC01F00B202920090002810DB1B28BB
:10D0100001DA0DF0AAF90098854201DC294600E00A
:10D0200081B2681A0204120C06D00298824203D917
:10D030000020207604B0F0BDA37E0198DB1D3818D7
:10D040001B18DB1E73603181039BF3603282031D6A
:10D0500033600170090A41708270110AC1700120A9
:10D06000207604B0F0BDF8B504460246237E243293
:10D070008068002B0DD04004400C82185078157841
:10D0800003022B43D0789578000228431818884271
:10D0900001D20020F8BD2046083000278B4206D37D
:10D0A0001170090A51709770390AD1701FE0C91ABE
:10D0B0008EB2310A9670D170002E18D005460088C5
:10D0C0004004400CB04201D80DF04FF9E00B710460
:10D0D000C003490C0843298801220904C917D20357
:10D0E000C903891889B29043014329600AE0517845
:10D0F0001278A37E09021143DB1D591889B22288D8
:10D10000FFF7E0FE27760120F8BDF0B5476803463B
:10D110007E0485682433760CBC46F4186F047F0CBB
:10D12000A646BE420AD166466E403504ED0F012682
:10D13000754003D0002181820846F0BD65782778CC
:10D14000068A2D023D43AE4207D3751BE678A778C9
:10D1500034023C43641BDB1E05E0837EAC1B9D193F
:10D160007346EB181B1D0B601188A14200D9148077
:10D17000118881820120F0BDF8B50446A1882430D1
:10D180004904490C0D18A08A002843D0218A0818A8
:10D1900080B2208269782A7809021143EA78AB7854
:10D1A00012021A438918814201D20DF0DEF8687824
:10D1B000297800020843E978AA780D021543228AEB
:10D1C00041190027914223D1002D18D0A088261D97
:10D1D0004004400CA84201D80DF0C7F8E00B6904E8
:10D1E000C003490C0843318801220904C917D2033E
:10D1F000C903891889B290430143316007E0A37ED7
:10D200002288DB1D181881B2201DFFF75BFE2782E4
:10D21000A7820120F8BDF8B58C46C36801460446D4
:10D220005E0424314068760C75184104490C0127CE
:10D230008E4206D143401804C00F784001D0002030
:10D24000F8BD002A01D0281D10606046002803D0D8
:10D25000A27E291D0CF0FFFEE878A9780602204680
:10D260000E430C30002E18D0044600884004400CB9
:10D27000B04201D80DF079F8E80B7104C003490CF5
:10D280000843218801220904C917D203C903891858
:10D2900089B29043014321600AE069782A78A37E2D
:10D2A00009021143DB1D591889B22288FFF70AFED3
:10D2B0000120F8BD416880684A044304520C5B0CAD
:10D2C0009A4207D141400804C00F0121484001D0D3
:10D2D0000120704700207047C16840684A04430439
:10D2E000520C5B0C9A4207D141400804C00F012147
:10D2F000484001D00120704700207047F0B44268D8
:10D3000081680446530424345B0C4D041F196D0CD2
:10D31000AB4205D14A401204D20F0124624022D10F
:10D32000028A848A16197C783A7824021443FA789F
:10D33000BF7812023A43A718BE4217D3002A02D080
:10D34000AA4213D30FE0827EDB1D1419E318008874
:10D350009BB2C01A80B22232904202D2480403D05B
:10D3600004E09D4202D10020F0BC7047F0BC0120D7
:10D370007047F0B5876803467C042433640C82B0A0
:10D38000E618C56801966E04760CA64203D17D406E
:10D390002D04ED0F15D1A64208D9351B867EAD1B95
:10D3A000ED1F2DB2AE460025AC4607E00588877E0E
:10D3B0002D1BED1BED1F2DB2AE46B4467546002D5C
:10D3C00004DA0021C182084602B0F0BD458A00950A
:10D3D000002D18D0019F7D783E782D023543FE78D0
:10D3E000BF7836023E430ED06446A41BA6B200248A
:10D3F0004476964205D3009CE3185B1BDB1E0B6052
:10D4000010E0C4821FE07646761B37B200264676CF
:10D41000974212DB857EED1D2D19009CE318EB1859
:10D42000DB1E0B60C28209680A78C2764A780277EE
:10D4300089784177012002B0F0BD944502D30124E0
:10D440004476D8E7C682002002B0F0BDF7B50446A6
:10D4500084B02430019020890F464104490C019882
:10D4600002910D18E08A002801D0B84202D20020B3
:10D4700007B0F0BD608A002818D069782A780E02BB
:10D480001643E978AA78090211430091711888427D
:10D4900001D00CF06AFF617E00980A4602432046E4
:10D4A0000830002A05D000292ED038E0002600964A
:10D4B000F1E7618A00290DD0A27E029BD21DD2180D
:10D4C000019BC9185118E27EC91E0A70227F4A705A
:10D4D000627F8A70628AF119D21962822970090A00
:10D4E00069700026AE70EE700699002941D0697807
:10D4F0002A78A37E09021143DB1D591889B22288BC
:10D50000FFF7E0FC668234E0628A01995118891BBA
:10D51000E27EC91E0A70227F4A70627F8A7000997B
:10D52000628AC919D21962822E70320A89B26A706F
:10D53000A9700A0AEA70069A002A1AD005460088DD
:10D540000F464004400CB84201D80CF00EFFF00B1F
:10D550007904C003490C0843298801220904C9172A
:10D56000D203C903891889B290430143002029607E
:10D5700060820020E0822076012007B0F0BDF0B488
:10D580004568846802466E042432760C6704B3183A
:10D590007F0CBE4205D165402C04E40F01256C4090
:10D5A00002D1048A002C02D0F0BC002070471C1D60
:10D5B0000C60807EC01DC018C01E486058781C7862
:10D5C000000220430881CA60DC789D7823022B4347
:10D5D0000B82002803D1D21E4A600B810882F0BC66
:10D5E00001207047F8B504460346616880684A0424
:10D5F0002433520C4604D318760C00270125B2427E
:10D6000004D141400804C00F684005D1208A002899
:10D6100002D1A08A002801D00020F8BD58781978DE
:10D6200000020843D9789B780D021D4317D0261DB0
:10D63000AA4201D80CF099FEE00B6904C003490C22
:10D640000843318801220904C917D203C903891884
:10D6500089B2904301433160A7820120F8BDA37EC7
:10D660002288DB1D181881B2201DFFF72BFCF3E781
:10D6700038B5049C00932346FFF75CFC38BD134685
:10D6800010B50A461946FFF74FFC80B210BD10B521
:10D69000FFF77CFC10BD10B5FFF70CFE10BD10B5F8
:10D6A000FFF71AFE10BD10B5FFF772FC10BD10B5E4
:10D6B000FFF7D9FC10BD10B50022FFF7ACFD10BD7F
:10D6C00010B5FFF722FD10BD10B5FFF755FD10BDD9
:10D6D00010B5FFF713FE10BD30B500240346002A35
:10D6E0000BD0181D18600023521E04E04518056079
:10D6F0005B1C2846DBB29342F8DB046030BD014678
:10D700000A680020002A02D0104612680A6070479A
:10D7100002680A6001607047F8B50D46064600F0E1
:10D72000ADF9002801D10CF020FEF848A9000F182F
:10D73000B000B96A00900858002801D00CF015FE1E
:10D74000B868FFF7DCFF040030D0B96A00982B00FE
:10D750000C5020460CF024FF0805050A0D10151882
:10D76000232821463046F6F7ACF91FE0F4F717FFFF
:10D770001CE0FAF75CFE19E021463046F8F704FC9D
:10D7800014E0F7F75FFC11E0E049E14B7A310A461B
:10D7900000912E3A2146304608F0C6FC06E02146AC
:10D7A000304609F07DF801E00CF0DFFD2046F8BDC1
:10D7B000FFB581B0064600900A981F461818C4B2FB
:10D7C000002E08D00025FF2801D90CF0CEFD0298CC
:10D7D000002804D101E00125F5E70CF0C6FDF01C9E
:10D7E00080088000B04201D00CF0BFFD0A99039878
:10D7F000884201D90CF0B9FD002D0BD1C34900209E
:10D800004C310870C34A4A80C1490870BF497A3117
:10D8100008704A80BD480399017047708470C470D5
:10D82000047144710A998171C7712946684600F0F4
:10D830002DF900980421C01C800880000090002D64
:10D8400004D1B24A90642246FFF746FF0098A10037
:10D85000001D401800900020A1008E460099C91CB0
:10D86000890889000091002D0FD1A84A83009A18D9
:10D870009162944600210A4605E063468F009B6A48
:10D88000491CDA51C9B2A142F7D3009A7146511826
:10D89000401CC0B200910828E0D3881B0299088080
:10D8A000002005B0F0BD30B59B490968884201D21F
:10D8B000102030BD0278954B9200D21841889B7899
:10D8C0000FE0946A8D006459002C08D04B1C4380F3
:10D8D0008180926A890051588160002030BD491CC6
:10D8E00089B28B42EDD84180052030BD8A4A12684A
:10D8F000914201D210207047082801D307207047B9
:10D9000008700020488070470EB56946FFF7EEFFAB
:10D91000002801D00CF029FD6846FFF7C4FF00285D
:10D9200001D000200EBD01200EBD10B50446082810
:10D9300001D30CF01AFD7548005D10BD3EB50546DB
:10D9400000246946FFF7D2FF002804D00CF00DFD3B
:10D9500001E0641CE4B26846FFF7A5FF0028F8D098
:10D960002846FFF7E2FF001BC0B23EBD10B50446DB
:10D9700000F084F8002801D0E0B210BDFF2010BDF7
:10D9800070B50C460546062901D0072C10D15F4E14
:10D99000B06CFFF7B4FE5F49002805D0B26C801A66
:10D9A000001F0004800C00E008462880884201D156
:10D9B000002070BD2146FFF7AFFE040002D1288889
:10D9C00000F08BF8204670BD524A904201D00829E1
:10D9D00001D3002070479FE64E4A10B5904201D017
:10D9E000082901D3002010BD00F081F810BDF8B562
:10D9F00006464848494F0C4686423DD0082C01D384
:10DA00000720F8BD304600F072F8050034D023003E
:10DA10000CF0C6FD0805050A0D12171E1E1C29462E
:10DA20003046F6F76CF813E0F4F7C9FD10E029462C
:10DA30003046FAF725FD0BE029463046F8F7DAFACA
:10DA400006E029463046F7F704FB01E00CF08DFCB8
:10DA50002E48A20017180021B200B86A062C815087
:10DA600001D0072C02D1304600F037F82946B868BB
:10DA7000FFF74EFE0020F8BD3846F8BD23498978EF
:10DA8000814201D90120704700207047F3B51F4F34
:10DA900081B00546002422486100465A1D48F61C04
:10DAA000C01E06402868C01C8008800028600299BB
:10DAB000002906D1A100C91988603A5D3146FFF7F7
:10DAC0000BFE2868001D2860395D641C71434018F6
:10DAD000E4B22860082CDED3FEBD014610B50B4829
:10DAE0008900806C091D4118FFF712FE10BD70B54A
:10DAF0000C460546FFF7C2FF002805D00349A000E9
:10DB00004018806AA900405870BD0000AC08002091
:10DB100052000020FFFF00001C0000200230000027
:10DB2000D0A50100014610B5AA4800220068026095
:10DB3000037A9B001818C260018211460C3000F075
:10DB400040F910BDFFB5002681B0154604460028F7
:10DB500033D000200090E01C80088000A04201D05B
:10DB60000CF003FC002D38D00021084600F023F90A
:10DB700006466F1E7E4300200A9900F01CF90499A6
:10DB800000224018361811461046FFF778FD7843FA
:10DB90008619002210460C99FFF771FD0B99401869
:10DBA0000621301869430818A9000C300818081815
:10DBB00086B20098002802D00FE00120CAE7701A50
:10DBC0000C3887B283480460204625720C306060B0
:10DBD0000CF0A0FA3846FFF7A5FF02980680002057
:10DBE00005B0F0BDFFB57B4C0546206883B000282A
:10DBF00001D10CF0BAFB2068017AA94205D9A9002D
:10DC0000426802915158002902D0734807B0F0BD14
:10DC10000068002848D00C99059800F0CCF8C51C85
:10DC20006E4E0022354006990498FFF728FDC01C6F
:10DC3000304001904019001D86B2664800210068FE
:10DC4000046801E0214614462268002A02D0A38815
:10DC5000B342F7D1A288B24226D32268002901D06C
:10DC60000A6000E002602068002700280CD13046DE
:10DC70000830A28880B2824206D9A019921B0760A0
:10DC8000828000F09EF8A680A088608025800C9B92
:10DC9000059A201D0093064629460123FFF74AF9FD
:10DCA000002803D0002002E00420AFE70420A842AF
:10DCB00001D90CF05AFB208800978019069B049A22
:10DCC0000199FFF7D5FC43480068416802980C5061
:10DCD00000209BE770B53F4C06462068002801D124
:10DCE0000CF043FB2068017AB14210D94568B300BB
:10DCF000E85800280BD041880022EA500260818059
:10DD0000114600F05EF8216800200A7A08E03248E7
:10DD100070BD4B6884001B59002B0DD1401CC0B254
:10DD20008242F6D8002002E08A88101880B2096882
:10DD30000029F9D1FFF7F6FE002070BD70B5254D22
:10DD4000286800280AD0002404E02046FFF7C2FF1C
:10DD5000641CE4B22868007AA042F6D870BD70B5A1
:10DD60001C4E054630680024002801D10CF0FDFA55
:10DD70003068017AA94205D94068A90040580028B6
:10DD800000D0041D204670BD70B5124E05463068A7
:10DD90000024002801D10CF0E8FA3068017AA94289
:10DDA00007D94068A9004158002902D00888091DF8
:10DDB0004418204670BD10B50A460121FFF7B4F89B
:10DDC00010BD002903D00A6802600860704701494D
:10DDD0000968F8E75800002002300000FCFF00004E
:10DDE000F8B507780D460446012F19D0072F02D049
:10DDF0000C2F19D114E0A068216906780B2E0BD0E6
:10DE0000052003F0DCFC052E0ED07823002205202F
:10DE1000216903F044FC07E0782300220620F8E79C
:10DE20000520216903F0CBFC002D0ED000202870C6
:10DE300029462046F5F718FCFE482978C05D88423F
:10DE400001D10320F8BD0220F8BD00212046F5F7DE
:10DE50000BFC0020F8BD70B50E460C462036317A1A
:10DE600001208AB01546002909D0012905D1297859
:10DE7000042902D10520107000200AB070BD60682E
:10DE8000019005A802900D21C01C0CF041F903225D
:10DE900005A8A1680CF0DFF8012030720620694661
:10DEA0000870606A049029466846FFF799FFE4E726
:10DEB00070B50C46154620310A7A0120062686B038
:10DEC000002A2CD0012A28D12978042925D1696873
:10DED0001022A06801F061FB6868C07B000606D5CF
:10DEE000D44AA0681023103A014601F04BFB1022DF
:10DEF000A168E06801F051FBA068C07B000606D570
:10DF0000CC4AE0681023103A014601F03BFB2E702A
:10DF1000A0686860E068A860002006B070BD606816
:10DF20000190C448203802900120087268460670AB
:10DF3000606A049029466846FFF752FFEDE7027BCE
:10DF4000032A06D0002228235A540B780D2B02D026
:10DF500003E0042070470A76CA61027B9300521CDA
:10DF60000273C15003207047F0B50E4615460C46AB
:10DF700020360246317A0120072393B000290CD0C5
:10DF8000012924D002292ED0032904D1297804297B
:10DF900001D12B70002013B0F0BD012030726068F9
:10DFA00000280DD0A1690B70606848602069886006
:10DFB0006069C860606A48621046FFF7C0FFEAE720
:10DFC00006202870206968606069A86009E02978E7
:10DFD0000629E0D1022030720420287095482038AC
:10DFE00068600320D7E729780429D4D1A0891028B4
:10DFF0000AD9103880B2A081A1681023091805A899
:10E000006A6801F0BFFA23E010282FD0C2B21020B6
:10E01000801AA1680DAF1190C0190CF01CF811986E
:10E020000006000E06D0401EC1B28020785438464B
:10E030000CF06EF8626910230DA909A801F0A2FA8C
:10E04000102309A905A86A6801F09CFA0320307220
:10E050006068019005A80290062069460870606A11
:10E06000049029466846FFF7BBFE94E71023226917
:10E07000A168E2E7F7B50E4620360D46337A012057
:10E080000821002B07D0012B04D11378072B01D1D5
:10E0900011700020FEBD6C6901272170E868606086
:10E0A000686A6062A168287C0870A781A068A96876
:10E0B0002022401C0BF0CFFFA08920222030A0811D
:10E0C000A068696821300BF0C6FFA0892146203086
:10E0D000A08137720098FFF732FFFEBDF7B50E46FC
:10E0E0000C462036317A01201746002913D0012929
:10E0F00023D0022979D003290CD13978072909D1F5
:10E1000079681022E0690BF0A6FF092038701834F6
:10E1100000207C60FEBD216A0820087045480E3052
:10E12000486020208881606A4862E26988681060DF
:10E130006068886001203072AEE039780729E9D143
:10E14000256A08202870606A6862E0690068A86033
:10E1500051681022E0690BF07EFFE0696860A868F2
:10E16000002707700120A881A96807224870A889A4
:10E17000401C80B2A881A968081861690BF06BFF88
:10E18000A8890722C01D80B2A881A9680818216942
:10E190000BF061FFA8891022C01D80B2A881A96878
:10E1A0000818E1680BF057FFA8891022103080B2E0
:10E1B000A881A9680818A1680BF04DFFA88904225E
:10E1C000103080B2A881A96808181A4924390BF0C8
:10E1D00042FFA889001D80B2A881A9680F54A889B0
:10E1E000401CA881022055E0FFE73978072991D12A
:10E1F00051681022A0690BF02EFF256A08202870B4
:10E20000E0696860606A6862A96800200870012798
:10E21000AF81A86807224770A889401C80B2A881F6
:10E22000A968081861690BF016FFA889C01D80B2A3
:10E23000A88101E00CA60100A9680722081821693D
:10E240000BF009FFA8891022C01D80B2A881A9681F
:10E250000818E1680BF0FFFEA8891022103080B288
:10E26000A881A9680818A1680BF0F5FEA889042206
:10E27000103080B2A881A9680818FC490BF0EBFEA9
:10E28000A889001D80B2A881A9680F54A889401CE4
:10E29000A8810320307229460098FFF750FEFEBD8A
:10E2A000F8B50E460D4620360746317A0120002982
:10E2B00008D0012905D11178072902D10A20107050
:10E2C0000020F8BD2C6A0820207068686060686AC9
:10E2D0006062E9690722A0680BF0BDFE0720A081FB
:10E2E000A0680722C01DA9690BF0B5FEA089032212
:10E2F000C01D80B2A081A168081869690BF0ABFE4F
:10E30000A0891022C01C80B2A081A16808182969C8
:10E310000BF0A1FEA0891022103080B2A081A1686C
:10E320000818E9680BF097FEA0891022103080B21F
:10E33000A081A1680818A9680BF08DFEA08921466C
:10E340001030A081012030723846FFF7F8FDF8BD8B
:10E35000F8B50E460D4620360746317A01201446A0
:10E3600000290DD001290AD12178072907D1606839
:10E370000C21001D0BF0CCFE0B2020700020F8BDFE
:10E380006C6908202070E8686060686A60622969CA
:10E390001022A0680BF05FFE1020A081A068202250
:10E3A0001030A9680BF057FEA0892022203080B2DF
:10E3B000A081A168081869680BF04DFEA08921466C
:10E3C0002030A081012030723846FFF7B8FDF8BD3B
:10E3D000F0B50E460C462036317A012006278FB064
:10E3E000154600290BD0012932D0022905D1297800
:10E3F000042902D10C20107000200FB0F0BD217D47
:10E4000008A8CA07D20F02718807C10F08A80171B6
:10E410006846027041700722801CE1680BF01BFE09
:10E4200002A80722013021690BF015FE60680590F3
:10E430000AA8069010236A46A16801F0A3F80120FB
:10E44000307268460774606A0890294604A820E084
:10E4500029780429D1D1062205A8E1690BF0FBFD3A
:10E4600006A806220230A1690BF0F5FD00200890F5
:10E470006068019009A80290102305AA696801F05C
:10E4800081F80220307268460770606A049029465D
:10E490006846FFF7A5FCB0E770B50D460C46203581
:10E4A000297A01208CB01646002909D0012905D10E
:10E4B0003178042902D10D20107000200CB070BDFD
:10E4C0006068019006A802900822E1680BF0C3FD85
:10E4D000082208A8A1680BF0BEFD012028720620C2
:10E4E00069460870606A049031466846FFF778FC18
:10E4F000E4E770B50D460C462035297A01208CB032
:10E500001646002908D00129D8D131780429D5D15F
:10E510000E2010700020D1E76068019006A80290DC
:10E520000822A1680BF097FD0020089009900120B7
:10E530002872062069460870606A04903146684671
:10E54000FFF74EFCBAE730B50B4620331C7A0120AA
:10E550008BB0002C09D0012C05D11178042902D1EF
:10E560000F20107000200BB030BD4868019005A846
:10E5700002908C6868462578057564784475CC6887
:10E58000257885756478C4750020069007900890FA
:10E5900001201872062368460370486A04901146E9
:10E5A0006846FFF71DFCDEE770B50C4620340346D5
:10E5B000257A0120002D0AD0012D15D0022D05D17C
:10E5C00011780E2902D110201070002070BD01209A
:10E5D0002072C868052202704A684260234A921F6E
:10E5E0008260921CC2600BE015780F2DEED10220E4
:10E5F0002072C86804240470526842608A6882608D
:10E60000496A416201461846FFF799FC70BD30B572
:10E61000011D02463132947803258379ED432C4362
:10E6200023408371DB070DD04B79547923404B7124
:10E630000B79127913400B718278C9788A4200D91C
:10E64000817030BD00224A710A71F5E7F7B50C46BA
:10E6500086B000206946264608702036317A0127A8
:10E660001E2015461F297BD202E00000E8A501000C
:10E670004B007B449B885B009F441E0015023C02BC
:10E680005402670286029802CF02F3022C0357035A
:10E690006F037D03AC03C103CA03F50318046204CE
:10E6A0009804A904DD04FC040E05280562059805FC
:10E6B000C3058005840588056069002802D00078BC
:10E6C00013287DD0A0680590002849D00121684614
:10E6D0000170606A04900321684601710A2141714A
:10E6E000E069029020790028EFD005990978002987
:10E6F000E7D00C2964D20B000BF052FF0CFD1A4B33
:10E7000090B5E8FCFBFAF9F807FD022828D160690A
:10E71000002802D00078082852D1022168460170F2
:10E72000606A049005984178684601710021B7E25B
:10E730000620616A03F043F820790728E6D1606972
:10E7400000F04DFF02280CD0606900F048FF04285B
:10E7500007D060690028B8D000780128D6D103E03E
:10E7600019E261690120087005980079C11F0A2922
:10E7700001D30A2050E06169072288706069059919
:10E7800030300BF068FC01203072616903200870A2
:10E7900034E00728BAD16069002896D001780929A9
:10E7A000B4D10599C978890707D105994979002914
:10E7B000DFD1059989790029DBD10599497900E0F4
:10E7C0004CE202462032537D9943D2D10599937D84
:10E7D00089799943CDD105990979CB1F0A2BC8D2E4
:10E7E00012798A4236D80722C01C05990BF033FCF7
:10E7F0000120307261690A200870032069460870A0
:10E80000606A04906069313001906069001D029077
:10E8100060691C3003909FE22076F0E311288DD1CF
:10E82000606900F0DCFE042804D0606900F0D7FEC7
:10E830000B2893D16069059910223730491C0BF0E1
:10E840000AFC6069017804297CD12421095C827862
:10E85000914201D90620DFE70521017003203072C3
:10E8600068460170E0E3112894D1606900F0B7FEBA
:10E87000062804D0606900F0B2FE0C288AD1E06856
:10E88000002813D02069002810D06069017806297B
:10E8900010D00D2101706069059910225730491C74
:10E8A0000BF0D9FB6069573009218AE100206946E5
:10E8B000087070E1072101706069059910224730E6
:10E8C000491C0BF0C8FB60694730EDE70228F0D126
:10E8D000606900F084FE0028EBD0606900F07FFEE4
:10E8E0000128E6D0606900F07AFE05E0AFE08BE039
:10E8F0006AE02AE00AE0D4E00828DAD00521684678
:10E900000171059841786846417144E11128D0D1E0
:10E9100060690028CDD001780E29CAD1C16A40783B
:10E92000022810D0002014225043143008580599B2
:10E930001022491C0BF08FFB0520616A00F03DFEA0
:10E940000F205CE0EFE10120EDE70B28B1D1606919
:10E950000028AED001780F29ABD1C16A40780228D7
:10E9600026D00020142250430C30095805984278D4
:10E970000A70807848706069C16A4078022819D0AE
:10E980000020142250431030085805990822C91C51
:10E990000BF061FB0520616A00F00FFE60694178B1
:10E9A000022909D000220832825C5208520071E02C
:10E9B0000120D7E70120E4E70122F4E7012100E08C
:10E9C000002108314254B9E311289ED16069002822
:10E9D0009BD00178102998D1C16A4078022811D0C3
:10E9E0000020142250431830085805991022491C61
:10E9F0000BF031FB0520616A00F0DFFD1120616939
:10EA00000870B3E30120ECE7082886D1606900288C
:10EA10009FD00178112999D10599C06A4978017070
:10EA200060690599C06A0622401C891C0BF013FB23
:10EA30000520616A00F0C1FD60694178022904D0B7
:10EA400000220832825CFD2323E00122F9E711282D
:10EA5000BBD160690028BBD001781229B5D1C16A49
:10EA60004078022819D00020142250431C30085846
:10EA700005991022491C0BF0EEFA0520616A00F09E
:10EA80009CFD60694178022909D000220832825C2D
:10EA9000FB231A40022993D190E70120E4E70122E9
:10EAA000F4E70720B8E6287801288ED16069696804
:10EAB00014221C30F2F76AFB6069017F002901D043
:10EAC0002176ABE30178032901D0032037E0022748
:10EAD000C77081794907490F8171017A4907490F48
:10EAE0000172417A4907490F41726069FFF78FFD52
:10EAF000377296E228781328E3D107206946087018
:10EB0000616A0491916802916946087161690722FE
:10EB1000C91C02980BF09FFA61690420087000205C
:10EB20003072BBE028780328CBD1606901780529D1
:10EB3000696807D0082247300BF08DFA0420307244
:10EB400005206FE208225730F6E728780328B8D16D
:10EB5000606901780529696811D008224F300BF0EF
:10EB60007AFA052030726069006A00280AD0022013
:10EB70002870002028716069006AA860F9E0082206
:10EB80005F30ECE704204DE22878022899D12879FB
:10EB9000002801D0207641E36069A96801626069BC
:10EBA000002901D1F949016206200BE228781328D7
:10EBB00087D1A868E0616069017805292BD04730CA
:10EBC00007213172E16802220A706269126A4A60A2
:10EBD000886060693030C8606069C01C0861626923
:10EBE000087D926A400812784000D207D20F104385
:10EBF00008756269926A521C8A61FD22104062693E
:10EC0000D26A1278D207920F104308756069C06A01
:10EC1000401CC86153E25730D2E728780C28BAD19B
:10EC20006069017805291AD00B2101700720694617
:10EC30000870606A0490E0690290112008710298DF
:10EC40000321017051681022401C0BF004FA0021CE
:10EC50006846FFF7C5F800203072E06186E20621C1
:10EC6000E3E72878132896D1072069460870606A80
:10EC70000490A86802901120087102980421017084
:10EC800061690A78072A0ED0002232720C220A70BB
:10EC900061691022401C47310BF0DDF90021684604
:10ECA000FFF79EF862E21022401C57310BF0D3F9B7
:10ECB00000216846FFF794F80A203072E1680320CB
:10ECC00008706069006A48606069573088606069F0
:10ECD0004730F3E128780C28A1D1606969681022D7
:10ECE00037300BF08BF9002801D0042094E56069DF
:10ECF0000078072817D00A203072E16803200870D6
:10ED00006069006A486060695730886060694730B0
:10ED1000C860606A48620698FFF711F907466069A3
:10ED2000FFF775FC6AE208207AE128780D289AD16D
:10ED30000B20307261696868897810224018511A76
:10ED40000BF0E6F9082069460870606A049068686C
:10ED5000019060698078087268E129781129BBD137
:10ED600061698979C90703D00C20307209203EE01F
:10ED7000307203276FE228781228ADD1606914221F
:10ED8000291D1C30F2F702FA6069018DC06A4172D8
:10ED9000090A817260698178C06AC1716069C26A5A
:10EDA000117AC909C9011172437A626919438379D9
:10EDB000D26A9B079B0F001D012B00D00023007916
:10EDC0009B01C00003431943117260694078012818
:10EDD00076D0B3E160694178022901D0012100E0D9
:10EDE00000210831405CC00707D00E20EAE06946E8
:10EDF0000870606A1146049019E11320B8E728787A
:10EE0000132894D1A868E0610F2030720520EEE746
:10EE1000287803288BD16069C16A4078022801D024
:10EE2000012000E00020142250431030085808222E
:10EE300069680BF010F910203072E1680620226931
:10EE400008706069406A48606069C36A4078022857
:10EE500001D0012000E0002014277843103018581A
:10EE6000CA6088602BE12878102886D16069C26A60
:10EE70004078022801D0012000E0002014214843FE
:10EE80000C30105802230932696800F07BFB112016
:10EE90003072E168052008706069006A4860606946
:10EEA000C06A093088603948083807E128780F2897
:10EEB000A7D161694878CA6A022802D0012001E01E
:10EEC00058E1002014235843143010588A78696898
:10EED0000BF0C1F860694178C26A022901D00121B2
:10EEE00000E00021142359431431525881785018FE
:10EEF0001022511A0BF00CF9072069460870606A5D
:10EF00000490E069029011200871029806210170B6
:10EF10006169CA6A4978022901D0012100E0002113
:10EF200014235943143151581022401C0BF093F80C
:10EF300000216846FEF754FF0020E06112206FE0D8
:10EF40002878132891D1072168460170606A0490DF
:10EF5000906802900B226846027102980170616904
:10EF6000CA6A4978022901D0012100E00021142356
:10EF700059430C3151580A7842704978817061695F
:10EF8000CA6A4978022903D0012102E0ECA50100F8
:10EF9000002114235943103151580822C01C0BF092
:10EFA0005AF800216846FEF71BFF26E760694178A2
:10EFB000022901D0012100E000210831405C8007D6
:10EFC00003D5142030720A2011E71620D0E62878E5
:10EFD00013287AD1A868E061072069460870606A42
:10EFE0000490E069029011200871029808210170D4
:10EFF0006169CA6A4978022902D0012101E010E161
:10F00000002114235943183151581022401C0BF091
:10F0100022F800216846FEF7E3FE0020E06115209B
:10F0200030720A2069460870606A04902946684672
:10F03000FEF7D6FE2BE02878132846D10720694634
:10F040000870606A04909068029008200871029825
:10F050000921017061690622C969097841706169F5
:10F06000801CC969491C0AF0F6FF00216846FEF7BA
:10F07000B7FEAAE761694878022801D0012200E0C2
:10F0800000220832895C490703D51720C8E70746E4
:10F09000B4E0012852D06FE02878132815D1A86871
:10F0A000E06118203072E168052008706069006A2C
:10F0B00048606069C06A09308860F748C860606A63
:10F0C00048620698FEF73BFFE1E76EE028780F28DC
:10F0D0006BD16069C16A4078022801D0012000E04C
:10F0E0000020142250431C300858102269680AF08E
:10F0F000B2FF072069460870606A0490E0690290D8
:10F100001120087102980A2101706169CA6A497860
:10F11000022901D0012100E00021142359431C31B0
:10F1200051581022401C0AF096FF00216846FEF755
:10F1300057FE0020E06160694078AAE7192017E6D1
:10F1400060694278022A09D0002108314118097803
:10F1500000290DD0CA0703D00E2106E00121F4E7F3
:10F16000890701D5102100E012210170002772E00B
:10F17000012A01D00D20FBE51C20F9E51D2030728D
:10F180000B2034E62978142948D1F1E5606901782B
:10F19000012943D0082941D00021317200F019FA29
:10F1A0000C2069460870606A049037E028781328BC
:10F1B00005D01420107003271B2030724BE007216C
:10F1C00068460170606A0490A8680290022168464F
:10F1D0000171029805210170217E4170002168466D
:10F1E000FEF7FEFD0B2168460170606A0490294617
:10F1F0006846FEF7F5FD07461B203072012F0DD043
:10F2000029E0012168460170606A04900421684683
:10F210000171217E41710020207612E0207E0028BD
:10F220000FD06169132008701A2030720A206946D5
:10F230000870606A049029466846FEF7D1FD0746CB
:10F2400009E06069002801D0142101706846007847
:10F25000002800D022E5384609B0F0BDF7B50F46CA
:10F260002037387A012686B00C46002804D00128C1
:10F2700028D002281CD197E02079012804D0022848
:10F2800011D0032814D10AE0A068407801280ED1DB
:10F290000620616A02F06DFA00287FD10CE0A168B7
:10F2A0001320087008E0A0684178022901D00526E3
:10F2B00074E00078082871D1012038720A2069466C
:10F2C000087033E008980078132867D10721684652
:10F2D0000170606A0490089885680295227902207E
:10F2E000012A04D0022A29D0032A57D10FE006466A
:10F2F000684606710B202870207B00214007400FD4
:10F3000068706846FEF76CFDA068067045E006462A
:10F310006846067105202870207B687000216846C9
:10F32000FEF75EFD3E720B2168460170606A049034
:10F3300068460899FEF754FD06462FE068460171BD
:10F3400001202870207C6870607CC007C00FA87006
:10F35000A07C4007400FE870E17C2971C0071FD0F6
:10F36000207D4007400F6871607D4007400FA87105
:10F3700000216846FEF734FDA06807222946303098
:10F380000AF069FEE068017AA06820300171A16886
:10F3900028798870A16809200870002630465BE74C
:10F3A0000020A8716871E3E7A168142008700121AA
:10F3B00068460170606A0490042168460171217BEF
:10F3C00041710021FEF70CFDE7E7F0B585B00F466F
:10F3D00005460124287B800040198038C66F3078AC
:10F3E000411E0E290AD22C4980004631401880382F
:10F3F000C36F3A463146284698470446002C01D050
:10F40000012C11D1287B401E0006000E287301D06C
:10F410000324DFE70D2069460870706A049000211C
:10F4200001966846FEF7DCFC032CD3D0204605B0DD
:10F43000F0BD70B515460A46044629461046FFF74A
:10F44000C4FF0646002C0FD0207814280CD1207E53
:10F45000002806D000202870204629460C30FFF7EF
:10F46000B4FF204600F0B5F8304670BD704710B5C7
:10F47000012903D0022901D0052010BD417000F000
:10F48000A8F8002010BD002808D0027E002A05D070
:10F490000A4601460C31CCE7E6A501000120704781
:10F4A00030B5044687B00D46062002F088F929469B
:10F4B000052002F084F92078142805D00020694640
:10F4C00008702046FFF7DFFF07B030BD7FB50E465E
:10F4D00000216A46117301780D2903D00E2903D04B
:10F4E000002407E0446900E08468002C02D0217EFB
:10F4F000002912D0154601462846FEF720FD0328B4
:10F5000009D1324629462046FFF793FF6946097B19
:10F51000002900D0042004B070BD25460C35EAE770
:10F5200000B50023012285B005280CD0062808D19B
:10F530006846027004910221017143710021FEF7B7
:10F540004FFC05B000BD6846027004910271F4E7FB
:10F5500010B592B00C4605216B46197001902348F6
:10F560000290001D039009920BA96846FFF7AEFFB9
:10F57000002805D1102220460C990AF06CFD0020CD
:10F5800012B010BD30B505E05B1EDBB2CC5CD55CC3
:10F590006C40C454002BF7D130BD10B5002409E0F5
:10F5A0000B78521E5B00234303700B78401CDC0970
:10F5B000D2B2491C002AF3D110BD70B50C460546E5
:10F5C00002F0FDF8782300222146284602F067F871
:10F5D00070BD4178012900D00821017070470028D2
:10F5E00001D000787047082070470000E0A50100B6
:10F5F00070B50D46040012D0002D10D02101284610
:10F600000AF086FD1022544928460AF024FD52488B
:10F6100001210838018044804560002070BD012030
:10F6200070BD70B54C4E00240546083E11E071686F
:10F6300020014018817BAA7B914209D1C17BEA7BE2
:10F64000914205D10C2229460AF0D8FC002806D0A8
:10F65000641C30888442EADB0020C04370BD204631
:10F6600070BD70B50D4606000AD0002D08D03A4C8A
:10F67000083C20886188401C884203D9042070BD62
:10F68000102070BD3046FFF7CCFF002801DB401C86
:10F690000AE02088616800014018102231460AF013
:10F6A000DAFC2088401C20802870002070BD70B5D6
:10F6B00014460D001FD0002C1DD00021A17002287F
:10F6C00002D0102817D108E0687829780002084392
:10F6D00011D00121A17010800BE02846FFF7A1FF97
:10F6E000002808DB401CA070687B297B00020843CF
:10F6F0002080002070BD012070BD70B50546144605
:10F700000E000AD000203070A878012807D004D954
:10F71000114908390A8890420BD9012070BD002C8C
:10F7200004D0287820702888000A507002200870C1
:10F7300010E0002C0CD0496800014118102220462E
:10F7400010390AF088FC287820732888000A607332
:10F7500010203070002070BD64000020F8B5FE4C11
:10F76000207EE17D88421AD00126FC4D0027E07DF5
:10F77000215C14200A4642435019037C052B0FD00C
:10F78000037C062B1AD0037C072B26D0437C012B4D
:10F7900031D00AF0EAFD207EE17D8842E7D1F8BD54
:10F7A0000674E07D162807D0E07D401CE075491CFA
:10F7B000C8B2AA5802210CE00020F7E70674E07DE9
:10F7C000162808D0E07D401CE075491CC8B2AA5834
:10F7D00003219047DFE70020F6E70674E07D162856
:10F7E00007D0E07D401CE075491CC8B2AA5808212A
:10F7F000EFE70020F7E74774E07D162807D0E07DAB
:10F80000401CE075491CC8B2AA580721E1E7002056
:10F81000F7E770B50024D24E0C207072D14825460F
:10F820004473047328300476C475CF4809F0A0FAF5
:10F83000CE480575F572CE49601E88607571B57049
:10F84000F57035717570CB48E83905704570142036
:10F85000604340180574641CE4B20B2CF7D30120FC
:10F86000F9F708F90020F9F705F90120B071F9F767
:10F8700077FCC148F9F786FCC04C2070C048F9F706
:10F8800081FC6070F9F798F870BD10B5F9F7BFF812
:10F89000BA4C2078F9F792FC6078F9F78FFCB04CFD
:10F8A000207A002803D0F9F774FA0020207210BDE6
:10F8B000F8B5F9F766F9AA4D0446A879002802D0F0
:10F8C0000AF053FDF8BDE87A002801D10AF04DFD99
:10F8D000A74F01237969AB4A601A9B0598420ED362
:10F8E0000E1B9E420BD3904203D9501A0019401CA4
:10F8F00005E0964233D9101B4018401C40420028B6
:10F9000001DB0AF032FD0126AE710024EC72687A48
:10F91000042114225043914A80180174B868401C95
:10F9200004D0481FB8600120F9F7A4F80020F9F7C7
:10F93000A1F8F9F787F809F0FBFAF9F782F992488C
:10F940000460046001209149C0030860F9F7ECF9F4
:10F9500088480078022808D0032803D007E00AF07E
:10F9600004FDCEE7E878002801D0AE7000E0AC706E
:10F97000F9F753F9F8BD034678490B2014224243A6
:10F980005218203A127F002A04D0401E0006000EB2
:10F99000F4D170471422424351180A46803AD36684
:10F9A000012220390A777047012805D0032805D1A4
:10F9B000002903D1002070470029FBD010B4684C07
:10F9C000002363706B4A002890700CD002280AD084
:10F9D00007291AD2080078440079001887441505D1
:10F9E000070D0F111300D37003E01B2000E03A2035
:10F9F000D0700120607010BC70475820F8E7772065
:10FA0000F6E79620F4E7B520F2E710BC0020704737
:10FA100010B558484078F9F71CF980B210BD411E66
:10FA20001422504310B54D4A8418203C0A2902D8AC
:10FA3000207F002801D10AF098FC207F012801D006
:10FA40000AF093FC0020207710BD70B5454C607B18
:10FA5000217B884201D1012500E00025F9F791F8CA
:10FA6000F9F7F7F8617B227B914201D1012100E097
:10FA70000021A942EBD170BDF7B50646481E844669
:10FA80008EB0C0B2142205905043344A85180495B4
:10FA9000287C2D1D07282AD12F4C0027E07D227EAF
:10FAA000824221D0235C059A934201D1012701E0D3
:10FAB000002F04D0162811D0421CA25C2254162814
:10FAC0000ED0401C227EC0B28242EBD1002F0BD060
:10FAD000207E002806D0207E401E04E00022ECE7B5
:10FAE0000020EFE716202076049A0120107460466B
:10FAF0001B4C0A2813D814204143184808182038F2
:10FB0000007F00280BD00498007C012809D00498BD
:10FB1000007C012803D01098807A012805D00AF0D3
:10FB200024FC1098807A01285BD104980B4B007C50
:10FB3000022831D0084C207E16285ED0207EE17D40
:10FB4000401C884201D10AF010FC0499012048743D
:10FB5000217E059860541BE0200B00203C0B002008
:10FB6000440C0020F80A0020500C0020080B002054
:10FB7000240C00207600002059150100740000209C
:10FB80005DF70000FFFFFF0000F5004080E200E0AD
:10FB9000207E162835D036E0607A059A01469042DC
:10FBA00006D0014614277843C018807C9042F8D1D3
:10FBB000627A824208D1617A14225143C918897C41
:10FBC00061720121A17207E014224243D218142766
:10FBD0007943927CC9188A7414220C215043C018AE
:10FBE00081741098007A06281DD2010079440979A1
:10FBF00049188F440C161412100EE07D0028A2D074
:10FC0000A3E7002001E0207E401C2076B1E0002028
:10FC10000CE0B4200AE0732008E0322006E00A205D
:10FC200004E0062002E00AF0A0FB002002901098F9
:10FC300001680298081A28601099097A002912D0E0
:10FC40000221401A0102090A2960109802684068DE
:10FC500010180002000A68601098807A0228109834
:10FC600003D0007B6FE00421EBE7007A002812D07C
:10FC70000222029812181098436810461030181883
:10FC80000A90F84843780298834202D9E078002825
:10FC900003D00A9805E00422EBE702981B1A0A98A1
:10FCA0001818637A10300C2B1CD0637A14277B430E
:10FCB000ED4FDB195B68994214D0EC4F617ABC467A
:10FCC00014235943E84BC9184B6889689B1B891B4F
:10FCD0001B0209021B0A090A984235D8634533D82A
:10FCE000614531D831180A980123081A0002000A28
:10FCF000286010998018C9680002000A471ADC4A77
:10FD00009B05BC469F4201D2384610E00F1A9F4225
:10FD100001D260460BE0944503D9511A0818401CE3
:10FD200005E0974206D9101A4018401C40420028AE
:10FD30005DDC01E00AF019FB29680A980818000246
:10FD4000000A6860002028726868102710300002DE
:10FD5000000A68601098407AA8721098007A687259
:10FD600003280ED200280CD001F078F9002803D027
:10FD700007E0002011B0F0BD3221029802910F1A65
:10FD80001037B8480178012901D0032909D14078FA
:10FD90000299884205D9E178002902D10299401AD6
:10FDA000C7196A682868921B801B944601021202D8
:10FDB000AE4B090A120A8F4219D81F46994216D82B
:10FDC000BA4214D8617A0C2915D0677A61460C22A0
:10FDD000039200921422A44B7A43D21893689B1B7F
:10FDE000834216D80397977C0C2FF3D16FE00598C8
:10FDF00001F0BBF8BDE70498022205990274627A0B
:10FE00000C2A00D0627A827461720120A07211B053
:10FE1000F0BD0C2F5BD00022384694461422924B42
:10FE20004243D21853689B1B8B4223D2907BAB7A00
:10FE3000984219D804980521059D01748D4C207EA7
:10FE400016280DD0207EE17D401C884201D10AF0A9
:10FE50008CFA207E2554207E162800D0D3E6D0E6EA
:10FE6000E07D0028F3D0F4E701208446907C0C2844
:10FE7000D4D102E06146002928D03D4600901420EC
:10FE80002A46424378480621161831741C38007EF1
:10FE90001628784814D0017EC07D491C814201D1CA
:10FEA0000AF063FA7348017E4554017E16290BD08F
:10FEB000017E491C0176B57C0098A842DFD106E09E
:10FEC000C07D0028ECD0EDE70021F3E7009704990E
:10FED0000220654D0874607AB84207D104990098F1
:10FEE0008874059860720120A0721DE003980C2FA1
:10FEF0000DD00C2801D10AF038FA0398142250438F
:10FF00004019059981740499009888740CE00C28B4
:10FF100001D10AF02AFA0398142250434019059996
:10FF2000817404990C208874012011B0F0BD30B5A3
:10FF30000D46514A441900210B46101A8B4101D23B
:10FF40000AF013FA4D48854201DD0AF00EFA4C48DA
:10FF5000854201DA0AF009FA4A48844205DA002C9F
:10FF600001DB204630BD474800E04748201830BD3F
:10FF7000401E70B5C0B2142148433B494418607B11
:10FF8000062813D201007944097949188F44020CDC
:10FF90000A080604002033E0B4200DE073200BE0D3
:10FFA000322009E00A2007E0062005E00AF0DDF92A
:10FFB000617B0020002923D002214018616840188D
:10FFC0000002000AF8F745FE0C2565572A4A441935
:10FFD00000210B46101A8B4101D20AF0C6F92748BE
:10FFE000854201DD0AF0C1F92548854201DA0AF0AF
:10FFF000BCF92448844207DA002C03DB204670BD9C
:020000040001F9
:100000000421DAE71F4800E01F48201870BDF0B552
:10001000064683B01D480190457A029534687068A1
:10002000001B070212483F0A001B00900C2D42D013
:100030001420294641430C4801220818844641688F
:100040000B4892058646081B904227D3631A9342B9
:1000500024D30246704672451AD900984018401CB5
:100060001CE00000760000203C0B0020FFFF3F005A
:10007000FFFFFF00200B0020FF7F841E0020A10750
:1000800000E05EF80080841E00807BE1440C0020CC
:1000900073450ED9411A0819401C404200280ADA5B
:1000A00060460295857C0198C0790028BED003B0D7
:1000B000F0BD0AF05AF90298854226D0142148432F
:1000C000FE490123401802908068FD499B058C463B
:1000D000011B8646994210D3221A9A420DD36346D9
:1000E000614503D900997144491C06E019466245EF
:1000F0002DD9091A0819401C4142002905DD029832
:10010000B17A807B814200D374460C2D15D0EB4927
:100110001420454368184268121B1202120ABA42A0
:100120000BD2B37A827B934200D38468857C01989A
:10013000C0790028BBD10C2DEAD13068A042B6D0DE
:10014000E0190002000A3460706003B0F0BD0AF0EC
:100150000CF9DAE7F0B5DB490446486885B0C0051C
:10016000C00D1CD0103840B200280CDA0207120F64
:10017000083A920892005118C9698007C00EC14020
:100180000806800F09E08108CF4A890089180968AC
:100190008007C00EC1400806800F002808D0002745
:1001A0002078002806D0012804D0002005B0F0BD3A
:1001B0000127F5E72079062813D20100794409794F
:1001C00049188F44020C0A080604002015E0B420E8
:1001D0000DE073200BE0322009E00A2007E0062042
:1001E00005E00AF0C2F821790020002905D002219B
:1001F0004618B64D002F02D003E00421F8E7002096
:10020000E871694602AAA068F8F72EFD694608223F
:100210008A56E06801A980180122C01C1F2801DA53
:10022000019209E003AAF8F71FFD6846007B002849
:1002300002D00198401C019000990198401810309C
:100240000002000A0190881B0002000A00906079F9
:100250006946887200980390F8F793FC009A019B16
:10026000121A181A9A4912020002120A000A8A4245
:1002700016D8884214D86846FFF7C9FE009903983B
:10028000814205D088190002000AF8F7E2FCA0605C
:100290000120E979002989D0002FB0D005B0F0BD48
:1002A0000020F6E7F3B58FB08A480C460B9008F0B3
:1002B00067FD894A0F99854F5618884D203E0028C2
:1002C00009D08748007D002801D00AF04EF8207838
:1002D00001287DD037E1687B16280AD0687B297B0E
:1002E000401C884201D10AF040F82078012804D04F
:1002F0000AE0287B0028F6D0F7E7F07F002801D03D
:100300000AF033F80120F077697B0F981422754EBC
:100310005143891908742078022822D0687B14215F
:1003200048438619207930726079707232460C32F7
:100330003146A068F8F798FC0C2030560F2804DDF1
:100340001F3830733068401C30600C217156301DEE
:10035000E26801905018C01C1F286EDA0120019934
:10036000DBE058494868C005C00D1ED0103840B2C7
:1003700000280CDA0207120F083A9208920051186E
:10038000C9698007C00EC1400806800F09E08108D6
:100390004D4A8900891809688007C00EC1400806C7
:1003A000800F002801D109F0E0FF687B1421484349
:1003B00086190021E0686A460691117006A9F8F7CF
:1003C00053FC6A46002010560F2802DD012001E090
:1003D000B2E000200699401807900220B072207900
:1003E000307260797072A068311DC01C06911F28A0
:1003F00001DA012009E0F8F737FC684600780028A8
:1004000004D0069806990068401C0860307A0628D7
:1004100014D201007944097949188F44020C0A0862
:10042000060400200DE0B4200BE0732009E0322028
:1004300007E00A2005E0062003E062E009F095FFEE
:100440000020217900295AD00221401806907168B5
:10045000103008180799089009180698081A0C9087
:100460000020F871F8F78DFB0446306007982018DB
:100470000002000AF060787A0C283CD0797A1420C7
:1004800041430E480818406808990290401800023D
:10049000000A0390707A6946887402A8FFF7B7FDD6
:1004A0000299039A091B121B09021202084B090A3E
:1004B000120A0C9899421ED8824215E03C0B00208B
:1004C000FFFFFF0000ED00E000E400E0440C00202E
:1004D000FFFF3F00500C0020180C0020F80A0020FD
:1004E000080B00203809002005D802990698081842
:1004F0000002000A3060F8790028B1D110E0042130
:10050000A3E704AA0199F8F7AFFB6846007C00282E
:1005100004D0019801990068401C08602078B072EE
:10052000687B162806D0687B401C68730B9808F01F
:100530003FFC42E00020F8E7F07F002801D009F0FE
:1005400014FF0120F077FE490F98087420780228E4
:1005500001D109F00AFFFA4E207930726079707289
:1005600032460C323146A068F8F77EFB0C2030563C
:100570000F2804DD1F3830733068401C30600C22B7
:10058000B256301DE16801908818C01C1F2802DA9D
:10059000012001990BE003AA0199F8F765FB684671
:1005A000007B002804D0019801990068401C086075
:1005B0002078B072E24901200875687B297B884267
:1005C00024D07C7A0C2C23D0F8F7DBFA14214C438E
:1005D000DC4961180A7C042A18D00A7C032A15D049
:1005E0004B6889681B1A081A1B020002D64A1B0AAC
:1005F000000A102B0AD31146934207D8884205D827
:10060000687B297B884201D0F8F707FB11B0F0BD69
:10061000687B297B8842F7D111B0F0BD10B500206E
:10062000F8F717FA10BD10B50120F8F712FA10BD4F
:10063000C64800787047F1B5009802281CD0C44C19
:10064000607A0C2801D109F090FE0026A6710125E0
:10065000E572607A03211422BA4F5043C019017425
:10066000F8F7E0FA009800280BD0012827D00328DB
:1006700075D009F07AFEF8BDB4480078F8F7A4FD0B
:10068000F8BDB448007F002801D009F06EFE657106
:10069000B04D00202E60F8F7EDF9A968481C04D091
:1006A000012300221846F8F719FA607A617A401C93
:1006B000C0B2142251437A5801219047F8BD01205D
:1006C000F8F7D8F9607900280DD0A2488068401C5E
:1006D00009D0607A617A401CC0B2142251437A5822
:1006E00006219047F8BD9B48007F012808D00228CA
:1006F00010D0032820D0042832D009F036FEF8BDEF
:100700002079002803D02671F8F791FAE570914816
:100710000677F8BD207A002802D1F8F711FB257280
:10072000607A617A401CC0B2142251437A58002189
:10073000904788480677F8BD864F0123397B786853
:100740000022411A1846F8F7C9F92079002803D089
:100750002671F8F76CFAE57002203877F8BD19E0D9
:100760007C4E217870680123411A00221846F8F760
:10077000B5F9207A002802D1F8F7E2FA2572607AFA
:10078000617A401CC0B2142251437A58002190472C
:100790003577F8BD607A617A401CC0B214225143AB
:1007A0007A58052189E710B5694C607A0C2801D187
:1007B00009F0DBFD607A617A401CC0B2142251431B
:1007C000604A52580421904710BDF0B583B0F8F745
:1007D000D8F900900C205E4C0290617A5E4801903E
:1007E0000C2920D0617A1420414356480918097C0D
:1007F000042918D0617A142251430818007C032878
:100800006FD0019900980A684968121A081A1202F2
:1008100000024D4B120A000A102A62D319469A426E
:100820005FD888425DD84B488068401C01D009F0F1
:100830009CFD00206071607A0C2807D16078002848
:1008400004D04648C178417081780170607A0C28E4
:1008500015D0617A142041433A480918097C0429CB
:100860000DD1617A0291617A01221423594309184A
:100870000A74617A59430818807C6072A272384DFC
:10088000687B297B374F884233D0374E287B142131
:1008900048438019007CC05D0128287B06D048436E
:1008A0008019007CC05D02282FD042E0142148430B
:1008B0008019807A01280AD0287B02211422504313
:1008C0008019007CC155287B162808D00AE0287BB7
:1008D0000021142250438019007CC15529E00020DA
:1008E00002E0CAE1287B401C2873687B297B884290
:1008F000CCD1134D287D00285FD0287CC15D012913
:100900003DD0C05D022845D04DE0287B14214843EE
:100910008019807A012801D009F027FD297B002069
:100920001422514389198872297B51438919097C02
:10093000C855287B142148438219287B484315E079
:10094000080B00203C0B0020FFFF3F00740000203C
:10095000440C0020240C0020340C002076000020E1
:10096000F80A0020170C0020380900208019017CAB
:100970000098FFF781F8287B1628B3D1AFE7A97A52
:10098000012904D00221C155002028750BE0002167
:10099000C15508E0A87A012801D009F0E6FC002042
:1009A000A872297CC855287D002806D0297CFE4ADB
:1009B0000098FFF761F80020287502980C281DD0D8
:1009C000014614204143F9480818017C012915D13A
:1009D00007210174F64D287E16283AD0287EE97D3D
:1009E000401C884201D109F0C0FC297E029868545D
:1009F000287E162831D0287E401C2876607A0C2864
:100A00007ED0A07A00287CD00020A072607A1421C9
:100A10004843E6494618E748B56873680246F668F1
:100A20007C32C36796605560E34D687E002816D01F
:100A30000226607A1422DD4950434018407B062884
:100A40001BD201007944097949188F440A14121005
:100A50000E0CE87D0028C6D0C7E70020CDE70426AD
:100A6000E7E700200CE0B4200AE0732008E0322021
:100A700006E00A2004E0062002E009F076FC0020EF
:100A80002873697E022901D0012910D12969009AB1
:100A900009188A1A1202120A422A08D90320687613
:100AA00032390802000A28613220287308E032280F
:100AB00006D2207A00280AD1F8F742F9012005E091
:100AC000207A002803D0F8F764F900202072BB498F
:100AD0001022487820700978012901D0032906D115
:100AE00001212171297B884201D9421A1032A37851
:100AF000002B00D0921C2179002904D1002B01E0A9
:100B000087E095E05BD09446AD4A00990092019A47
:100B1000176852687F1A511A3F0209023F0A090AF0
:100B2000BC451BD8A64A974218D8009A914215D8BE
:100B3000297B884223D92B69421A9A1A1202120A77
:100B4000101880190002000A2A616860002914D078
:100B5000032028770006000E3CD14AE000202071D7
:100B6000A070297B002923D0286940188019000231
:100B7000000A6860022028772CE00120E9E7814222
:100B80000BD92A69511889190902090A69600028D4
:100B900001D00420DDE70220DBE7002B01D109F0C2
:100BA000E4FB286980190002000A6860002004E064
:100BB000296989190902090A6960287719E0287BDF
:100BC00000280FD02969081880190002000A6860FF
:100BD0000220287728690123811900221846F7F797
:100BE0007DFF09E0286980190002000A6860002082
:100BF00028770120F7F73EFF607A142148436B49BC
:100C00000C2240188256012300206968F7F766FF1E
:100C10000EE00120F7F72EFF0020F7F72BFFF7F784
:100C200011FF207A002803D0F8F7B3F800202072D3
:100C3000A078002804D0F7F7FAFF0020E070A07039
:100C40006078002804D05D48C178417081780170D7
:100C50002079002806D000205849E0700978002942
:100C600000D120715248017EC07D814203D0554899
:100C70004078F8F7A9FA0120E07103B0F0BDF0B5B3
:100C8000514C0746607A83B00C2801D109F06DFB06
:100C9000607A1421454E48438019007C032801D016
:100CA00009F063FB444DA868401C01D009F05DFBCE
:100CB000607A1421484381190C20085600216A46A5
:100CC00000911171C01901AA6946F7F7CDFF6A4674
:100CD000042010560F2801DD012000E000200099BB
:100CE0004018696840180102090AA9606079002863
:100CF00004D0012300221846F7F7F0FE03B0F0BD40
:100D000030B5334C314A0B1AA34212D3451AA542CF
:100D10000FD3934203D9101A43185B1C09E0954284
:100D200004D9511A0818401C434202E009F01DFB87
:100D30000023184630BD10B50146012300220220D1
:100D4000F7F7CCFE10BD10B50220F7F793FE10BDEB
:100D500010B5F7F716FF10BDF0B51B4D0446E87A45
:100D600083B0002801D109F000FB642C68D3194935
:100D700000200246091B824162D31748417B007B59
:100D800081425DD10848007D002859D1687A14213C
:100D9000064F4843084EC519306801AA0019694634
:100DA000F7F762FF694619E0080B00203C0B0020B2
:100DB000200B0020B80B0020240C0020760000201F
:100DC000FFFF3F0074000020440C0020FF7F841EC2
:100DD0000020A107FF1FA107F80A002004200856E1
:100DE000002802DD0098401C0090A96800986B68FC
:100DF0000A18D21A12026E4B120A9A4220D8AA7C02
:100E00000C2A08D014235A43D2195268511A0902E5
:100E1000090A814214D3B068401C05D00120F7F7BD
:100E200029FE0020C043B060306800193060A86817
:100E3000009940180002000A7061012003B0F0BD63
:100E4000002003B0F0BDF0B50646401EC5B2142028
:100E5000584968434418207C002801D109F085FADC
:100E60005548017B407B81420CD0544A14234B43AC
:100E70009B181B7CB3420CD016290CD0491CC9B25C
:100E80008142F3D14E48017D002964D0007CB042FC
:100E900061D10020F0BD0021F1E7217C052905D0BA
:100EA000217C062902D0217C072928D10121217427
:100EB000C17D0023027E8A4221D00246565CAE42AA
:100EC00001D1012301E0002B04D0162911D04E1CC2
:100ED000965D565416290ED0491C167EC9B28E4214
:100EE000ECD1002B0BD0117E002906D0117E491EBB
:100EF00004E00026ECE70021EFE716211176617C83
:100F000000292AD06774C17D0023027E8A4224D042
:100F1000425CAA4201D1012301E0002B04D0162932
:100F200012D04A1C825C425416290FD0491C027E02
:100F3000C9B28A42ECD1002B0FD0027E0146002AB2
:100F400006D00A7E521E04E00022EBE70021EEE705
:100F500016220A7601E01B480027217C01299CD13A
:100F6000617C002999D10120F0BD30B505461420DF
:100F7000104A0521684380180174124C207E1628FF
:100F80000FD0207EE17D401C884201D109F0EDF9AF
:100F9000207E2554207E162807D0207E401C2076F7
:100FA00030BDE07D0028F1D0F2E70020F7E7000037
:100FB000FFFF3F003C0B0020F80A0020380900200A
:100FC000080B0020200B002070B51E490A68002A7B
:100FD00017D000231D4601244A68521C4A60092A82
:100FE00000D34D600E792246B2400E6816420AD0F8
:100FF00072B60B6893430B6062B6496801600020CB
:1010000070BD052070BD5B1C092BE5D309F0ADF95F
:10101000F7E701200C49800508607047EFF3108165
:10102000CA07D20F72B601218140064803681943EE
:101030000160002A00D162B6EBE70248002101609E
:10104000416070477C00002000E200E00120810741
:101050000860704701208107486070471048C068E9
:10106000C00700D0012070470D488068C00700D03D
:10107000012070470A484069C00700D0012070472E
:101080000748C069704706498A69D20306D589694D
:101090008907890F814201D10120704700207047E4
:1010A000000400408107C90E002808DA0007000F7D
:1010B00008388008BE4A80008018C06904E08008B3
:1010C000BC4A800080180068C8400006800F704746
:1010D000B94948788978884201D3401A02E0212230
:1010E000511A0818C0B27047B3492331487889783B
:1010F000884201D3401A02E02122511A0818C0B2D6
:101100007047AD49463148788978884201D3401A02
:1011100002E02122511A0818C0B27047A54910B543
:101120000C310868FF22120290430122D2031043BF
:101130000860A14900202331487088702339487025
:1011400088704631487088709C4807F011FE9B48B3
:10115000401C07F00DFEF7F7A7FF00F020F910BDC7
:1011600020207047B4E770B50C4605460026FFF70F
:10117000AFFF9149A04214D30A46203A00232046EB
:10118000641EE4B200280BD08878105C2870887840
:101190006D1C401CC0B288702128F0D18B70EEE726
:1011A000012600F0FCF8304670BD202070479BE718
:1011B00070B50C4605460026FFF796FF7E492331A1
:1011C000A04214D30A46203A00232046641EE4B20B
:1011D00000280BD08878105C287088786D1C401C23
:1011E000C0B288702128F0D18B70EEE7012600F0A4
:1011F000D6F8304670BD202101700020704710B530
:101200000446FFF77EFF2070002010BD70B50C462D
:101210000546FFF776FF68494631A04215D30A46D6
:10122000203A00232046641EE4B200280BD08878C0
:10123000105C287088786D1C401CC0B28870212812
:10124000F0D18B70EEE7002400E05D4C00F0A7F8D1
:10125000204670BD70B50C460546212901D909F01C
:1012600084F853484068103840B2FFF71BFFC6B2FD
:101270000D20FFF717FFC0B2864204D209F075F8BF
:1012800001E0F7F750FF21462846FFF76CFF0028E2
:10129000F7D070BDF8B507464848474C401E464E4B
:1012A0000078254646362335002806D1A978687887
:1012B000212200F069F800280ED0A1786078212260
:1012C00000F062F8002814D0B1787078212200F084
:1012D0005BF8002828D033E037496878C91C0F54E0
:1012E0006878401CC0B26870212829D1002068703D
:1012F00026E03149607820390F546078401CC0B234
:101300006070212801D1002060702C4F7F1E38783A
:10131000002815D0A1786078212200F035F8002847
:101320000ED0002038700BE02349707826310F541E
:101330007078401CC0B27070212801D100207070FC
:10134000A9786878212200F01FF800281BD0A17826
:101350006078212200F018F8002814D0B178707855
:10136000212200F011F800280DD0F7F7C0FE134835
:1013700007F006FD01214903884201D008F0F5FF7E
:101380000E4807F015FDF8BD401C884205D090427C
:1013900001D1002901D0002070470120704710B50D
:1013A000064807F0EDFC002801D1F7F78FFE10BDCD
:1013B00000ED00E000E400E0740C00208500002057
:1013C000072000000C4908784A78401CC0B29042BF
:1013D00000D008707047094A074820BF40BF20BFAF
:1013E0004178037843701368002B02D103788B4255
:1013F000F3D00020704700008700002000E200E0EA
:10140000F0B50121184A08031060184A0023136040
:10141000174B1860174803690569DB43DB06DB17C8
:10142000102425430561144D6960144E31605B1C26
:1014300000E020BF1768002FFBD0002B02D103690A
:10144000A34303610E4880687160A96000211160A8
:101450000121074A09031160F0BD10B50446FFF7EA
:10146000CFFF2060002010BD80E100E000C10040FF
:1014700080E200E000ED00E000C3004000C000405A
:1014800000C50040FEB5EC4C07466068FF213E01F8
:1014900081552178FF2913D009010831415832467E
:1014A000491E083209020192090A805800F0BAF96F
:1014B000002802D02478254615E0616820788855F8
:1014C0002770FEBDDC484268019811582801009041
:1014D0000830105800F0A6F9002806D1D6482C464E
:1014E000416800980D5CFF2DECD1D3482101406884
:1014F00085554754FEBD70B5CF4A04460020157A85
:1015000053680AE00201561C9E5DA64203D10C32CC
:101510009A588A4204D0401CC0B28542F2D8FF20BB
:1015200070BD10B5FFF714FCC34C0146207862680B
:1015300000010830105800F075F9012807D920780B
:101540006168000108300858FFF7F5FB10BDFFF790
:101550006FF8F7F739FE10BDF8B5B74F3E78FFF7D3
:10156000F7FB0146FF2E68D0340125467868083520
:10157000405900F057F9022802D9786840595AE0DA
:10158000AD494868025D0A70A11C425C002A0CD07B
:10159000521E425441590122D20589180902090AF2
:1015A00041513046FFF76EFF30E0631CC25C009291
:1015B000221D94468258002A10D001239B029A4291
:1015C0000FD99205920D43595703DB191B021B0AD1
:1015D00043516346C3589A1A920A09E0FF21C15445
:1015E0000AE0435952039A181202120A4251002289
:1015F00042543046FFF746FF8F480C344168C268BA
:101600000098095980001258009890478A4C207819
:10161000FF2812D0FFF79CFB01462078626800018A
:101620000830105800F0FEF8012896D9207861683B
:10163000000108300858FFF77EFBF8BDF0B51D46E5
:1016400014460E460746FF2B01D308F08EFEA00776
:1016500001D008F08AFE7848FF21C7604460057217
:101660000674017000224270104604E00201521C10
:10167000401CA154C0B2A842F8D3F0BD70B56E4C66
:1016800006466578207C854201D308F06EFEE0684E
:10169000A90046506078401C6070284670BDFFB5B8
:1016A00081B01D46FF24FFF753FB634F0646797850
:1016B0000198814201D808F058FE5F480021037A62
:1016C000406810E00A019446521C825CFF2A25D033
:1016D000019FBA4205D162460C328758029A97425E
:1016E0001ED0491CC9B28B42ECD8FF2C18D0210166
:1016F0004A1C019B83540B460C33029AC250039B35
:101700004D4F0022012B0ED00B1DC25001239B0216
:101710009D4216D9AA05920D08D008E00C46E0E7D4
:10172000FF2005B0F0BD0B1DC550EFE71A4653036F
:101730009B190E461B0208361B0AAA1A8351920AED
:1017400009E0002D00D101256B039B191D022D0A14
:101750000B460833C550891C42543D463E7820460E
:10176000FFF790FE2878B04201D0FFF7DAFE01982B
:10177000D7E770B50C460546FFF7EAFA064621465C
:101780002846FFF7B8FEFF2817D02B4D040120464E
:10179000696808300858314600F044F8012109030F
:1017A00040186968A41C095D400B002901D089021A
:1017B0000818002800D1012070BD002070BDF3B5CD
:1017C00081B00F460198FFF796FEFF2819D01A4EF8
:1017D000357871682A462C4604E0844205D02546B7
:1017E0002301CC5CFF2CF8D10BE0FF2C09D0A542E3
:1017F0000BD11001085C3070FF2804D0FFF791FE78
:1018000003E00020FEBDFFF79EFA39460198FFF77E
:10181000B0FF22017168FF23541C0B558A5C2B0119
:10182000CA54FEBD401A00020121000AC9058842BF
:1018300000D9002070470000C00C00200348044A73
:101840000168914201D10021016070478C000020A5
:10185000BEBAFECA3B480021017041701021817060
:10186000704770B5064614460D460220F1F778FB26
:1018700001203449344A0870E41E146196605560B2
:1018800070BD10B50220F1F76BFB2E4901200870E6
:101890002E48002101604160816001202C49C00573
:1018A000486010BD10B527480178002917D00121E4
:1018B000274AC905916025490B680022002B05D0F5
:1018C0004B68002B02D08968002902D04270102199
:1018D00003E0012141701F490968817002700020F6
:1018E000F1F73EFB10BD17480178002912D01748C8
:1018F000016800290AD00168002905D04168002943
:1019000002D08068002803D0002070470220704772
:1019100001207047407870470A48017800290FD0AD
:101920000A480168002905D04168002902D0806872
:10193000002801D01020704706480068C0B27047E8
:10194000807870479000002000F5004000F10040D2
:1019500000F5014000F400402D4800210170417065
:10196000704770B5064614460D460120F1F7F8FAA7
:1019700027490120274B08709E60DC601D6170BD07
:10198000F8B504460120F1F7EBFA2149012008706F
:1019900020494C60204900264E6003211F4D090656
:1019A000A9601F4F002C08D0012C01D008F0DDFCED
:1019B0003E60032000066860F8BD38600120000624
:1019C000F9E710B51248017800290ED00321134A17
:1019D0000906916010494A680021002A03D0114A83
:1019E0001268427000E0417001700020F1F7B8FA0F
:1019F00010BD07480178002907D007484068002833
:101A000002D008480068C0B27047407870470000B4
:101A10009300002000F5004000F1004000F5014077
:101A200000F2004000F4004070B5FF4D00246C70DF
:101A30002C706C616C72AC720120E8726C776C6215
:101A4000FA48EC6207F094F9002801D008F08DFC08
:101A50002C7670BD00B5F649002804D0012806D0C8
:101A600008F083FC00BDF3484861F34802E0F34806
:101A70004861F348886100BDF0B50125F1490226AF
:101A80000E60F1490027CF63CD63F049C96A0907A9
:101A90000DD4EF49CB6AEF4A53620B6B93624B6BE9
:101AA000D3628B6B1363C96BD30519435163E04C4D
:101AB000002820D0012822D008F057FCE648A06377
:101AC000FF2004306063256303202061E3499620F2
:101AD0004860D549182008560722D243811A9042FF
:101AE0002FD011DC163135D00A2931D00E292DD056
:101AF00012290FD128E0CF486061CF4802E0CF48DB
:101B00006061CF48A061D9E7001D18D0042814D027
:101B100008280FD008F029FCD249D1488860D34862
:101B2000D1494160D2490160D2480660D2491020B3
:101B30004860F0BD0420E060EEE7E760ECE7FC20E1
:101B400000E0F820E060E7E7F420FBE7F020F9E7A9
:101B5000EC20F7E7D820F5E710B50C460146C7485A
:101B600008F0F9FCB048047210BDAF48407F7047E0
:101B7000AD4A517010707047F0B504460D4650796B
:101B8000117900020843690009190884501C0146B4
:101B90000E78012730464E78360230438E78C97869
:101BA0003604304309060843117800020843A900AF
:101BB0006050284608303E468640002B09D0012B55
:101BC00001D008F0D2FB206B3043AF403843206394
:101BD000F0BD206BB043F8E730B50D460446082948
:101BE00001D908F0C2FB0022002D0CD9A4489100B5
:101BF000635809180B6053001B191B8C0B62521C95
:101C0000D2B2AA42F3D3206B9E49086030BD10B512
:101C100004460722D2430830854994421BD008DC91
:101C2000163020D00A281CD00E2818D0122806D131
:101C300013E0201D0DD0042808D0082804D008F097
:101C400094FB7948047610BD042000E00020C860B1
:101C5000F7E7FC20FBE7F820F9E7F420F7E7F020AE
:101C6000F5E7EC20F3E7D820F1E78748007A7047E2
:101C70006F49C2784A6202461378184653781B02AD
:101C800018439378D2781B041843120610430002BD
:101C9000C8617047252808D0262808D0272808D0F2
:101CA00041000A2807D8091D06E0022105E01A2193
:101CB00003E0502101E0891DC9B25D4A9160674986
:101CC00048617047584948617047F8B5002813D0FB
:101CD0000220554E6D4AB07203231360614C604A76
:101CE000626001276A4D002908D001290CD0022921
:101CF0001FD008F03AFBF8BD0120EAE7012801D027
:101D00006F60F8BD2F60F8BD47490128C96A04D04B
:101D1000022808D008F029FBF8BD01200005014386
:101D2000F1626060F8BD012040050143F16260602E
:101D3000F8BD7069002801D108F017FB7169706A5D
:101D4000401854498860494853498160B17A012953
:101D500017D05249C1600120F16AC0030143F1620A
:101D60004A490E68444A10209060002008603D4AAD
:101D700009149160FF216A461170494C20612F615E
:101D800004E0C560E7E71078401E10701078002866
:101D900002D020690028F6D01078002801D108F080
:101DA000E4FA0020E060206160606061A061374873
:101DB000066001142B4841602F4A10215160C9026E
:101DC0004160F8BDF8B5314801688F082A49BF0065
:101DD0004A68D206D60F10228A6000240460214887
:101DE0001F498160FF20694608702D4D2C612849EC
:101DF0000120086103E069460878401E08706846C3
:101E00000078002802D028690028F4D068460078BD
:101E1000002801D108F0A9FA2C610348012144727D
:101E20008472C17219483DE0D40C0020040D0020DA
:101E30000015004006010200250003020501030011
:101E40001F00030280E100E0C01F0040800000107E
:101E5000C0000010001700405B0600004015004065
:101E60000040000400F501404080004080F5014042
:101E70001011004080E200E000130040D60C00206A
:101E80000016004040160040F40C002000120040F4
:101E90000010004040850040488100400410004090
:101EA000001100400760002E02D0F8491020486061
:101EB000F8BD01460A7810464A78120210438A7823
:101EC000C97812041043090608430002F049000AC9
:101ED000C8637047EF4902200860EF490860704707
:101EE000EE49022008607047ED490870704710B550
:101EF000EC4806F045FF002801D008F036FA10BD86
:101F000010B5E84806F054FF10BDE149486070473D
:101F100030B5E54C0546606AA84201D308F025FAC1
:101F200001202073E149002025614860E0484560B8
:101F30000120E16A80050143E162DE49486030BD6D
:101F4000D94802210173C6210161D84A002151609C
:101F5000416AD74AC63151600121C26A89050A43E4
:101F6000C262D448416070470121D248890581602E
:101F7000CD48C26A8A430021C26201737047CE48CD
:101F800001214160C160C94900204860C8494860DA
:101F9000C54948627047C94940200862C8490A6873
:101FA00002430A607047C6480168402291430160BD
:101FB000C249002008627047C1480168102291435D
:101FC0000160C049012088617047BF490020C86195
:101FD000BB4801681022114301607047BA49CA69C1
:101FE000012A01D000207047B44A92685206520E6E
:101FF000524202700020C8610120704730B50C00C9
:10200000054601D108F0B1F9E00703D0012C01D059
:1020100008F0ABF9002D0BD00221A3480129417231
:10202000C472A74806D0022909D008F09EF930BD35
:102030000121F2E7016804221143016030BD01680B
:1020400008221143016030BDF8B5974C0025E17AB4
:102050008A0701D5420712D4CA0606D59B4A537A8D
:10206000002B02D0927A002A09D00A0702D5227FDB
:10207000002A04D1490703D5617F002900D1012539
:10208000677A002201238E49002F1AD002263040A1
:1020900028433CD0086886087C48B6004568ED06B1
:1020A000ED0F1027876000200860824A8849916000
:1020B000FF216A461170844F38618249012008610E
:1020C0000CE07C4D8248A8600868800880000860A9
:1020D000A272E372F8BD1078401E107010780028CC
:1020E00002D038690028F6D01078002801D108F015
:1020F0003CF9002038616072A0720120E0727048E3
:102100000660002DE6D0614810214160F8BD012F26
:1021100004D0022F0AD008F028F9F8BD0868042579
:10212000A84308606272E372A372F8BD08680825CC
:10213000A84308606272E372A672F8BDF8B55A4807
:102140005C49C26A8A600021C162017B574D002947
:1021500002D06968012909D000235B4C216901295B
:1021600006D00022817A012904D006E00123F4E799
:102170004022F7E7E668012E04D000261643012925
:1021800002D004E02026F9E76268012A05D0002287
:102190003243504F022902D007E01022F8E73E6890
:1021A000012E02D1E668012E04D000261643022932
:1021B00002D007E00826F9E73A68002A02D1E2686F
:1021C000012A04D000223243022902D005E0042271
:1021D000F9E7002B01D0022300E00023134302297A
:1021E00007D16068012804D16868012801D001275F
:1021F00000E0002738481F4301680906090E02D095
:102200006169012900D00021304E3172006800065A
:10221000000E02D0A069012800D00020707227486B
:10222000006A002803D0FFF75EFB012800D00020E1
:10223000B0720026E660266166606661A6611B4892
:1022400046601B493C464868174D28620A686A6226
:10225000A97A022909D16978002906D00C4B5B685C
:102260001B780B40297899430DD02E770C4FE1074E
:1022700039D03978032931D002292FD003F0D3F88F
:102280000121686A49E001212977EFE70013004046
:102290000015004080E100E080E200E000E100E0A5
:1022A00095000020040D0020D40C00204081004047
:1022B0004085004000F5014000800040401500408E
:1022C000001200400010004000110040F40C0020FB
:1022D00000400004001400404016004002F068F97D
:1022E0000121686A24E0A0060ED53878032806D0BC
:1022F000022804D00221104603F0A4F80FE00221C6
:10230000104602F056F90AE0A00708D538780328ED
:102310000CD002280AD00021104603F093F84B4855
:102320000078002807D0022805D017E000211046C9
:1023300002F03FF9F3E7464F79680622A81C0931FD
:1023400007F05CFE002807D1287A79680978C90966
:10235000884201D1012000E0002068772046FFF785
:1023600073FE3A480078002826D0012837D002288A
:1023700048D0032833D007F0F8FFA87A02281AD1F2
:10238000287B002817D033494E60022857D00128F7
:1023900001D007F0EAFF696A2869884201D807F08E
:1023A000E4FF2D48296941600120E96A8005014365
:1023B000E9622A494860F8BDA00701D500F02EFC6B
:1023C000200702D5012000F060FC600702D5002044
:1023D00000F05BFCA006D0D500F0DCFBCDE7A00749
:1023E00001D505F0D8FB200702D5012005F04DFCF2
:1023F000600702D5002005F048FCA006BDD505F019
:10240000FFFBBAE7A007BF27002802DA3C4001F033
:10241000BBFB200703D53C40012001F08BF860078F
:1024200003D53C40002001F085F8A00602D53C40D1
:1024300001F044FB6006A0D501F078F89DE729691A
